:020000040000FA
:061000006FEF6AF0120020
:0610080074EF24F0120059
:0610180018EF39F0120090
:06102A000400A5D5000042
:1010300000060000E10000009CD50000B70E000093
:10104000090000009AD50000F3050000020000002E
:0C10500040D50000800200005A000000A3
:04105C00020100008D
:10106000000000013200000000000180004D00007F
:10107000000200000000000001320000000000013A
:10108000A700FBFFDFFF015700EFFF0400014E0048
:10109000F2FF0700014C00F3FF0800014A00F5FFD2
:1010A0000A00014400F8FF0B00014800FAFF0D00A0
:1010B000014E00FCFF0F00015000FFFF1000013245
:1010C0000000000A00012E000200090001330002A6
:1010D000000A00012D0004000800012D0004000892
:1010E00000012F0005000800013100070007000182
:1010F0002E00070006000132000800060001330040
:10110000090005000136000A0004000134000A004D
:1011100003000139000B000300013D000C00020038
:101120000141000D0001000146000E0001000146D2
:10113000000E00FFFF0141000D00FFFF013D000C0C
:1011400000FEFF013E000C00FDFF0139000B00FD19
:10115000FF0136000A00FCFF0133000900FBFF011C
:1011600032000800FAFF0135000800F9FF012E00E7
:101170000600F9FF012E000600F9FF012D00040012
:10118000F8FF012D000400F8FF012E000200F7FF18
:10119000012E000200F7FF0132000000F6FF012DD2
:1011A000000000F7FF012E00FEFFF7FF012900FEFF
:1011B000FFF8FF012B00FDFFF8FF012F00FBFFF8F8
:1011C000FF012B00FBFFF9FF013100F9FFF9FF01DF
:1011D0002E00F9FFFAFF013200F8FFFAFF01330099
:1011E000F7FFFBFF013600F6FFFCFF013900F5FFBA
:1011F000FDFF013900F5FFFDFF013D00F4FFFEFF9B
:10120000014100F3FFFFFF014600F2FFFFFF013243
:1012100000F6FF010001C60200008E00015B00EE37
:10122000FFFEFF015100F0FFFDFF014800F3FFFA50
:10123000FF014100F5FFF9FF013C00F7FFF8FF0156
:101240003A00FAFFF6FF013600FCFFF6FF013C0012
:10125000FFFFF4FF0128000100F8FF012900020050
:10126000F8FF0126000300F9FF012B000500F9FF3C
:10127000012E000700FAFF012F000800FBFF0133D9
:10128000000900FBFF013F000C00FCFF0100000013
:101290000000000201000000000001320000000018
:1012A0000001CE003F006A000200000000000001C3
:1012B000320000000000011202000096FF01410010
:1012C0000D000100013E000C0003000134000A0083
:1012D0000300012F00080005000140000A0008007B
:1012E000013D0007000A00011B0002000500011B70
:1012F0000002000500013C0001000C00013700FF66
:10130000FF0B00012F00FDFF0900013600FAFF0965
:1013100000013500F9FF0800013D00F6FF0700015C
:101320003C00F5FF0500014400F3FF040001460006
:10133000F2FF0100010000000000000201000000B7
:1013400000000132000000000001900164FF4AFF2C
:10135000020000000000000132000000000001A2B5
:1013600000FBFFE0FF012D00F7FFFFFF012600F962
:10137000FFFDFF011D00FBFFFDFF012000FBFFFC47
:10138000FF012700FBFFFAFF012B00FDFFF8FF0123
:101390002E00FEFFF7FF013200FFFFF6FF013200D3
:1013A0000100F6FF0133000200F6FF012B000300ED
:1013B000F8FF0127000500FAFF012A000600FAFFE6
:1013C000012B000700FBFF012B000800FDFF012F90
:1013D000000900FDFF0160001300FEFF019B001FDC
:1013E000000000012B00F9FF0500012A00FAFF06AA
:1013F00000012700FBFF0600012800FCFF07000199
:101400002400FCFF0600012400FEFF070001280065
:10141000FFFF0800012800FFFF0800012D00010068
:101420000900012D0001000900012F00030009003F
:10143000012D000400080001280004000700012E0F
:101440000006000700012E00070006000132000818
:101450000006000133000900050001310009000405
:10146000000136000A0004000134000A00030001F4
:101470006B0015000400017300170001000150000B
:10148000100000000151001000FEFF0148000E0096
:10149000FDFF014A000E00FBFF014A000E00FBFFAA
:1014A0000141000B00F9FF0140000A00F8FF01397B
:1014B000000800F8FF013D000700F6FF013C0005B1
:1014C00000F5FF0138000200F5FF0141000100F3C3
:1014D000FF0128000000F8FF012900FEFFF8FF01CE
:1014E0002400FEFFF9FF012800FCFFF9FF0128009E
:1014F000FCFFF9FF012E00FAFFF9FF012E00F9FFB2
:10150000FAFF012B00F9FFFBFF0187001B00000021
:101510000196000000E2FF01DE033AFF0000017DBA
:1015200000E7FF0000016900EBFF0200015600EF39
:10153000FF0300014400F3FF0400013800F6FF053B
:1015400000013D00F6FF0700013500F8FF0700012C
:101550003D00F9FF0A00013A00FAFF0A00013F00CE
:10156000FCFF0C00013D00FEFF0C00014600FFFFE8
:101570000E0001500001001000014E0004000F0099
:1015800001480006000D0001440008000B00012086
:1015900000040005000127000600050001220006E6
:1015A00000030001260007000300012400070002D9
:1015B000000129000800020001550011000100018E
:1015C00000000000000002010000000000013200E5
:1015D0000000000001EA008A00E5FF0200000000B0
:1015E000000001320000000000016900EBFFFFFF76
:1015F000015B00EEFFFDFF014F00F1FFFBFF012249
:1016000000FAFFFDFF012200FAFFFDFF013C00F799
:10161000FFF8FF013900F9FFF7FF013400FDFFF685
:10162000FF013300FEFFF6FF0138000200F5FF0165
:1016300034000300F6FF0139000700F7FF013C000A
:101640000900F8FF011D000500FDFF01260007004D
:10165000FDFF014A000E00FBFF015B001200FDFFD1
:101660000164001400FFFF01640014000100015632
:101670000011000300014F000F0005000145000CA0
:10168000000700013C0009000800013900070009BB
:10169000000131000400090001370001000B0001C6
:1016A0003200FFFF0A00013600FCFF0A000139008A
:1016B000F9FF0900013C00F7FF0800014300F4FFB7
:1016C0000600014A00F2FF0500015600EFFF03008B
:1016D000015F00EDFF0100010000000000000201B9
:1016E00000000000000132000000000001770176D8
:1016F000FF4EFF0200000000000001320000000069
:101700000001A200FBFFE0FF012D00F7FFFFFF013A
:101710002600F9FFFDFF011D00FBFFFDFF0120007A
:10172000FBFFFCFF012700FBFFFAFF012B00FDFF81
:10173000F8FF012E00FEFFF7FF013200FFFFF6FF6A
:101740000132000100F6FF0133000200F6FF012B19
:10175000000300F8FF0127000500FAFF012A000638
:1017600000FAFF012B000700FBFF012B000800FD22
:10177000FF012F000900FDFF0160001300FEFF01C3
:101780009B001F000000012B00F9FF0500012A004B
:10179000FAFF0600012700FBFF0600012400FCFF02
:1017A0000600012800FCFF0700012400FEFF0700DF
:1017B000012800FFFF0800012800FFFF0800012D9D
:1017C0000001000900012D0001000900012F0003A4
:1017D00000090001280004000700012D0004000892
:1017E00000012E0006000700012E00070006000180
:1017F0003200080006000133000900050001310035
:10180000090004000136000A0004000134000A0047
:101810000300016B001500040001730017000100B4
:101820000150001000FFFF0150001000FFFF0148B1
:10183000000E00FDFF014A000E00FBFF014A000EF2
:1018400000FBFF0141000B00F9FF0140000A00F816
:10185000FF0139000800F8FF013D000700F6FF0115
:101860003C000500F5FF0138000200F5FF014100D2
:101870000100F3FF0128000000F8FF012900FEFF2E
:10188000F8FF012400FEFFF9FF012800FCFFF9FF2B
:10189000012800FCFFF9FF012E00FAFFF9FF012EDD
:1018A00000F9FFFAFF012B00F9FFFBFF0187001B86
:1018B0000000000196000000E2FF01DE033AFF0095
:1018C00000017D00E7FF0000016900EBFF0200015D
:1018D0005600EFFF0300014400F3FF04000138004D
:1018E000F6FF0500013D00F6FF0700013500F8FF97
:1018F0000700013D00F9FF0A00013A00FAFF0A0063
:10190000013F00FCFF0C00013D00FEFF0C00014602
:1019100000FFFF0E0001500001001000014E000406
:10192000000F0001480006000D0001440008000BF4
:10193000000120000400050001240006000400014D
:101940002400060004000126000700030001240013
:1019500007000200012900080002000155001100E3
:101960000100010000000000000201000000000072
:101970000132000000000001EA008A00E5FF0200D9
:10198000000000000001320000000000016900EBCF
:10199000FFFFFF015B00EEFFFDFF014F00F1FFFBCA
:1019A000FF012200FAFFFDFF012200FAFFFDFF0107
:1019B0003C00F7FFF8FF013900F9FFF7FF013400A1
:1019C000FDFFF6FF013800FEFFF5FF0133000200C6
:1019D000F6FF0134000300F6FF0139000700F7FFAE
:1019E000013C000900F8FF011D000500FDFF012872
:1019F000000700FCFF0149000E00FCFF015B001224
:101A000000FDFF0164001400FFFF016400140001E9
:101A10000001560011000300014F000F00050001F6
:101A200045000C000700013C0009000800013900D6
:101A3000070009000131000400090001370001001E
:101A40000B00013200FFFF0A00013600FCFF0A0014
:101A5000013900F9FF0900013C00F7FF08000143CC
:101A600000F4FF0600014A00F2FF0500015600EFF6
:101A7000FF0300015F00EDFF010001000000000016
:101A8000000201000000000001320000000000011F
:101A90008D0189FF32FF02000000000000013200CA
:101AA0000000000001960000001E00012C063C0111
:101AB000000001A5000000DFFF01300290FF0000E0
:101AC000012B000700FBFF012A000600FAFF012797
:101AD000000500FAFF0127000500FAFF01260003B8
:101AE00000F9FF0124000200F9FF0124000200F9BF
:101AF000FF0128000000F8FF012D000000F7FF01A2
:101B00002900FEFFF8FF012900FEFFF8FF012D006C
:101B1000FCFFF8FF012F00FBFFF8FF012B00FBFF8C
:101B2000F9FF012E00F9FFFAFF012B00F9FFFBFF7F
:101B3000012F00F8FFFBFF013100F7FFFCFF01362A
:101B400000F6FFFCFF013400F6FFFDFF013900F550
:101B5000FFFDFF013C00F4FFFFFF017800E8FFFEFE
:101B6000FF014600F2FF0000014700F2FF02000102
:101B70003D00F4FF0200013D00F4FF0200013B00C4
:101B8000F5FF0400013600F6FF0400013300F7FF03
:101B90000500013300F7FF0500013100F9FF0700E0
:101BA000012E00F9FF0600012B00FBFF0700012BAF
:101BB00000FBFF0700012D00FCFF0800012400FED0
:101BC000FF0700012900FEFF0800012D00000009A9
:101BD000000128000000080001290002000800019F
:101BE000260003000700012600030007000127006C
:101BF00005000600012A0006000600012E0007006D
:101C00000600012F0008000500019100E3FF00001D
:101C1000020100000000000132000000000001C1CC
:101C2000007400000002000000000000013200000B
:101C3000000000015F00EDFFFFFF015000F0FFFF1B
:101C4000FF014800F2FFFDFF013600F6FFFCFF0137
:101C50002800F9FFFCFF012700FAFFFBFF0120002D
:101C6000FBFFFCFF012300FBFFFBFF012200FDFF48
:101C7000FAFF011B00FEFFFBFF012000FEFFFAFF41
:101C80000123000000F9FF0132000100F6FF0131DD
:101C9000000400F7FF0139000700F7FF0140000AC8
:101CA00000F8FF0145000C00F9FF0154001000FB93
:101CB000FF0156001100FDFF0169001500FFFF0143
:101CC000690015000100015B0012000300014F00D4
:101CD0000F0005000122000600030001220006009B
:101CE0000300013C0009000800013500070008005E
:101CF00001360004000A0001320001000A0001322E
:101D000000FFFF0A00013600FCFF0A00013900F95C
:101D1000FF0900014000F6FF0800014300F4FF0640
:101D200000014F00F1FF0500015600EFFF03000125
:101D30006400ECFF0100010000000000000201004F
:101D40000000000001320000000000011001FFFF50
:101D50005DFF0200000000000001320000000000F2
:101D6000014B000F00FFFF0146000E00FFFF01487E
:101D7000000E00FDFF013E000C00FDFF013B000BCB
:101D800000FCFF013C000B00FBFF0136000900FADC
:101D9000FF0135000800F9FF012A000600FAFF01E3
:101DA0002B000500F9FF0128000400F9FF012800BD
:101DB0000400F9FF012B000300F8FF0129000200D5
:101DC000F8FF0128000100F8FF012D000000F7FFD7
:101DD0000132000000F6FF012E00FEFFF7FF012E8A
:101DE00000FEFFF7FF012B00FDFFF8FF012F00FBB6
:101DF000FFF8FF012B00FBFFF9FF012E00FAFFF9AE
:101E0000FF013200F8FFFAFF013200F8FFFAFF018C
:101E10002F00F8FFFBFF013800F6FFFBFF01340045
:101E2000F6FFFDFF013900F5FFFDFF013D00F4FF66
:101E3000FEFF014100F3FFFFFF014100F3FF00003F
:101E4000016900EBFF0000016000EDFF020001529C
:101E500000F0FF0400014A00F2FF0500014300F416
:101E6000FF0600013D00F6FF0700014000F7FF09F3
:101E700000014000F8FF0A00013F00FAFF0B0001DB
:101E80003C00FBFF0B00013D00FEFF0C00013C008D
:101E9000FFFF0C0001320000000A00012E000200CA
:101EA0000900012E0002000900012D0004000800B5
:101EB000012D0004000800012F0005000800012E7C
:101EC000000700060001310007000700013200088A
:101ED000000600013300090005000136000A000475
:101EE000000134000A000300013E000C0003000161
:101EF0003D000C0002000146000E000100014600FA
:101F00000E000100010000000000000201000000BE
:101F10000000013200000000000139000000DEFF77
:101F20000200000000000001320000000000016912
:101F300000EBFFFFFF015B00EEFFFDFF014F00F133
:101F4000FFFBFF012200FAFFFDFF012400FAFFFC66
:101F5000FF014000F6FFF8FF013D00F9FFF6FF0129
:101F60003600FCFFF6FF013C00FFFFF4FF013C00E0
:101F70000100F4FF0136000400F6FF013D000700F8
:101F8000F6FF0140000A00F8FF0124000600FCFFF4
:101F90000122000600FDFF0154001000FBFF015B61
:101FA000001200FDFF0169001500FFFF016400142D
:101FB00000010001560011000300014F000F000551
:101FC00000012600070003000120000500040001B5
:101FD00043000A00090001390007000900013B0025
:101FE00004000B0001370001000B00013C00FFFF63
:101FF0000C00013600FCFF0A00013D00F9FF0A0059
:10200000014000F6FF0800012000FBFF040001264C
:1020100000F9FF0300014F00F1FF0500015B00EE36
:10202000FF0300016400ECFF01000100000000005C
:102030000002010000000000013200000000000169
:10204000BC01B0FF02FF02000000000000013200EE
:102050000000000001AC00DEFFFBFF014300FDFFBC
:102060000D00013C00FFFF0C0001280001000800EA
:102070000123000100070001240002000700011DE8
:102080000003000500011900030004000120000501
:1020900000040001190004000300011D00050003F5
:1020A00000012300070001000133000A00020001C3
:1020B00091001D00010001940284000000017300E2
:1020C000000017000196001E0000000173000000D0
:1020D000E9FF011D013900000001C9001700DFFF01
:1020E000019001B0FF000001A0000000E0FF019698
:1020F00000E2FF000001A00000002000019E027A23
:10210000FF0000014600F2FF0000012300F9FFFF7D
:10211000FF011D00FBFFFDFF011500FDFFFDFF019D
:102120001B00FEFFFBFF011E00FFFFFAFF0147003F
:102130000200F2FF010000000000000201000000A8
:102140000000013200000000000158075AFF5C0443
:10215000020000000000000132000000000001C782
:1021600001A8FFE9FF0141000000F3FF015C014409
:1021700000F1FF014C00F1FFFEFF011001CBFFF465
:10218000FF0141000000F3FF01C7015800E9FF0112
:102190003C0000000C00010701CDFF0D00015700BD
:1021A000EFFF040001570011000400010501330096
:1021B0000B00013C0000000C00010601CDFF0C00EB
:1021C000016100EDFF04000161001300040001063D
:1021D0000133000C0001410000000D00010000006F
:1021E00000000002010000000000013200000000B9
:1021F0000001FF00A8FF83FF0200000000000001B3
:1022000032000000000001C6015800160001410024
:102210000000F3FF010501CDFFF5FF016200EDFFB6
:10222000FBFF0161001300FCFF0105013300F5FF16
:102230000141000000F3FF010501CDFFF5FF01574B
:1022400000EFFFFCFF0157001100FCFF0107013305
:1022500000F3FF013C000000F4FF01C701A8FF17D5
:102260000001410000000D0001100135000C0001CB
:102270004C000F000300015C01BCFF0F0001410096
:1022800000000D000201000000000001320000000B
:10229000000001AC00000099FF02000000000000F7
:1022A0000132000000000001C60158001600013C88
:1022B000000000F4FF010601CDFFF4FF016200ED14
:1022C000FFFBFF0160001300FDFF0106013300F476
:1022D000FF0141000000F3FF010501CDFFF5FF0103
:1022E0005700EFFFFCFF0157001100FCFF01070141
:1022F0003300F3FF013C000000F4FF01C701A8FF19
:10230000170001410000000D0001100135000C0014
:10231000014C000F000300015C01BCFF0F000141F4
:102320000000000D0002010000000000013200006A
:10233000000000019B000000A3FF0200000000005D
:1023400000013200000000000155001100000001F2
:1023500046000000F2FF015500EFFF0000014600BB
:1023600000000E0002010000000000013200000029
:1023700000000197001C00AAFF02000000000000FE
:1023800001320000000000014100FFFFF3FF0124C3
:1023900000F9FF0200012000FAFF0200011900FC11
:1023A000FF0300012000FBFF0400011D00FDFF05ED
:1023B00000011B00FEFF0500011B00FEFF050001E0
:1023C0001E00000006000128000100080001240092
:1023D000020007000124000400060001230005009C
:1023E000050001240006000400012B000800030082
:1023F000012E00090002000132000A00000001372E
:10240000000B000000012E000900FEFF012B000858
:1024100000FDFF0128000700FCFF0123000500FB71
:10242000FF0124000400FAFF0126000300F9FF0168
:1024300023000000F9FF0123000000F9FF01220042
:10244000FDFFFAFF012200FDFFFAFF012700FAFF5E
:10245000FBFF012400FAFFFCFF012B00F8FFFDFF4A
:10246000012E00F7FFFEFF013700F5FFFFFF01150A
:1024700000FCFF010001130100003700012300F9F7
:10248000FFFFFF012000FAFFFEFF011B00FBFFFE24
:10249000FF011600FCFFFEFF011900FDFFFCFF011C
:1024A0001500FDFFFDFF011500FFFFFCFF011900F6
:1024B000FFFFFBFF011E000100FAFF0120000400E6
:1024C000FBFF0123000500FBFF012B000800FDFFBF
:1024D00001000000000000020100000000000132C5
:1024E0000000000000015000190029000200000057
:1024F0000000000132000000000001CD000000D704
:10250000FF012D0009000100012600070003000162
:102510001C00040004000115000300030001160064
:102520000200040001190000000500011400000071
:102530000400011600FEFF0400011200FEFF03006C
:10254000011500FDFF0300011900FCFF0300011647
:1025500000FCFF0200011900FBFF0100011900FB54
:10256000FF01000100000000000002010000000067
:102570000001320000000000019700C4FFBCFF0210
:1025800000000000000001320000000000013E00D9
:10259000FDFFF4FF011900FBFFFFFF011900FCFF25
:1025A000FDFF011D00FDFFFBFF012900FEFFF8FFFD
:1025B0000124000200F9FF0122000300FAFF0120BC
:1025C000000500FCFF0120000600FEFF01230007BC
:1025D00000FFFF0141000D000000012400FAFF048C
:1025E00000011D00FDFF0500011B00FEFF050001AD
:1025F0001E00FFFF06000123000100070001240068
:102600000200070001200004000500012700060069
:10261000050001260007000300012B00080003004D
:1026200001280008000100012D0009000100013C03
:10263000000C00FFFF0139000B00FDFF0138000A0C
:1026400000FBFF012E000700FAFF0116000200FC4C
:10265000FF0116000200FCFF0115000100FCFF0154
:1026600019000000FBFF011E000000FAFF0122001C
:10267000FDFFFAFF012000FCFFFBFF012300FBFF31
:10268000FBFF0132000A0000000137000000F5FFE7
:10269000017C01B4FF0000015A00EEFF0100011EA1
:1026A00000FAFF0100011900FBFF0100012F00F8F3
:1026B000FF0500012E00FAFF0700012D00FCFF08B6
:1026C00000013200FFFF0A000123000100070001A2
:1026D000190001000500011B0002000500011D009A
:1026E0000300050001190004000300011D0005009E
:1026F0000300011E00060001000123000700000086
:102700000100000000000002010000000000013292
:102710000000000000015A003500F6FF0200000032
:1027200000000001320000000000012800F8FF0056
:1027300000012300F9FFFFFF012000FAFFFEFF0167
:102740001D00FBFFFDFF011500FDFFFDFF01150052
:10275000FDFFFDFF011500FFFFFCFF011500FFFF5E
:10276000FCFF0115000100FCFF0115000100FCFF4A
:102770000115000300FDFF0119000300FCFF011B10
:10278000000500FEFF0120000600FEFF011E0006FE
:1027900000FFFF01280008000000012800080000D9
:1027A00000011E00060001000120000600020001D9
:1027B0001D000500030001150003000300011500C2
:1027C00003000300011500010004000115000100D1
:1027D0000400011500FFFF0400011500FFFF0400C5
:1027E000011500FDFF0300011500FDFF0300011DA1
:1027F00000FBFF0300011B00FBFF0200012300F9A7
:10280000FF0100012300F9FF0000010000000000AB
:102810000002010000000000013200000000000181
:102820009100CBFFBBFF020000000000000132005E
:1028300000000000013E00FDFFF4FF011900FBFF56
:10284000FFFF011900FCFFFDFF012200FDFFFAFF61
:10285000012400FEFFF9FF0129000200F8FF011D1D
:10286000000300FBFF0120000500FCFF0122000621
:1028700000FDFF012300070000000141000D00FFE3
:10288000FF012700FAFF0500011D00FDFF05000103
:102890001B00FEFF0500011E00FFFF0600012300D4
:1028A00001000700012000020006000124000400CE
:1028B00006000124000600040001280007000400AF
:1028C000012B000800030001280008000100012D71
:1028D0000009000100013C000C00FFFF0139000B62
:1028E00000FDFF0138000A00FBFF012E000700FA7F
:1028F000FF0116000200FCFF0116000200FCFF01B0
:1029000015000100FCFF0119000000FBFF011E0083
:102910000000FAFF012200FDFFFAFF012000FCFF8A
:10292000FBFF012300FBFFFBFF0132000A00000058
:102930000137000000F5FF017C01B4FF0000015ADF
:1029400000EEFF0100011E00FAFF0100011900FB6B
:10295000FF0100012F00F8FF0500012A00FAFF0621
:1029600000013100FCFF0900013200FFFF0A0001F5
:102970001E0001000600011E0001000600011B00F0
:102980000200050001190003000400011C000400FE
:102990000400011B000500020001200006000200E7
:1029A00001230007000000010000000000000201F8
:1029B000000000000001320000000000015A003554
:1029C00000F6FF02000000000000013200000000DD
:1029D00000012800F8FF0000012400F9FFFEFF01BC
:1029E0001E00FAFFFFFF011D00FBFFFDFF011500A8
:1029F000FDFFFDFF011500FDFFFDFF011500FFFFBD
:102A0000FCFF011500FFFFFCFF0115000100FCFFAA
:102A10000115000100FCFF0119000300FCFF011576
:102A2000000300FDFF011B000500FEFF0120000662
:102A300000FEFF011E000600FFFF0128000800FF46
:102A4000FF01280008000100011E0006000100012E
:102A5000200006000200011B000500020001190011
:102A6000030004000115000300030001150001002C
:102A7000040001150001000400011500FFFF04001F
:102A8000011500FFFF0400011500FDFF0300011503
:102A900000FDFF0300011D00FBFF0300011900FB07
:102AA000FF0100012400F9FF0200012300F9FF00EB
:102AB0000001000000000000020100000000000111
:102AC000320000000000016F00F7FFBEFF020000AF
:102AD0000000000001320000000000014B000F0068
:102AE000000001C3000000D9FF014B00F1FF00000E
:102AF00001C30000002700020100000000000132B5
:102B00000000000000017B00DBFFC0FF02000000AE
:102B10000000000132000000000001370000000B3F
:102B2000000162027A000000013C000000F4FF0195
:102B3000DC00D4FF00000124000600FCFF011D00A2
:102B40000300FBFF011D000300FBFF011E0000004E
:102B5000FAFF0123000000F9FF012200FDFFFAFF48
:102B6000012400FCFFFAFF012000FBFFFCFF01280D
:102B700000F9FFFCFF012900F8FFFEFF012900F822
:102B8000FFFEFF012D00F7FFFFFF013700F5FF01FA
:102B900000013300F6FF0200012B00F8FF030001E3
:102BA0002800F9FF0400012300FBFF0500012000BD
:102BB000FCFF0500012000FEFF0600011E00FFFFD4
:102BC0000600011E000100060001200002000600B0
:102BD0000120000400050001240006000400013764
:102BE00000F5FF00000201000000000001320000BB
:102BF000000000014B002D0000000200000000005A
:102C00000001320000000000014600F2FFFFFF015A
:102C10002F00F7FFFDFF011D00FBFFFDFF011C0062
:102C2000FCFFFCFF011600FEFFFCFF011900FFFF87
:102C3000FBFF0115000100FCFF0110000100FDFF7A
:102C40000119000300FCFF0119000400FDFF011B36
:102C5000000500FEFF011B000500FEFF0123000729
:102C600000FFFF0128000800FFFF01280008000105
:102C70000001230007000100011E00060001000101
:102C80001D000500030001150003000300011500ED
:102C900003000300011600020004000114000000FC
:102CA000040001140000000400011200FEFF0300F4
:102CB000011900FDFF0400011500FDFF0300011DC7
:102CC00000FBFF0300011E00FAFF0100012400F9D0
:102CD000FF0200012300F9FF0000010000000000D6
:102CE00000020100000000000132000000000001AD
:102CF0006900FFFFC1FF0200000000000001320078
:102D000000000000013C000C00FFFF0133000A003E
:102D1000FEFF012D000800FCFF012B000700FBFF58
:102D20000120000400FBFF011D000300FBFF012048
:102D3000000200FAFF0123000000F9FF0123000058
:102D400000F9FF012600FDFFF9FF011D00FDFFFB5B
:102D5000FF012A00FAFFFAFF012400FAFFFCFF013D
:102D60002B00F8FFFDFF012E00F7FFFEFF013200F0
:102D7000F6FF0000014B00F1FF0100011E00FAFF09
:102D80000100011B00FBFF0200013300F7FF0500FB
:102D9000013100F9FF0700013100FCFF0900012D9E
:102DA00000FFFF09000128000100080001200002C7
:102DB00000060001240004000600012300050005B0
:102DC0000001240006000400012B0008000300019C
:102DD00033000A0002000132000A00010001000075
:102DE00000000000020100000000000132000000AD
:102DF00000000116000000F3FF02000000000000C8
:102E000001320000000000012800F8FF000001244A
:102E100000F9FFFEFF011E00FAFFFFFF011900FC91
:102E2000FFFDFF011900FCFFFDFF011900FDFFFC84
:102E3000FF011500FFFFFCFF011900FFFFFBFF0171
:102E400015000100FCFF0115000100FCFF01190045
:102E50000300FCFF0119000400FDFF011D00050037
:102E6000FDFF011B000500FEFF0128000800FFFF19
:102E700001280008000000012300070000000123D2
:102E8000000700010001200006000200011D0005EE
:102E900000030001150003000300011900030004F2
:102EA00000011500010004000115000100040001EB
:102EB0001900FFFF0500011500FFFF0400011900C4
:102EC000FDFF0400011500FDFF0300011D00FBFFD5
:102ED0000300011E00FAFF0100012400F9FF0200B7
:102EE000012800F8FF0000010000000000000201BE
:102EF00000000000000132000000000001AB00E112
:102F0000FF9EFF02000000000000013200000000F0
:102F100000014200F3FFFEFF012D00FFFF09000149
:102F20001E0000000600011B000200050001150044
:102F30000300030001160004000200012300070043
:102F400001000137000B00010001FF003300000009
:102F5000012D00000009000137000B000000012DC9
:102F6000000000F7FF016E0016000000014F00098D
:102F700000F3FF019B00E1FF0000013C000000F4B2
:102F8000FF013700F5FF0000013C0000000C0001CC
:102F90000401CCFF0000012800F8FF00000115002B
:102FA000FDFFFDFF011500FFFFFCFF011900000000
:102FB000FBFF010000000000000201000000000013
:102FC00001320000000000012200F3FFF0FF0200C8
:102FD0000000000000013200000000000155001157
:102FE0000000000146000000F2FF015500EFFF0065
:102FF0000001460000000E00020100000000000178
:103000003200000000000196002000ACFF0200002A
:103010000000000001320000000000013D00FEFF42
:10302000F4FF012300F9FF0100012000FAFF020074
:10303000012200FAFF0300011C00FCFF0400011C38
:1030400000FCFF0400011D00FDFF0500012000FE43
:10305000FF0600011900000005000128000100081A
:103060000001200002000600012400040006000107
:1030700023000500050001240006000400012B00C8
:1030800008000300012D00090001000137000B00BA
:1030900001000141000D00FFFF013E000C00FDFF9B
:1030A000011B000500FEFF0119000400FDFF0119CE
:1030B000000400FDFF0119000300FCFF012D0004C6
:1030C00000F8FF0132000100F6FF0119000000FBCB
:1030D000FF011E00FFFFFAFF011900FDFFFCFF01C9
:1030E0001900FDFFFCFF011C00FCFFFCFF011D009F
:1030F000FBFFFDFF011B00FBFFFEFF012300F9FFAB
:10310000FFFF013D00FEFF0C000129000800020046
:1031100001240006000400011D0003000500011E3B
:10312000000100060001140000000400011600FE6A
:10313000FF0400011900FDFF0400011500FDFF035D
:1031400000011D00FBFF0300012000FAFF02000147
:103150002300F9FF0100012800F8FF00000128000A
:10316000F8FF0000012300F9FFFFFF012000FAFF34
:10317000FEFF011D00FBFFFDFF011500FDFFFDFF30
:10318000011500FDFFFDFF011500FFFFFCFF01150C
:1031900000FFFFFCFF0124000200F9FF01240004EE
:1031A00000FAFF0112000300FEFF0116000400FEFA
:1031B000FF012E000900FEFF0100000000000002D8
:1031C00001000000000001320000000000012400A6
:1031D0000C00EEFF020000000000000132000000C1
:1031E0000000013C000C00FFFF0133000A00FEFF5D
:1031F000012D000800FCFF012B000700FBFF012050
:10320000000400FBFF011D000300FBFF0120000282
:1032100000FAFF0123000000F9FF0123000000F97C
:10322000FF012600FDFFF9FF012200FDFFFAFF016B
:103230002700FAFFFBFF012400FAFFFCFF012B002F
:10324000F8FFFDFF012E00F7FFFEFF013200F6FF41
:103250000000014B00F1FF0100011E00FAFF010018
:10326000011B00FBFF0200013300F7FF05000131E5
:1032700000F9FF0700013100FCFF0900012D00FFEC
:10328000FF090001230001000700012400020007DC
:1032900000012400040006000123000500050001D0
:1032A000240006000400012B000800030001330085
:1032B0000A0002000132000A0001000100000000C3
:1032C00000000201000000000001320000000000C8
:1032D0000116000000F3FF020000000000000132B0
:1032E0000000000000012800F8FFFFFF012300F9A3
:1032F000FFFFFF012000FAFFFEFF011600FCFFFEAA
:10330000FF011C00FCFFFCFF011500FDFFFDFF019C
:103310001500FFFFFCFF011900FFFFFBFF01150077
:103320000100FCFF0115000100FCFF011900030072
:10333000FCFF0119000400FDFF011D000500FDFF59
:10334000011B000500FEFF0128000800FFFF012807
:10335000000800FFFF012300070001000123000710
:1033600000010001200006000200011D000500030D
:10337000000115000300030001190003000400010F
:1033800015000100040001150001000400011900EE
:10339000FFFF0500011500FFFF0400011500FDFF00
:1033A0000300011900FDFF0400011B00FBFF0200E8
:1033B000012000FAFF0200012300F9FF01000128AB
:1033C00000F8FF0100010000000000000201000001
:1033D00000000001320000000000018B00D4FFB9A2
:1033E000FF020000000000000132000000000001A8
:1033F000B801580000000137000000F5FF013C0053
:10340000F4FF00000124000600FCFF01240004007A
:10341000FAFF0122000300FAFF0123000100F9FF77
:10342000012300FFFFF9FF012200FDFFFAFF012346
:1034300000FBFFFBFF012000FAFFFEFF012B00074E
:1034400000FBFF0127000500FAFF0120000200FA3F
:10345000FF011E000100FAFF0119000000FBFF013F
:103460001900FFFFFBFF011900FDFFFCFF01150024
:10347000FDFFFDFF011900FCFFFDFF011B00FBFF2D
:10348000FEFF011E00FAFFFFFF012300F9FF00000D
:10349000013101C3FF0000013C0000000C000118D5
:1034A000013800000001230007000100011E000692
:1034B00000010001100003000100011500030003DA
:1034C00000011600020004000114000000040001C5
:1034D0000F0000000300011500FFFF0400011200AF
:1034E000FEFF0300011200FDFF0200011500FDFFB9
:1034F0000300011900FBFF0100013D00F4FF020081
:1035000001FF00CDFF0000013C0000000C00011D88
:103510000139000000012D00090001000120000612
:1035200000020001120003000200010B0001000272
:1035300000011E0001000600011900000005000145
:103540001D00FDFF0500011C00FCFF040001200020
:10355000FAFF0200012900F8FF0200013200F6FF25
:10356000000001E600D2FF000001410000000D0054
:10357000020100000000000132000000000001ED27
:1035800005CB0089FC0200000000000001320000B1
:1035900000000001A400F5FFE1FF01A100F7FFE139
:1035A000FF012201F1FFC8FF010501F5FFCDFF0179
:1035B000DA00F9FFD5FF01B100FBFFDDFF01870055
:1035C000FEFFE5FF016E00FEFFEAFF0201000000C2
:1035D00000000132000000000001F8013E00280157
:1035E0000200000000000001320000000000018025
:1035F0000280FF0000020100000000000132000014
:10360000000000010C02EC0030FF0200000000008E
:10361000000132000000000001AB00F7FF210001B3
:103620009500F6FF1C00019600F5FF1C00019D00AF
:10363000F4FF1D0001C000F0FF230001CE00ECFFED
:103640002400016300F6FF1100016100F5FF100086
:10365000016400F4FF1000016000F4FF0F00012A74
:1036600000FAFF0600012700FAFF0500012400FA16
:10367000FF0400012000FAFF0200012000FAFF020F
:1036800000011E00FAFF0000013C00F4FF000001F1
:103690003D00F4FFFEFF014200F3FFFEFF01420088
:1036A000F3FFFEFF014600F2FF0000013700F5FFC7
:1036B0000000012D00F7FFFFFF012B00F8FFFDFFC9
:1036C000012000FBFFFCFF010E00FEFFFEFF010FCB
:1036D000000000FDFF011000FFFFFDFF01150001CC
:1036E00000FCFF012D000400F8FF0140000800F677
:1036F000FF0120000400FBFF0124000200F9FF018C
:103700002E000200F7FF012D000000F7FF012D0041
:10371000FFFFF7FF012E00FEFFF7FF012800FCFF6F
:10372000F9FF012700FBFFFAFF0201000000000083
:1037300001320000000000019E02FF00C9FE0200ED
:10374000000000000001320000000000011E000621
:103750000000000115000400010001120003000236
:103760000001160002000400011B00020005000118
:10377000190001000500014600FFFF0E00014C008A
:10378000FEFF0F00014C00FDFF0F00018E00FBFF4C
:103790001C00018F00FAFF1C000201000000000065
:1037A00001320000000000012902E9FEB40002001D
:1037B000000000000001320000000000015D00EE8A
:1037C000FFFBFF014700F2FFFEFF013700F5FF009E
:1037D00000012F00F7FF0300012700FAFF05000199
:1037E0002700FBFF0600012600FDFF0700012E0059
:1037F000FEFF0900015600FDFF1100012D00FFFF33
:103800000900012900FEFF0800012600FDFF070056
:10381000012000FCFF0500012400FAFF040001283C
:1038200000F8FF0100018A01EFFFB3FF011E000055
:1038300000FAFF0119000100FBFF0136000400F649
:10384000FF013A000600F6FF0136000600F7FF010F
:1038500060000C00F1FF0128000400F9FF012000C6
:103860000200FAFF010B00FFFFFEFF011000FFFF47
:10387000FDFF012E00F9FFFAFF018A00EBFFEEFFCA
:10388000014B00F4FFF7FF014A00F6FFF5FF01438B
:1038900000F7FFF6FF011D00FDFFFBFF011B00FE0F
:1038A000FFFBFF014B01F3FFBFFF010401F6FFCD5A
:1038B000FF011900050000000119000500010001C9
:1038C0001600040002000116000400020001350089
:1038D00007000800013A0006000A000194000C00ED
:1038E0001B00015E000800110001600009001100CA
:1038F000011D0003000500011C0004000400014438
:10390000000B000800014A000D000700014A000EEC
:103910000005000147000E0002000123000700001F
:10392000000123000700FFFF0120000600FEFF0149
:103930001D000500FDFF0120000500FCFF01240023
:103940000400FAFF0131000400F7FF013E0003000C
:10395000F4FF0141000100F3FF0146000000F2FF07
:103960000201000000000001320000000000010A16
:10397000000600000002000000000000013200000C
:103980000000000166001400040001510010000254
:1039900000013C000C0000000133000A00FEFF01A2
:1039A0002D000800FCFF0132000800FAFF0135007D
:1039B0000800F9FF0143000900F6FF014E000A006C
:1039C000F4FF014E000A00F4FF019E001200E6FF22
:1039D0000138012100CBFF0155000800F1FF015C17
:1039E000000900F0FF01BE000F00DDFF01BF000D68
:1039F00000DCFF01B1000A00DEFF01F7000C00D07F
:103A0000FF01F5000A00D0FF015A000100EEFF019E
:103A10001E00FFFFFAFF011500FFFFFCFF0112006F
:103A2000FEFFFDFF011200FDFFFEFF011000FDFF84
:103A3000FFFF011000FDFF0100012E00F7FF020053
:103A4000012F00F7FF0300013900F5FF03000132E9
:103A500000F6FF0100013200F6FF0000012E00F722
:103A6000FF0200013100F7FF0400013600F7FF06F6
:103A700000013900F7FF0700013C00F8FF090001D1
:103A80004300F7FF0A00014400F8FF0B0001890022
:103A9000F1FF1700019200F1FF1900018B00F2FF06
:103AA0001800018000F3FF16000201000000000072
:103AB00001320000000000019B01C4FFEF00020082
:103AC000000000000001320000000000015F00ED76
:103AD000FF0000015100F0FFFEFF013D00F4FFFE7A
:103AE000FF013100F7FFFCFF011500FDFFFDFF01A5
:103AF0001500FDFFFDFF011600FEFFFCFF01150094
:103B0000FFFFFCFF013C00FFFFF4FF014C0002003F
:103B1000F1FF0156000300EFFF0161000400EDFF1B
:103B20000162000500EDFF0165000700EDFF016582
:103B3000000900EEFF0132000600F8FF0132000626
:103B400000F8FF0135000700F8FF0131000700F918
:103B5000FF0132000800FAFF0133000900FBFF02F9
:103B600001000000000001320000000000011D0003
:103B7000F1FF090002000000000000013200000017
:103B8000000001FF00F6FFCEFF015601F2FFBDFF6E
:103B90000201000000000001320000000000018668
:103BA000023D01DF000200000000000001320000C1
:103BB000000000019300F7FFE4FF018200F9FFE736
:103BC000FF010701F3FFCDFF019F00F9FFE1FF01B6
:103BD000C500FAFFD9FF01D400FAFFD6FF01DD00CE
:103BE000FCFFD4FF020100000000000132000000D1
:103BF0000000018F01F7FFEF00020000000000004D
:103C000001320000000000017F000B00E9FF0146C7
:103C100000F2FFFFFF017D00F6FF17000141000DDC
:103C2000000100010000000000000201000000008F
:103C30000001320000000000011700F2FF00000246
:103C400000000000000001320000000000016A00D6
:103C5000FDFFEBFF0172000900EBFF015D000500B5
:103C6000120002010000000000013200000000000C
:103C7000012700F4FF1400020000000000000132E0
:103C80000000000000014F01BDFFFFFF0201000026
:103C900000000001320000000000016E004000EF53
:103CA000FF020000000000000132000000000001DF
:103CB0000901CBFF000002010000000000013200FA
:103CC00000000000016F003F00EBFF020000000059
:103CD00000000132000000000001FA00CEFF0000E9
:103CE0000201000000000001320000000000017924
:103CF000003A002C00020000000000000132000029
:103D000000000001F2021D0094000201000000000A
:103D10000001320000000000010401D5FF6AFF022B
:103D20000000000000000132000000000001F70266
:103D30001D0095000201000000000001320000009B
:103D40000000011D01FCFF55FF0200000000000003
:103D50000132000000000001BF021B008A000201C6
:103D6000000000000001320000000000012B0002F2
:103D7000001A0002000000000000013200000000F4
:103D800000012800FFFF0800012400FEFF070001DA
:103D90000700FFFF0100010700FFFF0100010E0007
:103DA000FEFFFEFF012800FCFFF9FF0201000000FA
:103DB000000001320000000000011800F2FFFEFFC9
:103DC0000200000000000001320000000000012499
:103DD000000200070001150003000300010B0002B0
:103DE0000001000141000D00000002010000000080
:103DF000000132000000000001EF007AFF330002F2
:103E00000000000000000132000000000001260058
:103E10000700FDFF0126000700FDFF01320008003A
:103E2000FAFF012E000700FAFF0135000700F8FF36
:103E30000136000600F7FF0136000600F7FF013AE1
:103E4000000600F6FF0138000500F6FF013B000404
:103E500000F5FF0139000300F5FF0133000200F611
:103E6000FF0137000100F5FF012D000000F7FF0101
:103E70003200FFFFF6FF012D00FCFFF8FF012600D6
:103E8000FDFFF9FF012300FBFFFBFF011D00FBFF0E
:103E9000FDFF012200FAFFFDFF011E00FAFFFFFFF8
:103EA000011E00FAFFFFFF011E00FAFF01000123BF
:103EB00000F9FF0100013F00F4FF0400014300F49A
:103EC000FF0600013900F7FF0700013500F8FF0782
:103ED00000020100000000000132000000000001AB
:103EE000F30085003C0002000000000000013200E9
:103EF0000000000001D600D7FFF4FF02010000001F
:103F00000000013200000000000140002500F5FF24
:103F1000020000000000000132000000000001C1AA
:103F200000DBFF0B00020100000000000132000076
:103F3000000000016B003F000C00020000000000C8
:103F400000013200000000000140014000000001BB
:103F500036013E0000000176027E00FDFF014C00AC
:103F60000F00FEFF012D000900FFFF0110000300FC
:103F7000FFFF010B000100FEFF0110000100FDFF2B
:103F80000119000000FBFF012800FFFFF8FF010BF3
:103F900000FFFFFEFF010B00FEFFFFFF012D00F7FA
:103FA000FFFFFF015000F0FFFFFF017B0281FF01D7
:103FB00000013B01C1FF0100014001C0FF030001FE
:103FC0000B00FEFF0100010E00FEFF0200011500C4
:103FD000FFFF0400011900000005000119000100A5
:103FE0000500011500010004000112000200030099
:103FF00001100003000100010000000000000201A8
:104000000000000000013200000000000147001520
:1040100000DBFF0200000000000001320000000091
:104020000001BA00EFFFDFFF015900F8FFF0FF01C8
:104030005E00F8FFEFFF0201000000000001320007
:1040400000000000016D00EBFFC2FF020000000055
:10405000000001320000000000016200FBFFEDFFE4
:10406000016000FEFFEDFF016000FEFFEDFF015F5C
:1040700000FFFFEDFF01C3000100D9FF01B90001FE
:1040800000DBFF0201000000000001320000000020
:1040900000015B014300C5000200000000000001B8
:1040A00032000000000001C800D8FFFFFF0201003D
:1040B0000000000001320000000000015002EBFE91
:1040C00022FF02000000000000013200000000009A
:1040D0000128000800010001260007000300012755
:1040E0000006000500012300050005000155000839
:1040F000000F000162000800120001B6000D00224E
:104100000002010000000000013200000000000178
:10411000F20156001E010200000000000001320002
:1041200000000000010C01E8FF3000020100000067
:104130000000013200000000000154002100DAFFFD
:10414000020000000000000132000000000001FF3A
:1041500000EAFF2E00020100000000000132000012
:10416000000000019B00B4FFCAFF02000000000035
:104170000001320000000000011101E6FF300002E2
:104180000100000000000132000000000001EC000E
:104190008A001F0002000000000000013200000041
:1041A0000000011C01E9FF340002010000000000D2
:1041B00001320000000000017C00E6FFBAFF0200AF
:1041C00000000000000132000000000001C201A652
:1041D000FF010002010000000000013200000000A9
:1041E00000019C005C00F0FF0200000000000001E4
:1041F00032000000000001C701A5FF02000201001B
:10420000000000000132000000000001E60068002C
:104210005B0002000000000000013200000000000E
:1042200001BD01A7FF0100020100000000000132F2
:1042300000000000000194005900FFFF0200000090
:1042400000000001320000000000018C01F2FFB20A
:10425000FF02010000000000013200000000000128
:104260007C0019004600020000000000000132003E
:1042700000000000018701F2FFB3FF02010000000F
:1042800000000132000000000001CB00AAFF560030
:104290000200000000000001320000000000018E5A
:1042A00001F0FFB2FF020100000000000132000037
:1042B00000000001DD007400C0FF020000000000EB
:1042C000000132000000000001BD01A7FF01000253
:1042D00001000000000001320000000000019B000E
:1042E0004B00370002000000000000013200000017
:1042F0000000014100F5FF0700020100000000007E
:10430000013200000000000117000000F2FF02006F
:10431000000000000001320000000000014600FF24
:10432000FF0E00020100000000000132000000004A
:10433000000119000100F1FF02000000000000016F
:104340003200000000000144000B000800020100E0
:10435000000000000132000000000001B60093FFE1
:104360000100020000000000000132000000000017
:1043700001350007000800020100000000000132C2
:104380000000000000011B000200F0FF020000001E
:1043900000000001320000000000013900F7FF07B3
:1043A00000020100000000000132000000000001D6
:1043B000F2007B004D00020000000000000132000E
:1043C00000000000014400F5FF08000201000000A9
:1043D00000000132000000000001A000A0FFF9FF72
:1043E0000200000000000001320000000000018A0D
:1043F00001EFFFB3FF0201000000000001320000E6
:10440000000000015C001A00CFFF02000000000065
:104410000001320000000000011301E7FF3100023B
:1044200001000000000001320000000000016D00EA
:104430002200C8FF0200000000000001320000005E
:104440000000013900F7FF07000201000000000032
:104450000132000000000001A4006200F9FF020028
:10446000000000000001320000000000014E0007C3
:10447000000E0002010000000000013200000000F8
:104480000001D40086FF24000200000000000001AB
:1044900032000000000001410000000D0002010098
:1044A0000000000001320000000000017700080059
:1044B0004700020000000000000132000000000080
:1044C0000131000700070002010000000000013276
:1044D00000000000000143026200B3FE0200000081
:1044E00000000001320000000000015101F2FFBE97
:1044F000FF02010000000000013200000000000186
:104500006B0019003B0002000000000000013200B7
:1045100000000000014B01F3FFBFFF02010000009B
:1045200000000132000000000001450023001600D9
:104530000200000000000001320000000000014BFA
:1045400001F3FFBFFF020100000000000132000084
:1045500000000001FD009EFF74000200000000004A
:104560000001320000000000015501F3FFBDFF0211
:1045700001000000000001320000000000011800EE
:104580000300F2FF02000000000000013200000002
:10459000000001FB001A00D5FF020100000000002E
:1045A00001320000000000017B00300038000200F2
:1045B000000000000001320000000000018101B392
:1045C000FF010002010000000000013200000000B5
:1045D000000186004F00F2FF020000000000000111
:1045E000320000000000017C01B4FF000002010065
:1045F0000000000001320000000000017F004C00BC
:104600000000020000000000000132000000000075
:1046100001F4001700D5FF02010000000000013284
:104620000000000000015600F3FF3200020000000D
:104630000000000132000000000001ED001600D66D
:10464000FF02010000000000013200000000000134
:10465000C400ECFF74000200000000000001320002
:1046600000000000018101B3FF0000020100000012
:1046700000000132000000000001FD00580084FF2E
:104680000200000000000001320000000000016D87
:1046900001B7FF000002010000000000013200002D
:1046A00000000001E4004900740002000000000066
:1046B000000132000000000001ED001600D6FF02EC
:1046C00001000000000001320000000000015B005A
:1046D000D3FFE1FF020000000000000132000000F3
:1046E0000000013D000A0007000201000000000078
:1046F00001320000000000011600F4FF0600020075
:104700000000000000013200000000000143000C26
:1047100000FAFF020100000000000132000000006A
:1047200000011700F4FF0700020000000000000174
:104730003200000000000147000200F2FF02010009
:104740000000000001320000000000018500B1FF00
:104750000D00020000000000000132000000000017
:10476000013E000300F4FF020100000000000132DE
:104770000000000000017F0004004C000200000067
:1047800000000001320000000000015001F3FFBEF4
:10479000FF020100000000000132000000000001E3
:1047A00002000000FFFF02000000000000013200D4
:1047B000000000000143000900F6FF0201000000B4
:1047C000000001320000000000011600F7FF0A009F
:1047D000020000000000000132000000000001247F
:1047E0000006000400020100000000000132000089
:1047F000000000010D00FAFFFBFF020000000000B6
:1048000000013200000000000102011B00D4FF0281
:104810000100000000000132000000000001020061
:104820000000FFFF02000000000000013200000055
:1048300000000135000800F9FF020100000000003F
:104840000132000000000001CB00EBFF7800020005
:1048500000000000000132000000000001200005FF
:10486000000400020100000000000132000000000E
:10487000000182004E000000020000000000000164
:104880003200000000000141000B00F9FF020100AE
:10489000000000000132000000000001C300010020
:1048A0008BFF020000000000000132000000000049
:1048B0000139000800080002010000000000013278
:1048C000000000000001AF0E3200CF08020100001E
:1048D00000000001320000000000020100000000A2
:0848E0000000000000000000D0
:0848E800E9CFE4FFEACFE4FF91
:1048F000E652D9CFE6FFDACFE6FFE1CFD9FFE2CF2C
:10490000DAFFE6529EA0E9D29E90FE0ECF6E3D0EDB
:10491000CE6E19C530F50501316B0501010E326F00
:1049200005011A511B111C111D1117E0D880000E32
:1049300005011A55000E1B55190E1C55000E1D556C
:1049400006E205011A6B1B6B1C6B1D6B06D0050183
:104950001A07000E1B5B1C5B1D5B05011A511B1126
:104960001C111D1102E00501326B0501000501E07B
:104970003DD10501115112111311141107E1050167
:10498000155116111711181101E12FD10501D75139
:104990000DE1050119A302D08C8E01D08C9E05017A
:1049A00019A702D08C8A01D08C9A0FD00501D705A7
:1049B0000CE1050119A302D08B8401D08B94050171
:1049C00019A702D0898401D08994050111511211CF
:1049D0001311141164E0010EE96E050EEA6E0E016A
:1049E000B751EE240E01B76F0E01B851EE200E0143
:1049F000B86F0E01B951EE200E01B96F0E01BA5118
:104A0000EE200E01BA6FB7CE4CF0B8CE4DF0B9CE55
:104A10004EF0BACE4FF04C6A4D6A4E6A800E4F1679
:104A20004C504D104E104F1028E0B7CEB7FEB8CE08
:104A3000B8FEB9CEB9FEBACEBAFE0E01BA9F010ECB
:104A4000050130110501306F0501010E316F0501BF
:104A50001107000E125B135B145B050119A307D04D
:104A600005012807000E295B2A5B2B5B06D0050198
:104A7000282B000E29232A232B2305010951050188
:104A8000012705010A510501022305010B5105010A
:104A9000032305010C51050104230501326B0501B7
:104AA000155116111711181164E0050EE96E050E67
:104AB000EA6E0E01BB51EE240E01BB6F0E01BC511C
:104AC000EE200E01BC6F0E01BD51EE200E01BD6F38
:104AD0000E01BE51EE200E01BE6FBBCE4CF0BCCE1F
:104AE0004DF0BDCE4EF0BECE4FF04C6A4D6A4E6AD0
:104AF000800E4F164C504D104E104F1028E0BBCE7C
:104B0000BBFEBCCEBCFEBDCEBDFEBECEBEFE0E010B
:104B1000BE9F040E050130110501306F0501010E25
:104B2000316F05011507000E165B175B185B050159
:104B300019A707D005012C07000E2D5B2E5B2F5BFC
:104B400006D005012C2B000E2D232E232F2305012B
:104B50000D510501052705010E510501062305012B
:104B60000F51050107230501105105010823050117
:104B7000326B0501315139E00501D75107E10501DB
:104B800030B18C8C050130B58C8809D00501D70572
:104B900006E1050130B18B8C050130B5898A000032
:104BA0000000000000000000000000000000000005
:104BB00000000000000000000000000000000000F5
:104BC00000000000000000000000000000000000E5
:104BD000000000000501D75103E18C9C8C9805D0A2
:104BE0000501D70502E18B9C899AD7D0030E0501F8
:104BF000005D01E0A0D00501E45101E179D005019B
:104C00002105DF6E05011E511F1137E1DF50EA6AF1
:104C1000310FE96E0E0EEA22EF500E01EA6AAC2562
:104C2000E96EAD51EA22EF6AEA6ADF34FE0BEA363A
:104C3000E96E790EE9260E0EEA22EE6AED6AEA6A5C
:104C4000DF34FE0BEA36E96E490EE9260E0EEA2243
:104C5000EE6AED6ADF50EA6A310FE96E0E0EEA2263
:104C6000EF6AEA6ADF34FE0BEA36E96E010EE926E6
:104C70000E0EEA22EE6AED6A3BD0EA6ADF34FE0BE2
:104C8000EA36E96E790EE9260E0EEA2222C5EEFF1B
:104C900023C5EDFFEA6ADF34FE0BEA36E96E490E02
:104CA000E9260E0EEA221EC5EEFF1FC5EDFFDF50FE
:104CB000EA6A310FE96E0E0EEA2220C5EFFFEA6ABA
:104CC000DF34FE0BEA36E96E010EE9260E0EEA220B
:104CD000EE50ED100DE1EA6ADF34FE0BEA36E96EC4
:104CE000010EE9260E0EEA221EC5EEFF1FC5EDFFDE
:104CF0000E01B6510501205D1DE10E01B051050107
:104D00001E1904E10E01B15105011F190AE1050147
:104D1000010ED86F0501D46B0501E35101E08A98BB
:104D200009D00501D86B0501010ED46F0501E351CF
:104D300001E08A8832D0040E0501005D2EE10501F4
:104D4000245124E025C54CF026C54DF0D8904D32B5
:104D50004C32D8904D324C324C50BB6EE1C54EF0C7
:104D6000E2C54FF0040ED8904E364F36E804FBE112
:104D7000300E4E16000E4F16CF0EBA1400014E1014
:104D80004C6E4FC04DF04C50BA6E04D0BB6ACF0E83
:104D9000BA14BA6E0501010E326F0501325101E1FC
:104DA00090D005011A511B111C111D1101E089D071
:104DB0000501006B0501275101E07ED034C500F5E7
:104DC00035C501F536C502F537C503F538C504F517
:104DD00039C505F53AC506F53BC507F53CC508F5E7
:104DE0003DC509F53EC50AF53FC50BF540C50CF5B7
:104DF00041C50DF542C50EF543C50FF544C510F587
:104E000045C511F546C512F547C513F548C514F556
:104E100049C515F54AC516F54BC517F54CC518F526
:104E20004DC519F54EC51AF54FC51BF550C51CF5F6
:104E300051C51DF552C51EF553C51FF554C520F5C6
:104E400055C521F556C522F557C523F558C524F596
:104E500059C525F55AC526F50501346B0501356B95
:104E6000366B376B386B0501396B3A6B3B6B3C6BC0
:104E70000501456B466B476B486B0501496B4A6BF7
:104E80004B6B4C6B05014D6B05014E6B4F6B506BC3
:104E9000516B0501526B536B0501546B0501556B4A
:104EA0000501566B576B0501586B0501596B5A6B21
:104EB0000501010E276F05D005011A6B1B6B1C6BDA
:104EC0001D6B8050800B06E00501DF5106E081502C
:104ED000010B03E10501010EDE6FE552E552E5CF5E
:104EE000DAFFE7CFD9FFE552E5CFEAFFE5CFE9FFEB
:104EF0001100D9CFE6FFDACFE6FFE1CFD9FFE2CF4D
:104F0000DAFFE652DF6ADFCF00F0020EE76E00182C
:104F1000E8AE02D0E73402D0E750005C3CE2DFCFDD
:104F2000E9FFEA6AE9BEEA68D890E936EA36D8903D
:104F3000E936EA36010EE926050EEA22010EEE6E8A
:104F4000EE6AEE6AEE6ADFCFE9FFEA6AE9BEEA6876
:104F5000D890E936EA36D890E936EA36110EE926D5
:104F6000050EEA22EE6AEE6AEE6AEE6ADFCFE9FF2C
:104F7000EA6AE9BEEA68D890E936EA36D890E936B6
:104F8000EA36090EE926050EEA22EE6AEE6AEE6AB4
:104F9000EE6ADF2AB8D70501006B0501196B050120
:104FA0001A6B1B6B1C6B1D6B05011E6B1F6B0501C8
:104FB000206B0501216B0501226B236B0501010E9E
:104FC000276FCD82CD9ECD9CCD9ACD98CD96CD9498
:104FD000FE0ECF6E3D0ECE6ECD809F809E909D804A
:104FE00092809F9C010EE66EE66A2BEC41F0E55242
:104FF000E552010EE66E0B0EE66E2BEC41F0E5522B
:10500000E5528D8496948D829692898C929C8D80A7
:1050100096908B8294928C9C959C8C9E959E8C985D
:1050200095988C9A959A949E828E000000000000BC
:105030000000000000000000000000000000000070
:105040000000000000000000000000000000000060
:10505000948E829E0501010EE36F0501010EE46F3F
:105060008A9893980501010ED46F0501D76B05014D
:10507000010ED86F0501DD6B0501D96BDA6BDB6BB7
:10508000DC6B0501DE6B9380F19E0501010EDF6F85
:1050900093968196C5EC34F0E552E552E5CFDAFF00
:1050A000E7CFD9FF120017EC35F0BAEC36F0F3EC8D
:1050B00035F015EC39F0E66AD950FEEC38F007010E
:1050C000B45101E0B3D0DF0424E1C3EC36F00CE1CD
:1050D0000501010EE36FE46B6EEC36F002E2E16A6B
:1050E000E552E16E00500DD01CEC37F006E1ED50BA
:1050F00004E10501E36B010E03D00501010EE36F2E
:10510000E46F000EE66EE66AD8C5E6FF4CEC37F0B9
:105110008BD0020EDF5C2EE1C3EC36F009E1050115
:10512000D76B96909492959C959E9598959A1BD046
:105130001CEC37F00DE1ED500BE10501010E5AECCE
:1051400037F094949294949C929A959292926CD007
:10515000ECEC38F0020EEE1867E1ED5065E1050168
:10516000020E5AEC37F094849284948C928A958241
:1051700092825AD0040EDF5C07E1010EDBCFB0FE55
:10518000020EDBCFB1FE50D0050EDF5C07E1010E51
:10519000DBCFAEFE020EDBCFAFFE46D0080EDF5CEB
:1051A0000FE1ECEC38F0180ED880EE54000EED5400
:1051B00003E2180E66EC37F0010EDBCFAAFE34D006
:1051C000090EDF5C0FE1ECEC38F0060ED880EE54EF
:1051D000000EED5403E2060E66EC37F0010EDBCF55
:1051E000ABFE22D00A0EDF5C03E16DEC37F009D094
:1051F0000B0EDF5C03E16DEC37F016D00C0EDF5CBC
:1052000007E1010EDBCFB4FE020EDBCFB5FE0CD002
:105210000D0EDF5C09E1C3EC36F004E00501010E80
:10522000DF6F02D00501DF6B97EC40F0FAEC38F04D
:105230002BEF35F017EC35F0200EE12402E3E168A6
:10524000E6520AEC38F020EC37F0E66AD950040F49
:105250000DEC39F0060F0DEC39F0080FF0EC38F0DA
:105260000C0F96EC37F0D950040F08EC37F004E23D
:10527000EA0E006EBA0E83D2D950060F08EC37F052
:1052800004E2BC0E006EBA0E7AD2FAEC36F0040ECE
:10529000005C000E015804E2920E006EBA0E6FD24E
:1052A000060EDBCF00F0070EDBCF01F0040E005C32
:1052B000000E015804E26A0E006EBA0E60D20701B9
:1052C000B45101E065D2080EDBCF10F0090EDBCF40
:1052D00011F00A0EDBCF12F00B0EDBCF13F010C073
:1052E00038F011C039F012C03AF013C03BF0080E8C
:1052F000DBCF3DF0090EDBCF3EF00A0EDBCF3FF0F7
:105300000B0EDBCF40F080EC69F034C00CF035C000
:105310000DF036C00EF037C00FF00C0EDBCF14F0DE
:105320000D0EDBCF15F00E0EDBCF16F00F0EDBCF20
:1053300017F014C038F015C039F016C03AF017C095
:105340003BF00C0EDBCF3DF00D0EDBCF3EF00E0E32
:10535000DBCF3FF00F0EDBCF40F080EC69F00C505C
:105360003424086E0D503520096E0E5036200A6E1A
:105370000F5037200B6E01EC37F03B6E03EC59F009
:10538000D7EC35F039C0E6FF3AC0E6FF3BC0E6FF98
:105390003CC0E6FF84EC5EF0FAEC38F0E5528BECB2
:1053A00038F038C039F0BBEC38F073EC5AF0140E1A
:1053B00038C0DBFF150E39C0DBFF160E3AC0DBFF2D
:1053C000170E3BC0DBFF05012751FDE04E6B4F6B15
:1053D000506B516B4D6B8D908B92D950080FAFEC89
:1053E00038F002E698EC35F006E2020E4D6FB7ECAD
:1053F00037F0F6EC35F0D9500C0FAFEC38F002E690
:1054000098EC35F012E2080E05014D114D6F0C0EAF
:10541000DBCF38F00D0EDBCF39F00E0EDBCF3AF0DC
:105420000F0E31EC35F003EC36F0C3EC37F002E64A
:1054300077EC35F004E23C0E006EBA0EA0D1CFEC52
:1054400037F002E677EC35F004E20E0E006EBA0E8D
:1054500096D1C7EC36F0D7EC35F0AC0E3E6EC50EEB
:105460003F6EA70E406E470E416E6FEC59F00FEC89
:1054700037F0DBCF0CF0150EDBCF0DF0160EDBCFC7
:105480000EF0170EDBCF0FF00CC038F00DC039F066
:105490000EC03AF00FC03BF001EC59F029EC37F0A8
:1054A00060EC35F01CEC59F0180E39C0DBFF190E1A
:1054B0003AC0DBFF1A0E3BC0DBFF1B0E3CC0DBFF1C
:1054C000E0EC36F0080EDBCF08F0090EDBCF09F078
:1054D0000A0EDBCF0AF00B0EF3EC37F038C035F5CF
:1054E00039C036F53AC037F53BC038F5080EDBCF8A
:1054F00045F5090EDBCF46F50A0EDBCF47F50B0E5F
:10550000DBCF48F532EC37F029EC37F032EC37F0EE
:1055100039C00CF03AC00DF03BC00EF03CC00FF0AB
:10552000A5EC37F008C039F009C03AF00AC03BF0EA
:105530000BC03CF06FEC59F0D7EC35F0C7EC36F00F
:1055400039C014F03AC015F03BC016F03CC017F05B
:10555000C7EC36F039C018F03AC019F03BC01AF069
:105560003CC01BF0A5EC37F014C039F015C03AF080
:1055700016C03BF017C03CF06FEC59F039C010F08A
:105580003AC011F03BC012F03CC013F0A5EC37F06C
:1055900004C039F005C03AF006C03BF007C03CF04B
:1055A000DCEC59F00FEC37F0DBCF28F0150EDBCF39
:1055B00029F0160EDBCF2AF0170EDBCF2BF028C018
:1055C00038F029C039F02AC03AF02BC03BF001EC8A
:1055D00059F039C024F03AC025F03BC026F03CC059
:1055E00027F0140EDBCF30F0150EDBCF31F0160EA6
:1055F000DBCF32F0170EDBCF33F030C038F031C0E4
:1056000039F032C03AF033C03BF001EC59F039C008
:105610002CF03AC02DF03BC02EF03CC02FF0A5EC92
:1056200037F024C039F025C03AF026C03BF027C03F
:105630003CF06FEC59F039C020F03AC021F03BC08B
:1056400022F03CC023F03E6A3F6A406A400E416E41
:105650006FEC59F039C01CF03AC01DF03BC01EF091
:105660003CC01FF060EC35F01CEC59F01C0E39C04A
:10567000DBFF1D0E3AC0DBFF1E0E3BC0DBFF1F0E23
:105680003CC0DBFF080EDBCF04F0090EDBCF05F0DA
:105690000A0EDBCF06F00B0E39EC35F038C03DF5C5
:1056A00039C03EF53AC03FF53BC040F5E0EC36F07E
:1056B0000C0EDBCF08F00D0EDBCF09F00E0EDBCFAA
:1056C0000AF00F0EF3EC37F038C039F539C03AF56F
:1056D0003AC03BF53BC03CF50C0EDBCF49F50D0E57
:1056E000DBCF4AF50E0EDBCF4BF50F0EDBCF4CF5C3
:1056F0009AEC37F039EC35F038C041F539C042F555
:105700003AC043F53BC044F5FAEC36F0060EDB50E8
:10571000001803E1070EDB50011814E005013D51AC
:105720003E113F1140110EE1D880000E4555000E8C
:105730004655000E4755000E485504E2E30E006E34
:10574000B90E1DD0FAEC36F0060EDB50001803E15E
:10575000070EDB50011816E00501415142114311BB
:10576000441110E1D880000E4955000E4A55000E34
:105770004B55000E4C5506E2B80E006EB90E0FECFC
:1057800038F006D00501010E346F276B97EC40F01E
:10579000200EE15C02E2E16AE552E16E2BEF35F0AA
:1057A00017EC35F03F0EE12402E3E168E652E16ECA
:1057B000E5EC37F0E1EC38F0100FF0EC38F0040FC6
:1057C000F0EC38F0080F0DEC39F0140FF0EC38F075
:1057D0000C0F96EC37F00701B45101E06FD128ECC3
:1057E00035F00DE1040EDBCF04F0050EDBCF05F044
:1057F000060EDBCF06F0070EA8EC35F011E0100E18
:10580000DBCF08F0110EDBCF09F0120EDBCF0AF070
:10581000130EDBCF0BF0085009100A100B1035E106
:10582000080EDBCF0CF0090EDBCF0DF00A0EDBCF3C
:105830000EF00B0EDBCF0FF00C500D100E100F10F2
:1058400012E10C0EDBCF10F00D0EDBCF11F00E0EBF
:10585000DBCF12F00F0EDBCF13F01050111012102F
:10586000131001E12BD1140EDBCF14F0150EDBCF9A
:1058700015F0160EDBCF16F0170EDBCF17F0145015
:1058800015101610171001E119D1320EDB6A330E14
:10589000DB6A340EDB6A350EDB6A310EDB6A8D9013
:1058A0008B92D950100FAFEC38F002E698EC35F03F
:1058B0001FE2310EDB500209E76E310EE7CFDBFF4E
:1058C000100EDBCF38F0110EDBCF39F0120EDBCF2C
:1058D0003AF0130E31EC35F0100E34C0DBFF110E30
:1058E00035C0DBFF120E36C0DBFF130E37C0DBFF07
:1058F000D950140FAFEC38F002E698EC35F015E211
:10590000310EDB500809E76E310EE7CFDBFF140ED6
:10591000DBCF38F0150EDBCF39F0160EDBCF3AF0C7
:10592000170E31EC35F010EC36F0DCEC38F0190ED7
:10593000EECFDBFF1A0EEECFDBFF1B0EEECFDBFF51
:105940001C0EB7EC38F0100F91EC37F0290EEECFAB
:10595000DBFF2A0EEECFDBFF2B0EEECFDBFF2C0E94
:10596000B7EC38F0040FE96E000E7DEC36F0D9503C
:10597000080F91EC37F01D0EEECFDBFF1E0EEECFC1
:10598000DBFF1F0EEECFDBFF200EB7EC38F0140F5D
:1059900091EC37F02D0EEECFDBFF2E0EEECFDBFFBE
:1059A0002F0EEECFDBFF300EB7EC38F00C0FE96EA8
:1059B000000E8CEC36F0010EF36E180EF3CFDBFF09
:1059C00005012751FDE0180EDBCF34F5190EDBCFB2
:1059D00035F51A0EDBCF36F51B0EDBCF37F51C0E77
:1059E000DBCF38F51D0EDBCF39F51E0EDBCF3AF5D8
:1059F0001F0EDBCF3BF5200EDBCF3CF5210EDBCFBE
:105A00003DF5220EDBCF3EF5230EDBCF3FF5240E16
:105A1000DBCF40F5250EDBCF41F5260EDBCF42F57F
:105A2000270EDBCF43F5280EDBCF44F5290EDBCF65
:105A300045F52A0EDBCF46F52B0EDBCF47F52C0EB6
:105A4000DBCF48F52D0EDBCF49F52E0EDBCF4AF527
:105A50002F0EDBCF4BF5300EDBCF4CF5310EDBCF0D
:105A60004DF5320EDBCF4EF5330EDBCF4FF5340E56
:105A7000DBCF50F5350EDBCF51F5360EDBCF52F5CF
:105A8000370EDBCF53F5380EDBCF54F5390EDBCFB5
:105A900055F53A0EDBCF56F53B0EDBCF57F53C0EF6
:105AA000DBCF58F53D0EDBCF59F53E0EDBCF5AF577
:105AB000276B0701E35102E097EC40F03F0EE15CF9
:105AC00002E2E16AE552E16E2BEF35F017EC35F0BA
:105AD000100EE12402E3E168E6520AEC38F0F3EC40
:105AE00035F0EEEC37F0040F96EC37F062EC37F05F
:105AF000080F96EC37F00E01BF516FE028EC35F03F
:105B000002E10701B48D0701B45173E1CFEC36F027
:105B100004E2850E006EB90E5DD017EC38F002E697
:105B2000EEEC35F005E2D950040F4DEC36F004D020
:105B300023EC38F003EC36F0CFEC37F002E677ECEC
:105B400035F004E23C0E006EBA0E44D02FEC38F073
:105B500004E2550E006EB90E3DD0D9EC34F00C0FB6
:105B600081EC35F009E39AEC37F0A8EC35F004E06D
:105B70002F0E006EB90E2ED0C3EC37F002E6EEEC1D
:105B800035F005E2D950080F4DEC36F004D0B7ECF3
:105B900037F003EC36F0CFEC37F002E677EC35F077
:105BA00004E20E0E006EBA0E15D02FEC38F004E2AF
:105BB000FF0E006EB80E0ED0D9EC34F00C0F81EC55
:105BC00035F00BE39AEC37F0A8EC35F006E0D90E8F
:105BD000006EB80E0FEC38F00CD000EC38F002E29A
:105BE000E16AE552E16E00500701E35102E097ECF3
:105BF00040F0100EE15C02E2E16AE552E16E2BEF4B
:105C000035F017EC35F0180EE12402E3E168E652B6
:105C10000AEC38F020EC37F0E1EC38F00C0FF0EC47
:105C200038F0100F96EC37F028EC35F002E1070160
:105C3000B48D100EDBCF00F0110EDBCF01F0120E91
:105C4000DBCF02F0130EDBCF03F0D9500C0F91EC39
:105C500037F0EE500026EE500122EE500222EE50B8
:105C60000322040E00C0DBFF050E01C0DBFF060EA1
:105C700002C0DBFF070E03C0DBFF9AEC37F0DBCF7F
:105C800007F0D950100F91EC37F0EE50045C006E25
:105C9000EE500558016EEE500658026EEE50075851
:105CA000036E080E00C0DBFF090E01C0DBFF0A0E09
:105CB00002C0DBFF0B0E03C0DBFF17EC38F002E67F
:105CC000EEEC35F005E2D950040F5BEC36F004D071
:105CD00023EC38F010EC36F0CFEC36F004E2850E11
:105CE000006EB90E4AD03BEC38F002E677EC35F0A6
:105CF00004E23C0E006EBA0E40D047EC38F004E2ED
:105D0000550E006EB90E39D0D9EC34F0140F81EC79
:105D100035F007E353EC38F004E02F0E006EB90EB7
:105D20002CD0C3EC37F002E6EEEC35F005E2D950AA
:105D3000080F5BEC36F004D0B7EC37F010EC36F01F
:105D40003BEC38F002E677EC35F004E20E0E006E24
:105D5000BA0E13D047EC38F004E2FF0E006EB80E16
:105D60000CD0D9EC34F0140F81EC35F009E353EC8E
:105D700038F006E0D90E006EB80E0FEC38F00CD0FB
:105D80000701B45109E100EC38F002E2E16AE552A2
:105D9000E16E005097EC40F0180EE15C02E2E16A1F
:105DA000E552E16E2BEF35F017EC35F0370EE124BC
:105DB00002E3E168E6520AEC38F08BEC35F010ECC7
:105DC00039F017E15FEC38F014E1020EF36E100EBB
:105DD000F3CFDBFFBCEC35F02A0E34C0DBFF2B0E1B
:105DE00035C0DBFF2C0E36C0DBFF2D0E37C0DBFFCE
:105DF00064D12A0EDB6A2B0EDB6A2C0EDB6A2D0EB9
:105E0000DB6A290EDB6A8D908B92D950F60FB3ECCA
:105E100038F002E698EC35F01FE2290EDB5002095B
:105E2000E76E290EE7CFDBFFF60EDBCF38F0F70E7B
:105E3000DBCF39F0F80EDBCF3AF0F90E31EC35F06C
:105E4000F60E34C0DBFFF70E35C0DBFFF80E36C0B0
:105E5000DBFFF90E37C0DBFFD950F20FB3EC38F09F
:105E600002E698EC35F01FE2290EDB500809E76ED8
:105E7000290EE7CFDBFFF20EDBCF38F0F30EDBCFDE
:105E800039F0F40EDBCF3AF0F50E31EC35F0F20ECE
:105E900034C0DBFFF30E35C0DBFFF40E36C0DBFF92
:105EA000F50E37C0DBFFD950F60FB3EC38F002E641
:105EB0003AEC37F030E2BCEC35F0040E34C0DBFFD6
:105EC000050E35C0DBFF060E36C0DBFF070E37C000
:105ED000DBFF8BEC35F00F0E1F0B03E0AFEC35F062
:105EE000FDE1E6EC34F0CCEC35F08BEC35F00F0E48
:105EF0001F0B03E0AFEC35F0FDE1C2EC38F014E22B
:105F00009BEC36F003E0AFEC35F0FDE1E6EC34F06D
:105F1000EDEC36F009D08BEC35F0E0EC35F074ECBC
:105F200037F0FDE1F4EC38F0DAEC36F00CE265EC39
:105F300035F0A40E006EB80E6FEC38F002E2E16AA4
:105F4000E55212EC37F028EC35F012E1F60EDBCF1B
:105F500004F0F70EDBCF05F0F80EDBCF06F0F90EFC
:105F6000A8EC35F005E0790E006EB80E03EC39F0C0
:105F700067EC35F009E2AAEC36F003E07BEC37F091
:105F8000FDE137EC36F006D0B6EC36F003E0AFECCE
:105F900035F0FDE161EC36F0110EEECFDBFF120EB5
:105FA000EECFDBFF130EEECFDBFF140EB7EC38F0B5
:105FB000F60FE96EFF0E7DEC36F0190EDB6A1A0E55
:105FC000DB6A1B0EDB6A1C0EDB6AD950F20FB3ECE6
:105FD00038F002E63AEC37F022E21DEC36F00F0E14
:105FE0001F0B03E0AFEC35F0FDE1E6EC34F0CCEC58
:105FF00035F01DEC36F00F0E1F0B03E0AFEC35F063
:10600000FDE1C2EC38F014E29BEC36F003E0AFECBB
:1060100035F0FDE1E6EC34F0EDEC36F009D01DECA6
:1060200036F0E0EC35F074EC37F0FDE1F4EC38F0EC
:10603000DAEC36F00CE265EC35F0440E006EB80E8A
:106040006FEC38F002E2E16AE55212EC37F028EC2E
:1060500035F008E15FEC38F005E0190E006EB80E7F
:1060600003EC39F067EC35F009E2AAEC36F003E016
:106070007BEC37F0FDE137EC36F006D0B6EC36F0CD
:1060800003E0AFEC35F0FDE161EC36F078EC38F090
:10609000180EB7EC38F0F20FE96EFF0E8CEC36F00C
:1060A0001D0EDB6A1E0EDB6A1F0EDB6A200EDB6A2A
:1060B000010EF36E100EF3CFDBFF05012751FDE05B
:1060C000100EDBCF34F5110EDBCF35F5120EDBCF22
:1060D00036F5130EDBCF37F5140EDBCF38F5150E82
:1060E000DBCF39F5160EDBCF3AF5170EDBCF3BF5DC
:1060F000180EDBCF3CF5190EDBCF3DF51A0EDBCFCA
:106100003EF51B0EDBCF3FF51C0EDBCF40F51D0E21
:10611000DBCF41F51E0EDBCF42F51F0EDBCF43F583
:10612000200EDBCF44F5210EDBCF45F5220EDBCF71
:1061300046F5230EDBCF47F5240EDBCF48F5250EC1
:10614000DBCF49F5260EDBCF4AF5270EDBCF4BF52B
:10615000280EDBCF4CF5290EDBCF4DF52A0EDBCF19
:106160004EF52B0EDBCF4FF52C0EDBCF50F52D0E61
:10617000DBCF51F52E0EDBCF52F52F0EDBCF53F5D3
:10618000300EDBCF54F5310EDBCF55F5320EDBCFC1
:1061900056F5330EDBCF57F5340EDBCF58F5350E01
:1061A000DBCF59F5360EDBCF5AF5276B370EE15CA6
:1061B00002E2E16AE552E16E2BEF35F017EC35F0C3
:1061C000110EE12402E3E168E65243EC37F005ECFE
:1061D00035F0100EDB6A0501275102E1340502E0BB
:1061E000000502E1010EDF6E34052BE1346B090E70
:1061F00045C5DBFF0A0E46C5DBFF0B0E47C5DBFFBF
:106200000C0E48C5DBFF0D0E49C5DBFF0E0E4AC55F
:10621000DBFF0F0E4BC5DBFF100E4CC5DBFF456BE4
:10622000466B476B486B496B4A6B4B6B4C6B3D6BDA
:106230003E6B3F6B406B416B426B436B446B010E9B
:10624000276F000529E1006B010E11C5DBFF020E6F
:1062500012C5DBFF030E13C5DBFF040E14C5DBFF05
:10626000050E15C5DBFF060E16C5DBFF070E17C5AD
:10627000DBFF080E18C5DBFF116B126B136B146B81
:10628000156B166B176B186B096B0A6B0B6B0C6B32
:106290000D6B0E6B0F6B106BD950050FCEDBD95009
:1062A000010FCBDBD9500D0FC8DBD950090FC5DB6F
:1062B000DFCFE6FFE66A040E006EB80EC0DB036EA9
:1062C000150EE15C02E2E16AE55256EC37F0110E80
:1062D000E15C02E2E16AE552E16EBDD3D8C500F0AF
:1062E000016A00BE016882EC37F0FF0E026EB70E45
:1062F0002AEC36F002E2E16AE552E16E055097EFD2
:1063000040F06BEC38F0DE6ADD6A010EE66ED3EC2D
:1063100038F0030E47DB0701B4510FE10501D80542
:1063200004E187EC37F0E66A04D087EC37F0010E21
:10633000E66E4CEC37F097EC40F0E552E5528BD32B
:106340006BEC38F0BAEC36F050EC37F012EC38F079
:1063500094EC38F08CEC37F00701B45129E1030ECE
:10636000DB50070802E250EC37F0DF50010802E290
:10637000010EDF6E030EDB50030F0E01B65D0CE065
:106380006EEC36F002E2E16AE552E16E0050030E77
:10639000DB50030F0E01B66F010EDBCFE6FF020EDE
:1063A000DBCFE6FFDFCFE6FF4CEC37F097EC40F0B9
:1063B000050EE15C02E2E16AE552E16E4CD36BEC62
:1063C00038F0E652E652FD0EDB040BE1B0CEDEFF04
:1063D000B1CEDDFF020EB2CEDBFF030EB3CEDBFF8C
:1063E0000AD0AECEDEFFAFCEDDFF020EB4CEDBFFB5
:1063F000030EB5CEDBFFFB0EDBCFE6FFFC0EDBCFE3
:10640000E6FF020EDBCFE6FF030EDBCFE6FFB6CEE4
:10641000E6FF87EC37F06FEC63F0006E070EE15C8F
:1064200002E2E16AE552E16E0050040EE15C02E234
:10643000E16AE552E16E0FD36BEC38F0E652D3DB44
:1064400099EC38F039E10701B45156E10501D75113
:1064500003E0020ED75D28E1DF50000821E2D751AA
:1064600001E18D90DF0403E18D848D82898C020E21
:10647000DF5C03E18D848D82899C030EDF5C03E188
:106480008D948D82899C040EDF5C03E18D848D9256
:10649000899C050EDF5C10E18D948D92899C0CD057
:1064A000D7510AE18D8008D0D70506E1DF500008FA
:1064B00002E28C9201D08C8262EC37F0010F12DB89
:1064C00099EC38F017E10701B45116E10501D751F5
:1064D00008E1010EDB50000802E28B920BD08B82A8
:1064E00009D0D70507E1010EDB50000802E28992CE
:1064F00001D0898297EC40F0FAEC38F0ACD2FE0E75
:106500000501D95DFF0EDA59FF0EDB59FF0EDC598C
:1065100005E2D92B000EDA23DB23DC2397EF40F0D2
:106520000501D951DA11DB11DC1105E0D907000EA4
:10653000DA5BDB5BDC5B97EF40F06BEC38F0E6524C
:10654000E652E65250DB070E2DDA8CEC37F0DB50CA
:106550000BE1DFCFD9F5010EDBCFDAF5020EDBCF91
:10656000DBF5030EDBCFDCF597EC40F0050EE15CCC
:1065700002E2E16AE552E16E6ED2D9C5E6FFDAC504
:10658000E6FFDBC5E6FFDCC5E6FFF60E006EB70EE4
:106590006FEC38F002E2E16AE55256EF37F0E66A56
:1065A000DD0EE66E050EE66E15EC39F00701B4510E
:1065B00001E0120097EF40F0DDC500F0016A00BE77
:1065C000016882EC37F0EF0E026EB70E43DB02E299
:1065D000E16AE552E16E055097EF40F0DEC500F04C
:1065E000016A00BE016882EC37F0E90E026EB70E58
:1065F00031DB02E2E16AE552E16E05500501DE6B36
:1066000097EF40F09DBCFED716C1E6FF17C1E6FF2D
:1066100000C1E6FF01C1E6FFDD0E006EB70E6FECB4
:1066200038F002E2E16AE55256EF37F06BEC38F0F1
:10663000A1DB030EDB6A12EC38F08CEC37F094EC43
:1066400038F00701B45101E081D0ECEC38F0FF0ED6
:10665000D880EE54030EED5407E2010EDB68030E02
:10666000F36E020EF3CFDBFFDF50010802E2010EF2
:10667000DF6E030EDB50010802E250EC37F0DF045E
:1066800009E1040EDB50030805E10501E16B020E90
:10669000E26F06D0010EDBCFE1F5020EDBCFE2F5B3
:1066A000CAB415D0CB68FC0ECA140009CA6E9D92FC
:1066B0000F0152815293F00EBA140C09BA6E3F0EBC
:1066C000BA140009BA6E0E010E0ECC6FCA84030E06
:1066D000DB502AE1DF5023E0E1C500F0E2C501F024
:1066E000D89001320032D890013200320050BB6E97
:1066F000E1C502F0E2C503F0040ED890023603367D
:10670000E804FBE1300E0216000E0316CF0EBA1499
:1067100000010210006E03C001F0E85003D0BB6A14
:10672000CF0EBA14BA6E10D005012751FDE0E1C5B5
:1067300059F5E2C55AF54E6B4F6B506B516BDFCF7D
:1067400058F5040E346F276B97EC40F0050EE15CB2
:1067500002E2E16AE552E16E7ED1120068D92B0EA9
:10676000E12402E3E168E6528EDBF29E040E00C5EE
:10677000DBFF050E01C5DBFF060E02C5DBFF070EC2
:1067800003C5DBFF080E04C5DBFF090E05C5DBFFF3
:106790000A0E06C5DBFF0B0E07C5DBFF0C0E08C596
:1067A000DBFF0D0E09C5DBFF0E0E0AC5DBFF0F0E6A
:1067B0000BC5DBFF100E0CC5DBFF110E0DC5DBFF9B
:1067C000120E0EC5DBFF130E0FC5DBFF140E10C536
:1067D000DBFF150E11C5DBFF160E12C5DBFF170E12
:1067E00013C5DBFF180E14C5DBFF190E15C5DBFF43
:1067F0001A0E16C5DBFF1B0E17C5DBFF1C0E18C5D6
:10680000DBFF1D0E19C5DBFF1E0E1AC5DBFF1F0EB9
:106810001BC5DBFF200E1CC5DBFF210E1DC5DBFFEA
:10682000220E1EC5DBFF230E1FC5DBFF240E20C575
:10683000DBFF250E21C5DBFF260E22C5DBFF270E61
:1068400023C5DBFF280E24C5DBFF290E25C5DBFF92
:106850002A0E26C5DBFFF28E1E0EDBCF00F01F0EC8
:10686000DBCF01F0200EDBCF02F0210E74EC38F00C
:1068700002E0010EDF6E040EDB5002E0010EDF6E5F
:106880000501275106E1010EDF6EF36E030EF3CF13
:10689000DBFFDF5010E0150EDBCF00F0160EDBCF74
:1068A00001F0170EDBCF02F0180E74EC38F003E0A5
:1068B000DE52010EDD6EDF5012E0190EDBCF00F06C
:1068C0001A0EDBCF01F01B0EDBCF02F01C0E74ECB6
:1068D00038F005E0010EF36E020EF3CFDBFF030E7E
:1068E000DBCFE6FFE66A020EDBCFE6FFE66A010ECB
:1068F000DBCFE6FFE66ADFCFE6FFE66ACC0E006E8E
:10690000B70E9DD8036E0B0EE15C02E2E16AE55220
:10691000E16E03502B0EE15C02E2E16AE552E16EAA
:106920009AD085D8080EE12402E3E168E652E16ED0
:10693000F29E28C5DFFF010E29C5DBFF020E2AC526
:10694000DBFF030E2BC5DBFF040E2CC5DBFF050EA2
:106950002DC5DBFF060E2EC5DBFF070E2FC5DBFFA7
:10696000F28E08EC39F0C20E006EB70E68D8036ED6
:106970000B0EE15C02E2E16AE55298DA080EE15C96
:1069800002E2E16AE552E16E66D0F29E0501286BF3
:10699000296B2A6B2B6B2C6B2D6B2E6B2F6BF28E56
:1069A00097EF40F0E66E2CEC47F0FAEC38F0E55249
:1069B000120001DB1F0E3D6E050E3E6E3F6A406AFF
:1069C000CDDA0AEC6AF0A7DBD9501200C7DA040E60
:1069D000DBCF3DF0050EDBCF3EF0060EDBCF3FF008
:1069E000070ED8EF38F0DBCF03F0B8DADFCF3DF099
:1069F000010EDBCF3EF0020EDBCF3FF0030ED8DB03
:106A0000D880190E3854C6EF38F0040EDB6A050E34
:106A1000DB6A060EDB6A070EDB6A080EDB6A090E0C
:106A2000DB6A0A0EDB6A0B0EDB6AE5EF37F0BBDBD5
:106A3000E1CFD9FFE2CFDAFF120073DA63D3016E40
:106A4000026A00C0E6FFE66E02C0E6FFA9EF68F04A
:106A5000B2DA10EF39F0E552E5CFDAFFE7CFD9FF30
:106A60001200DBCF3BF03D683E683F68406880EF36
:106A700069F0DBCF07F004C038F005C039F006C07C
:106A80003AF007C03BF003EC59F01C0EDBCF3EF0B0
:106A90001D0EDBCF3FF01E0EDBCF40F01F0EDBCF15
:106AA00041F06FEC59F04CDB210E3E6EE60E3F6E6E
:106AB0005B0E406E400E416E6FEC59F073EF5AF072
:106AC00044DA00C039F0BBEF38F076DB1BD3D95085
:106AD000FA0FE96EFF0EDA20EA6ED8801E0EEE5431
:106AE000000E5BD3E66E000EDA20E66E1200D88050
:106AF000FF0E3954FF0E3A54FF0E3B54000E3C5427
:106B000012000FDAEE50385CEE503958EE503A5819
:106B1000EE503B581200F60EDBCF00F0F70EDBCF45
:106B200001F0F80EDBCF02F0F90EDBCF03F012001C
:106B3000000EEE5C000EEE58000EEE58000EEE5801
:106B40001200DA20EA6ED890030EEB50000A120011
:106B5000DBCF07F004500510061007101200D89084
:106B60000036013602360336E8061200DBCF3CF071
:106B70003C34000E3C181200FA0EDBCF00F0FB0E86
:106B8000DBCF01F0FC0EDBCF02F0FD0EDBCF03F01C
:106B9000E0DAE4D980EF69F038C0DEFF39C0DEFF0B
:106BA0003AC0DEFF3BC0DDFFDD52DD52120039C0CE
:106BB00004F03AC005F03BC006F03CC007F01200FC
:106BC000CDD9FA0EDBCF3DF0FB0EDBCF3EF0FC0E55
:106BD000DBCF3FF0FD0EECDA0F0E1200D880D6DAD4
:106BE000000E3C541200E66AD3EF38F0080E34C0B1
:106BF000DBFF090E35C0DBFF0A0E36C0DBFF0B0ED4
:106C000037C0DBFF12000C0E34C0DBFF0D0E35C0A9
:106C1000DBFF0E0E36C0DBFF0F0E37C0DBFF1200AE
:106C2000140E34C0DBFF150E35C0DBFF160E36C068
:106C3000DBFF170E37C0DBFF1200F20EDBCF00F0D8
:106C4000F30EDBCF01F0F40EDBCF02F0F50EDBCF5D
:106C500003F01200036E046A02C0E6FFE66E04C091
:106C6000E6FFA9EC68F0056E050EE15C1200D95054
:106C70000C0F57D90450EE24006E0550EE20016E23
:106C80000650EE20026E0750EE20036E1200DE6A00
:106C9000DE6ADD6ADD52DD52120043D90C0EEECF02
:106CA000DBFF0D0EEECFDBFF0E0EEECFDBFF0F0E88
:106CB000EECFDBFF120035D9140EEECFDBFF78EFFD
:106CC00038F000C0DFFF010E01C0DBFF020E02C082
:106CD000DBFF030E03C0DBFFDCEF38F0000EE66ED7
:106CE000E66AE66EE66AB6CEE6FFE66EE66A6FEC48
:106CF00063F0006E070EE15C1200DA20EA6E210EEE
:106D0000EECFDBFF220EEECFDBFF230EEECFDBFF5D
:106D1000240EEECFDBFF1200DA20EA6E250EEECF56
:106D2000DBFF260EEECFDBFF270EEECFDBFF280EBC
:106D3000EECFDBFF1200080EDBCF00F0090EDBCF39
:106D400001F00A0EDBCF02F00B0EDBCF03F0100ECA
:106D50001F0B120031DAEECF04F0EECF05F0EECFCC
:106D600006F0EFCF07F0100E1F0B120024D9100E03
:106D70001F0B1200E652E652E652DF6A010EDB6A92
:106D8000020EDB6A120028DAEE50ED101200040E3B
:106D9000DBCF3AF0050EDBCF3BF0ECEF58F00CDA2E
:106DA000D880FF0EEE54FF0EEE54FF0EEE54000E90
:106DB000EE54120001DAD880000EEE54800EEDD1B0
:106DC000180EDBCF00F0190EDBCF01F01A0EDBCF6F
:106DD00002F01B0EDBCF03F012000C0E38C0DBFFFD
:106DE0000D0E39C0DBFF0E0E3AC0DBFF0F0E3BC0AD
:106DF000DBFF1200040EDBCF00F0050EDBCF01F04D
:106E0000120008C038F009C039F00AC03AF0120088
:106E100088D8A80ED880EE54610EED54120090D997
:106E2000140E1200E16E0350DE6A800EDE6EDE6A22
:106E3000DD6ADD52DD521200CFD9010EEE181200CC
:106E4000100EDB6A110EDB6A120EDB6A130EDB6AB0
:106E5000120039C008F03AC009F03BC00AF03CC04B
:106E60000BF01200060EDBCF3AF0070EDBCF3BF043
:106E7000ECEF58F0FF0EEE5CFF0EEE58010EEE58F0
:106E8000000EEE581200E16EDF6A010EDB6A020EA0
:106E9000DB6A030EDB6A1200DFEC31F0FAEF38F048
:106EA000010EF36E030EF3CFDBFF1200E16E035011
:106EB00097EF40F0D76F96809482958C958E958849
:106EC000958A1200010EE66ED9501200F36E010E83
:106ED000F3CFDBFF020EDB6A1200010EDBCFB2FE46
:106EE000020EDBCFB3FE1200D890383639363A3670
:106EF0003B36E8061200D8900436053606360736CB
:106F0000E806120000C0E6FF01C0E6FF1200DECF77
:106F1000E6FFDDCFE6FF1200E76E040EE7CFDBFFF2
:106F20001200E96E000EDA20EA6E1200DBDD060EBA
:106F3000D2EF34F00C0EDBCF04F00D0EDBCF05F0FA
:106F40000E0EDBCF06F00F0E120039C03EF03AC035
:106F50003FF03BC040F03CC041F0120000C038F0B0
:106F600001C039F002C03AF003C03BF01200080E35
:106F7000DBCF38F0090EDBCF39F00A0EDBCF3AF069
:106F80000B0E31EF35F0080EDBCF39F0090EDBCFF9
:106F90003AF00A0EDBCF3BF00B0EB6EF35F00C0EDD
:106FA000DBCF39F00D0EDBCF3AF00E0EDBCF3BF02E
:106FB0000F0EB6EF35F000D9EECF00F0EECF01F0B6
:106FC000EECF02F0EFCF03F012000C0EDB6A0D0ED5
:106FD000DB6A0E0EDB6A0F0EDB6A1200070EE2DCC4
:106FE000E66AD9501200DBCF0BF00BDF0BC03BF091
:106FF00003EC59F0DCDD64DD6FEC59F073EF5AF00F
:10700000D950080F1ADD04D9D4EC2EF0006E0C0E06
:10701000E15C1200E16EDE6A3ADE05EF35F00FDD6D
:10702000FAEF38F0E0DD01D94DDFFEEF38F0040E65
:10703000DBCF39F0050EDBCF3AF0060EDBCF3BF0AD
:10704000070EB6EF35F0040EDBCF38F0050EDBCFC0
:1070500039F0060EDBCF3AF0070E31EF35F00C0EAB
:10706000DBCF00F00D0EDBCF01F00E0EDBCF02F018
:107070000F0EF3EF34F0140EDBCF39F0150EDBCF2B
:107080003AF0160EDBCF3BF0170EB6EF35F0140ECC
:10709000DBCF00F0150EDBCF01F0160EDBCF02F0D8
:1070A000170EF3EF34F0140EDBCF04F0150EDBCF28
:1070B00005F0160EDBCF06F0170EA8EF35F0F20E36
:1070C000DBCF04F0F30EDBCF05F0F40EDBCF06F0E0
:1070D000F50EA8EF35F0ABDCE652E6521200AFDC5D
:1070E000036E070EE15C1200DBCF03F010EF39F006
:1070F000150EEECFDBFF160EEECFDBFF170EEECF39
:10710000DBFF1200EECFE6FFEECFE6FFEECFE6FFAD
:10711000EFCFE6FF120038C000F039C001F03AC0EE
:1071200002F03BC003F01200CDDE030FDBDC15EFF5
:1071300039F07BD8E76E020EE7CFDBFFDB501200A1
:1071400039C000F03AC001F03BC002F03CC003F08F
:107150001200190E3D6E3E6A3F6A406A1200E96EE7
:10716000000EA1EF35F0E96EFF0EA1EF35F0EECF86
:10717000DBFFD950120001C03AF002C03BF003C05F
:107180003CF0120023DC32DD67EF35F0000E39549D
:10719000000E3A54000E3B541200EE54000EEE5412
:1071A000000EEE541200D9CFE6FFDACFE6FF120050
:1071B000DBCF40F00AEF6AF0D9CFE9FFDACFEAFF80
:1071C0001200140EDB6A150EDB6A160EDB6A170E50
:1071D000DB6A09DDEEEF37F0D950010F91EF37F0A0
:1071E000A5DEE66AD9501200B4DF0AEC6AF0D4DCFE
:1071F000E5EF37F0E552E552E5521200010F72DC7F
:10720000030ED2EF34F00BDF010EDE6E47EF36F0E7
:10721000D950040F12DC65EF35F064DCEEEF37F087
:1072200000500110021003101200010ED2EF34F0D2
:10723000D8CFE4FFE0CFE4FFE46EE9CFE4FFEACF8C
:10724000E4FFF3CFE4FFF4CFE4FFE65228EC4BF089
:107250008FEC4AF0030EDB6AA4A6A4D1A4960E011B
:10726000002B0E01AB510E01005D01E284D0006BDA
:107270000E0165EC4AF0EF6A79907B6A7A6A0E013A
:10728000A92B0E01AA510E01A95D01E3A96B1EEC09
:107290004BF0EA22EE50ED106EE0E7EC4BF094EC90
:1072A0004BF002E14B50491847E032EC4BF0EA2238
:1072B000EE50ED103AE055EC4BF041EC4AF01EEC8C
:1072C0004BF0EA22EE504A5C486EEE504B58496E45
:1072D000020E48C0DBFF030E49C0DBFFAAEC4AF0F8
:1072E000493412E248500008000E49540DE2AAEC5D
:1072F0004AF032EC4BF06BEC4BF017E2CDEC4BF07C
:10730000EE264950ED2218D0AAEC4AF0486C491EEE
:10731000000E492232EC4BF06BEC4BF006E2CDEC68
:107320004BF0EE5E4950ED5A07D0E7EC4BF0EA2205
:1073300048C0EEFF49C0EDFF65EC4AF0120EEF6E5B
:10734000F29E0E011EEC4BF0FDEC49F049C048F0F6
:10735000496A4850B66E1EEC4BF0FDEC49F04850BF
:10736000B56EF00EB4140009B46EF00EB414090931
:10737000B46E7980F28E0701000ED880AA55000EF7
:10738000AB552EE2B82B000EB923AA51B85DAB5114
:10739000B95926E3B86BB96B030EAE5D1FE2AC5171
:1073A000EA6A200FE96E010EEA2280CFEFFFAC51AE
:1073B000EA6A230FE96E010EEA2281CFEFFFAC519A
:1073C000EA6A260FE96E010EEA2282CFEFFFAC2BAC
:1073D000030EAC5D01E3AC6BAE2B02D0AA6BAB6BC2
:1073E000000ED880AF55000EB0551CE2000ED880BC
:1073F000BE55000EBF5516E2BA2B000EBB23AF518F
:10740000BA5DB051BB590EE3BA6BBB6B030EB35DF3
:1074100007E2B12B030EB15D01E3B16BB32B02D0D8
:10742000AF6BB06BBE51BF110BE0050EBD5D07E346
:10743000C18C9E9C9D8CC280C282BD6B01D0BD2B35
:107440000601005101E1AAD0DE6ADD6ADECF48F014
:10745000DDCF49F0040E485C000E495801E39ED090
:10746000E4EC49F0010E47EC4AF0FDE1010EE9269B
:10747000060EEA22EE50ED1075E0E4EC49F0010E44
:1074800047EC4AF0FDE198EC4BF0EE50ED1016E1C0
:107490009DEC4BF001E18180A1EC4BF003E1ED505C
:1074A00001E18182A5EC4BF003E1ED5001E1818423
:1074B000A9EC4BF003E1ED5001E18186E4EC49F0E9
:1074C000010E47EC4AF0FDE14BEC4BF047EC4AF083
:1074D000FDE1010EE926060E94EC4BF019E14B504C
:1074E000491816E19DEC4BF001E18190A1EC4BF0C5
:1074F00003E1ED5001E18192A5EC4BF003E1ED5089
:1075000001E18194A9EC4BF003E1ED5001E181969A
:10751000E4EC49F0010E47EC4AF0FDE198EC4BF049
:10752000EE2A000EEF22E4EC49F0010E47EC4AF09F
:10753000FDE14BEC4BF047EC4AF0FDE1090EE9268A
:10754000060E94EC4BF024E14B50491821E1E4EC99
:1075500049F0010E47EC4AF0FDE198EC4BF0EE6A81
:10756000ED6A16D09DEC4BF001E18190A1EC4BF05F
:1075700003E1ED5001E18192A5EC4BF003E1ED5008
:1075800001E18194A9EC4BF003E1ED5001E181961A
:10759000DF2A010E01E25AD7DB2A58D70501E05154
:1075A00001E0E0079EAC3DD09E9CC1AC07D0C19CE1
:1075B000010E0701C06FC16BBC6B18D0C4504A6E7E
:1075C0004B6E4A6AC35000014A10486E4BC049F0E6
:1075D0000701BC51E96EEA6A84EC4AF048C0EEFF4C
:1075E00049C0EDFFD890C037C137BC2B100EBC5D31
:1075F0000EE2C051BE15486EC151BF15496E4850CC
:10760000491005E1BC2BD890C037C137EFD7100E19
:10761000BC5D02E39D9C05D0BC51040DF328C26EF5
:10762000C282F2A435D0D59EF294F29A040E486E2E
:107630000701B75195EC4AF0EF50485C29E1080E7C
:10764000B75D0AE2C8EC4AF004E0E846FE0B4806E3
:10765000FCE1E81C891616D0100EB75D0AE2C8ECF2
:107660004AF004E0E846FE0B4806FCE1E81C8A16F6
:1076700009D0C8EC4AF004E0E846FE0B4806FCE1FD
:10768000E81C8B160701B75195EC4AF0020EEF6E1D
:10769000040EE15C02E2E16AE552E16EE552E5CFFB
:1076A000DAFFE7CFD9FFE552E5CFF4FFE5CFF3FFEF
:1076B000E5CFEAFFE5CFE9FFE550E5CFE0FFE5CF15
:1076C000D8FF1000D3EC4BF0E652896A92680701AC
:1076D000BE6BBF6B8A6A93688B6A94688C968C9435
:1076E00095969594928E010EE36F0501F369F46906
:1076F0000701B26BB16BB36BAD6BAC6BAE6BAA6BCE
:10770000AB6BAF6BB06BB86BB96BBA6BBB6BBC6B75
:1077100076827680769C769A76887696FA0E776E62
:10772000DE6ADD6A2CEC4AF004E6100E005C000E06
:1077300001580BE2E4EC49F084EC4AF0EE6AED6AA1
:10774000DF2A010EEFE3DB2AEDD70701DD6BDE6BED
:10775000DB6BDC6BDE6ADD6A2CEC4AF004E6400E83
:10776000005C000E01580CE2E4EC49F0000EE92642
:10777000020EEA22EF6ADF2A010EEEE3DB2AECD7E3
:10778000DE6ADD6A2CEC4AF004E6400E005C000E76
:1077900001580CE2E4EC49F0400EE926020EEA2220
:1077A000EF6ADF2A010EEEE3DB2AECD7DE6ADD6A40
:1077B0002CEC4AF004E6000E005C010E01580AE2CF
:1077C000E4EC49F0D4EC4AF0EF6ADF2A010EF0E372
:1077D000DB2AEED70701DF6BE06BE16BE26BB56B89
:1077E000B66BB76BDE6ADD6A2CEC4AF004E6180E65
:1077F000005C000E015812E2E4EC49F0DEEC4AF0C5
:10780000EE6AED6AE4EC49F0290EE926010EEA225F
:10781000010EEF6EDF2AE8E3DB2AE6D7D586D59A9C
:10782000D59CF294F29AF1940F01498FBE0EC16E6D
:10783000D08E7694A386A59679EC27F0A3EC62F01F
:10784000F28EF28C76840FEC46F0040EE15C02E2DC
:10785000E16AE552E16EC7EF49F028EC4BF0E652E1
:107860008FEC4AF0030EDB6A040EDB6AEBEC48F0A7
:107870000701AE5100080AE2DCEC41F00701AD2B34
:10788000030EAD5D01E1AD6BAE07F2D7B351000859
:107890000AE2FEEC41F00701B22B030EB25D01E1FA
:1078A000B26BB307F3D7200E0401E76E7819E8AE88
:1078B00002D0E73402D0E750785D01E23AD165505A
:1078C000020B01E036D1400EE66E400EE66E020E6F
:1078D000E66E3AEC61F0D7EC4BF0E76E030EE7CFC3
:1078E000DBFFDB50000801E3E7D0040EDB6A030E88
:1078F000DB50F36E040E4AEC4AF001E3DDD0040ED7
:10790000DB50EA6A400FE96E020EEA22EFCFDFFF9A
:1079100006015D5134E10D0E08EC4AF005E00A0E57
:10792000016EDF50015C2BE1010E5D6F070154EC2D
:107930004AF00D0EEF6EDD2B010EDB6ADD51F36EAA
:10794000010E4AEC4AF016E2D9EC4AF0E9BEEA68C8
:10795000D4EC4AF0EF50E66ED9EC4AF0E9BEEA68A2
:10796000190EE926060EEA22E552E750EF6E010EE7
:10797000DB2AE4D73BD90701DD6BDE6B8DD01B0E14
:10798000DF5C09E1595107E1010E596F1B0E5A6F77
:107990005B6B5C6B81D059050BE15B0EDF5C08E132
:1079A0001B0E5A5D05E15B5103E15B0E5B6F74D00A
:1079B00059054AE1410EDF5C47E11B0E5A5D44E187
:1079C0005B0E5B5D41E15A6B5B6B5C6B596B010E4F
:1079D000DB6ADBCFE9FFEA6AE9BEEA68D4EC4AF089
:1079E000EF500D0816E0D9EC4AF0E9BEEA68190E2E
:1079F000E926060EEA22EF50E66ED9EC4AF0E9BE1F
:107A0000EA68D4EC4AF0E552E750EF6E010EDB2A4B
:107A1000E0D7010EDBCFDDF7070154EC4AF0EF6A47
:107A2000F80E006EBC0E14EC4BF0000EE66E030E6A
:107A3000E66EF50E006EBC0E1BEC4BF002E2E16A46
:107A4000E552E16E035028D0080EDF5C0EE107011D
:107A5000DD5100080AE2DD0754EC4AF0EF6AF20E4D
:107A6000006EBC0E14EC4BF017D00D0EDF5C14E072
:107A70000A0EDF5C11E0200EDF5C0EE306015A6B9C
:107A80005B6B5C6B596B070154EC4AF0DFCFEFFF87
:107A900006015D6B0701DD2B0701DD51006E016AF8
:107AA000000E001806E1010E011803E1B487DD6B3A
:107AB000DE6B040EDB2A1BD70701B45139E0B4A1F9
:107AC00005D0EC0E006EBC0E14EC4BF00701B4A315
:107AD00005D0CD0E006EBC0E14EC4BF00701B4A522
:107AE00005D0B10E006EBC0E14EC4BF00701B4A72C
:107AF00005D0950E006EBC0E14EC4BF00701B4A936
:107B000005D0760E006EBC0E14EC4BF00701B4AD40
:107B100005D0550E006EBC0E14EC4BF00701B4AF4F
:107B200005D03C0E006EBC0E14EC4BF00701B46B9C
:107B300037D8050EE15C02E2E16AE552E16EC7EF7B
:107B400049F028EC4BF0DBC7DFFFDF2A400E08ECE2
:107B50004AF001E1DF6A0701DC51DF5C01E120D876
:107B60000701DB51EA6A000FE96E020EEA22FD0E00
:107B7000DBCFEFFFDB2B400EDB5D01E1DB6BDC518C
:107B8000DB5D01E1B485FD0EDBCF00F0016A00BED4
:107B9000016800C0F3FF01C0F4FFE552C7EF49F0F0
:107BA00028EC4BF00701DB51DC5D1DE00701905133
:107BB00005E0C4EC61F073EC4CF0F8D70701DC5140
:107BC000D880DB5507E2DC51DB5D1EEC4AF0DBC7F9
:107BD000DCF707D0400ED880DC551EEC4AF00701D8
:107BE000DC6BC4EC61F0E552C7EF49F0D3EC4BF02D
:107BF000E652DE6ADD6A020EDB6A030EDB6A07010B
:107C0000CDEC49F0EAEC4AF0020EF3CFDBFF0701BE
:107C1000E9EC49F004E1010E011801E1DE6B020E0E
:107C2000DB50DE6EDD6ACDEC49F02C0824E0CDECB3
:107C300049F00D0820E0CDEC49F0EAEC4AF0030EE3
:107C4000F3CFDBFF0701E9EC49F004E1010E011875
:107C500001E1DE6B020EDBCF02F002C003F0026A2C
:107C6000030EDB5000010224006E000E0320016EA3
:107C700000C0DEFFDD6E000EDFCF3AF0010EDBCF7D
:107C80003BF0420E3A1802E1520E3B1801E11FD2BE
:107C9000540E3A1802E1510E3B1801E115D2540E70
:107CA0003A1802E1530E3B1801E10BD2530E3A1879
:107CB00002E1430E3B1801E101D2530E3A1802E1F2
:107CC000510E3B1801E1F7D14D0E3A1802E1580E62
:107CD0003B1801E1EDD1530E3A1802E1450E3B1875
:107CE00001E1E3D1430E3A1802E1410E3B1801E1F4
:107CF000DAD14D0E3A1802E1510E3B1801E1D0D114
:107D00004D0E3A1802E1520E3B1801E1C6D1320E77
:107D10003A1802E1530E3B1801E1BCD1450E3A1866
:107D200002E1530E3B1801E1B2D1430E3A1802E1D1
:107D3000510E3B1801E1A8D14B0E3A1802E1430E57
:107D40003B1801E19ED14C0E3A1802E1420E3B185D
:107D500001E194D1440E3A1802E14E0E3B1801E1C4
:107D60008AD1490E3A1802E14E0E3B1801E180D14A
:107D7000420E3A1802E1510E3B1801E176D14C0E49
:107D80003A1802E1510E3B1801E16CD14C0E3A1841
:107D900002E1530E3B1801E162D14E0E3A1802E1A6
:107DA000510E3B1801E158D14E0E3A1802E1530E24
:107DB0003B1801E14ED1430E3A1802E1530E3B1835
:107DC00001E144D14D0E3A1802E1450E3B1801E1A4
:107DD0003AD1500E3A1802E1510E3B1801E130D170
:107DE000500E3A1802E1540E3B1801E126D1500E14
:107DF0003A1802E1530E3B1801E11CD14D0E3A181E
:107E000002E1410E3B1801E112D14D0E3A1802E198
:107E1000530E3B1801E108D1470E3A1802E1500E0B
:107E20003B1801E1FED0430E3A1802E1500E3B1818
:107E300001E1F4D0490E3A1802E1430E3B1801E18A
:107E4000EAD0490E3A1802E1520E3B1801E1E0D0A7
:107E5000490E3A1802E1530E3B1801E1D6D0530EF9
:107E60003A1802E1520E3B1801E1CCD0530E3A18F9
:107E700002E1530E3B1801E1C2D0530E3A1802E161
:107E8000420E3B1801E1B8D0430E3A1802E1420E0F
:107E90003B1801E1AED0430E3A1802E1520E3B18F6
:107EA00001E1A4D04F0E3A1802E1420E3B1801E165
:107EB0009AD0570E3A1802E14D0E3B1801E191D0CD
:107EC000520E3A1802E14D0E3B1801E188D0440EE3
:107ED0003A1802E1500E3B1801E17FD04F0E3A18DC
:107EE00002E1500E3B1801E176D0490E3A1802E14A
:107EF000500E3B186EE0580E3A1802E1540E3B1833
:107F000065E0540E3A1801E13B505EE0410E3A182C
:107F100001E13B5057E0560E3A1801E13B5050E06A
:107F2000490E3A1801E13B5049E04F0E3A1801E181
:107F30003B5042E0550E3A1802E1430E3B183AE03E
:107F4000580E3A1802E1430E3B1831E0430E3A183E
:107F500001E13B502AE0520E3A1801E13B5023E088
:107F6000580E3A1802E1520E3B181AE04D0E3A181C
:107F700002E14C0E3B1811E0030EDB5001E0AAD0E9
:107F8000020E9BEC4AF09BEC4AF0190E006EBC0E00
:107F90005AEC4BF001E3ADD0AAD0D0EC2BF0ABD033
:107FA0002AEC44F0A8D0CCD8A6D02ED9A4D02CEC62
:107FB00044F0A1D0C9D89FD0CBD99DD0FDD99BD0BA
:107FC00018DA99D01BDA97D0F6D895D028EC44F07F
:107FD00092D03BDB90D0A7DB8ED0A2DA8CD081DAB6
:107FE0008AD06DDA88D0A2EC44F085D02EEC44F033
:107FF00082D0A0EC44F07FD0A4EC44F07CD0A6EC7E
:1080000044F079D0A8EC44F076D0AAEC44F073D0D8
:10801000ACEC44F070D0AEEC44F06DD0B0EC44F079
:108020006AD00FEC45F067D066EC2DF064D01AEC06
:1080300029F061D0A0EC31F05ED081EC31F05BD062
:108040006EEC31F058D01CEC32F055D053EC28F0E7
:1080500052D09DEC32F04FD0BDEC32F04CD0CFEC92
:1080600032F049D0DCEC32F046D0EEEC32F043D0C6
:108070007FEC32F040D090EC32F03DD045EC45F052
:108080003AD054EC45F037D002EC33F034D016EC53
:1080900033F031D01AEC63F02ED0ADEC33F02BD0AE
:1080A000AEEC33F028D040D926D0DEEC30F023D02F
:1080B00001EC2EF020D091EC34F01DD0C5EC34F062
:1080C0001AD063EC46F017D0A8EC46F014D04DEC73
:1080D00045F011D071EC4BF071EC4BF0F10E006EED
:1080E000BB0EB5EC49F0036E0B0EE15C02E2E16AF7
:1080F000E552E16E03500701CDEC49F00D080DE0AB
:10810000B4510BE1520E006E016ADF50001803E11A
:10811000DE52DD50011801E0B48FDDC7DEF7040E3A
:10812000E15C02E2E16AE552E16EC7EF49F0070166
:10813000E35105E05C0E006ED40E14EC4BF012001F
:1081400062EC3BF097EF40F028EC4BF0BCEC4BF0CE
:10815000D6EC49F0020EC1EC4BF02BE1DF0412E14A
:1081600076EC4BF00AE0010E006E016ADB5000185D
:1081700008E1020EDB50011804E1010EDBCFE3F74A
:1081800001D0B48D020E08EC4AF012E176EC4BF00F
:108190000AE0010E006E016ADB50001808E1020ED1
:1081A000DB50011804E1010EDBCFBFFE01D0B48D1E
:1081B000BEDF30EF4BF0C1EC49F08FEC4AF0E66ADD
:1081C000A80EE66E070EE66EEBEC4BF01BE1020E1E
:1081D000DB500CE1A851A91103E1AA6BAB6B11D0E4
:1081E0007684A8C7AAF7A9C7ABF70BD0A851A911E5
:1081F00003E1AF6BB06B05D07684A8C7AFF7A9C712
:10820000B0F795DF30EF4BF0D3EC4BF0BCEC4BF01C
:1082100000EC4CF0020F00EC4CF0030F00EC4CF0C3
:10822000040F17EC4BF00FE1DF50926E010EDB50A4
:10823000936E020EDB50946E030EDB50956E040EAF
:10824000DB50966E74DF050EE15C02E2E16AE552F6
:10825000E16EC7EF49F0C1EC49F0FD0EDB501008AC
:1082600005E2100EF36EFD0EF3CFDBFFFC0EDB50CC
:108270002BE0FD0EDB508BEC6AF0F3500701BE13D0
:10828000F450BF13080EF36EFD0E4AEC4AF00DE2F7
:10829000010EF36EFD0EDB5003E0F0EC49F0FDE162
:1082A000F350F31C0F0148173DD0FD0EDB500C08B6
:1082B00039E3F1EC4AF004E0E846FE0B0006FCE18D
:1082C000E81C0F0149172ED0FD0EDB508BEC6AF035
:1082D000F3CF00F0F4CF01F0001E011E00500701A3
:1082E000BE170150BF17080EF36EFD0E4AEC4AF0A0
:1082F0000CE2010EF36EFD0EDB5003E0F0EC49F0F2
:10830000FDE1F3500F0148130DD0FD0EDB500C08BA
:1083100009E3F1EC4AF004E0E846FE0B0006FCE15C
:108320000F014913C7EF49F0C1EC49F0BCEC4BF029
:1083300017EC4BF009E1010EDBCFE6FFDFCFE6FFE4
:108340008ADFE552E552F3DEE552E552C7EF49F028
:10835000C1EC49F0E0EC49F0010EBEEC49F033EC21
:108360004AF026E1010EDB5002E1DF50896E2BEC72
:108370004BF01EE1010EDB5002E1DF508A6E2BEC68
:108380004BF016E1010EDB5002E1DF508B6E2BEC5F
:108390004BF00EE1010EDB5002E1DF508C6E2BEC56
:1083A0004BF006E1010EDB5002E1DF508D6EBFDEC7
:1083B000E552E552C7EF49F08450E66EE66A835015
:1083C000E66EE66A8250E66EE66A8150E66EE66A1E
:1083D0008050E66EE66AD40E006EBB0EB5EC49F036
:1083E000036E0D0EE15C02E2E16AE552E16E0350BC
:1083F0001200640E006ED40E14EF4BF0D3EC4BF071
:10840000DF6A010EF36EDB6E020EDB6AD20E006EC7
:10841000BB0E14EC4BF09DBCFED7DF6ADFCF00F043
:10842000100EE76E0018E8AE02D0E73402D0E75035
:10843000005C3EE2010EDB500701BE150001006E3C
:10844000020EDB500701BF150001016E0050011044
:108450001EE0DFCFE9FFEA6AE9BEEA6884EC4AF091
:10846000EECFE6FFEFCFE6FFDFCF00F0016A00BE00
:108470000168ADEC4BF0C70E026EBB0E9FEC4AF0EC
:10848000070EE15C02E2E16AE552E16E0550010E81
:10849000DBCF00F0020EDBCF01F0D89000360136C2
:1084A000010E00C0DBFF020E01C0DBFFDF2AB6D7E2
:1084B000610E006ED40E14EC4BF030EF4BF028EC54
:1084C0004BF0E0EC49F0EBEC4BF009E1B6EC4AF094
:1084D00005E2E4EC49F0020EDBCFEFFF28DE30EFDF
:1084E0004BF028EC4BF0E0EC49F0030EC1EC4BF004
:1084F00015E1B6EC4AF005E2E4EC49F0020EEFCFEC
:10850000DBFF020E9BEC4AF0BD0E006EBB0E1BECB7
:108510004BF002E2E16AE552E16E035030EF4BF0BE
:1085200004EC4CF001E08FD0020EDB50010801E2B8
:1085300087D0010EDB50070801E282D0410E08EC23
:108540004AF016E1020EDB500AE1F4EC49F003E0D8
:10855000F0EC49F0FDE1F350F31C921673D0F4EC0B
:1085600049F003E0F0EC49F0FDE1F35092126AD0DB
:10857000420E08EC4AF016E1020EDB500AE1F4EC80
:1085800049F003E0F0EC49F0FDE1F350F31C9316E1
:1085900059D0F4EC49F003E0F0EC49F0FDE1F35080
:1085A000931250D0430E08EC4AF016E1020EDB5055
:1085B0000AE1F4EC49F003E0F0EC49F0FDE1F3509E
:1085C000F31C94163FD0F4EC49F003E0F0EC49F0D2
:1085D000FDE1F350941236D0440E08EC4AF016E157
:1085E000020EDB500AE1F4EC49F003E0F0EC49F054
:1085F000FDE1F350F31C951625D0F4EC49F003E0AF
:10860000F0EC49F0FDE1F35095121CD0450E08EC5A
:108610004AF016E1020EDB500AE1F4EC49F003E007
:10862000F0EC49F0FDE1F350F31C96160BD0F4EC9E
:1086300049F003E0F0EC49F0FDE1F350961202D06E
:10864000B48D01D074DD30EF4BF0C1EC49F08FEC0C
:108650004AF0FAEC4BF0050E10EC4BF0010F17EC62
:108660004BF05FE1010EDB50070847E3410E08ECD9
:108670004AF009E1F4EC49F003E0F0EC49F0FDE1E7
:10868000F350801433D0420E08EC4AF009E1F4ECC8
:1086900049F003E0F0EC49F0FDE1F350811426D0FD
:1086A000430E08EC4AF009E1F4EC49F003E0F0EC89
:1086B00049F0FDE1F350821419D0440E08EC4AF061
:1086C00009E1F4EC49F003E0F0EC49F0FDE1F3508E
:1086D00083140CD0450E08EC4AF00FE1F4EC49F09D
:1086E00003E0F0EC49F0FDE1F3508414E76E020E74
:1086F000E7CFDBFFDB5008E002D0B48D12D0010ED3
:10870000F36E020EF3CFDBFF020E9BEC4AF0B40EC9
:10871000006EBB0E1BEC4BF002E2E16AE552E16E2B
:10872000035030EF4BF004EC4CF001E08FD0020E20
:10873000DB50010801E287D0010EDB50070801E29F
:1087400082D0410E08EC4AF016E1020EDB500AE13D
:10875000F4EC49F003E0F0EC49F0FDE1F350F31CD8
:10876000891673D0F4EC49F003E0F0EC49F0FDE138
:10877000F35089126AD0420E08EC4AF016E1020E5C
:10878000DB500AE1F4EC49F003E0F0EC49F0FDE1E4
:10879000F350F31C8A1659D0F4EC49F003E0F0ECE6
:1087A00049F0FDE1F3508A1250D0430E08EC4AF034
:1087B00016E1020EDB500AE1F4EC49F003E0F0ECC4
:1087C00049F0FDE1F350F31C8B163FD0F4EC49F077
:1087D00003E0F0EC49F0FDE1F3508B1236D0440E8B
:1087E00008EC4AF016E1020EDB500AE1F4EC49F025
:1087F00003E0F0EC49F0FDE1F350F31C8C1625D0BA
:10880000F4EC49F003E0F0EC49F0FDE1F3508C1298
:108810001CD0450E08EC4AF016E1020EDB500AE1CE
:10882000F4EC49F003E0F0EC49F0FDE1F350F31C07
:108830008D160BD0F4EC49F003E0F0EC49F0FDE1CB
:10884000F3508D1202D0B48D01D071DC30EF4BF0BB
:1088500097EF40F097EF40F097EF40F028EC4BF0A7
:10886000E652B6EC4BF052EC4BF062E1D950020FFD
:10887000F8EC49F0720ED880EE542E0EED543DE324
:10888000D950020FF8EC49F0EE50ED101FE00368EC
:108890000468056A2D0EE76E020EDBCF06F0030EAC
:1088A000DBCF07F0E7500626000E0722086A0650C5
:1088B000035C006E07500458016E08500558026EA4
:1088C000020E00C0DBFF030E01C0DBFF010EDB5018
:1088D000070813E3410E08EC4AF002E1DF6A0FD00B
:1088E000420E08EC4AF002E1080E05D0430E08ECF7
:1088F0004AF003E1100EDF6E02D0B48D19D0010EE4
:10890000DB50DF24E96EEA6ADEEC4AF0F8EC4AF06C
:10891000010EDB50DF2495EC4AF0EF0407E1010E75
:10892000DB50DF2495EC4AF0020EEF6E97EC40F03E
:10893000040EE15C02E2E16AE552E16EC7EF49F044
:1089400097EF40F097EF40F097EF40F097EF40F04F
:1089500097EF40F097EF40F097EF40F097EF40F03F
:10896000C1EC49F0070EE12402E3E168E652E16E52
:10897000FAEC4BF0030E10EC4BF052EC4BF047E1ED
:10898000DECF01F6DDCF02F6020EDBCF09F6030ED5
:10899000DBCF0AF6040EDB6A030EF36E040E4AEC1C
:1089A0004AF033E2010E15EC4AF0030EBEEC49F03A
:1089B000E76E050EE7CFDBFF010EE66ED950F6EC51
:1089C0004BF0BEEC49F0E76E060EE7CFDBFF070188
:1089D000B4511DE1050EDB5018E1060EDB5015E128
:1089E000E4EC4AF0010EE926060EEA22DECFEEFFA5
:1089F000DDCFEDFFE4EC4AF0090EE926060EEA228F
:108A0000F8EC4AF0040EDB2AC7D797EC40F0070ECB
:108A1000E15C02E2E16AE552E16EC7EF49F028EC61
:108A20004BF0FAEC4BF0010EC1EC4BF00DE1DF50D6
:108A300007E0F00E9314936E0601010E006F02D052
:108A40000601006B97EC40F0E552C7EF49F0D9CF33
:108A5000E6FFDACFE6FFE1CFD9FFE2CFDAFFE65259
:108A6000DF6AFF0EDF5C0AE2E868E85005E0E8062E
:108A700000D000D000D0F9D7DF2AF3D7E552E55275
:108A8000E5CFDAFFE7CFD9FF1200F29EF29C6592A4
:108A9000656ADDDF0FEF00F01200F29EF29C659236
:108AA000656AD5DFFF001200C1EC49F0100EE12429
:108AB00002E3E168E652E16EE66AD950010FD6ECB6
:108AC00049F0E66A7CEC4BF0FAEC4BF0010E10EC4E
:108AD0004BF0040FD6EC49F0020E10EC4BF0F6EC24
:108AE0004BF010EC4BF00A0FD6EC49F0060E10ECF0
:108AF0004BF0060FD6EC49F0070E10EC4BF00E0FC2
:108B0000D6EC49F0040E10EC4BF00F0FD6EC49F008
:108B1000050EBEEC49F0010EDBCF00F0016A00BE8D
:108B20000168ADEC4BF0A80E026EBB0E9FEC4AF054
:108B3000050EE15C02E2E16AE552E16E0550DFCF2D
:108B4000E6FFE66A9C0E006EBB0E1BEC4BF002E2E9
:108B5000E16AE552E16E0350040EDBCFE6FF050E3D
:108B6000DBCFE6FF900E006EBB0E1BEC4BF002E27B
:108B7000E16AE552E16E0350020EDBCFE6FF030E21
:108B8000DBCFE6FF840E006EBB0E1BEC4BF002E267
:108B9000E16AE552E16E0350D9500A0FF8EC49F052
:108BA000BFEC4AF0770E006EBB0E5AEC4BF002E2BF
:108BB000E16AE552E16E0350D950060FF8EC49F036
:108BC000BFEC4AF06A0E006EBB0E5AEC4BF002E2AC
:108BD000E16AE552E16E03500E0E9BEC4AF05E0E28
:108BE000006EBB0E1BEC4BF002E2E16AE552E16E57
:108BF00003500F0E9BEC4AF0520E006EBB0E1BECA6
:108C00004BF002E2E16AE552E16E035097EC40F06E
:108C1000100EE15C02E2E16AE552E16EB8D3B1DB2D
:108C2000120EE12402E3E168E652E16E110EDB6A06
:108C3000F36EDBCFF4FFE850F45C03E237EC4BF06B
:108C4000F7D764EC4BF002E2E16AE552E16E0050C6
:108C5000110EDB6A100EF36E110E4AEC4AF02CE294
:108C60005FEC4BF0EF50006E016A013404E20050FB
:108C70008008000E01541DE35FEC4BF0EFCF04F0D1
:108C8000200E045C16E35FEC4BF0EF50E66E180E1E
:108C90000201016AD825006ED9510122110EDB5064
:108CA000E8240024E96E000E0120EA6EE552E75048
:108CB000EF6E110EDB2ACED7120EE15C02E2E16A02
:108CC000E552E16E64D35DDB130EE12402E3E1685B
:108CD000E652E16E110EDB6A120EDB6A110EF36EC4
:108CE000120ED8DB08E206EC4BF0120EF0EC4BF063
:108CF000120EDB2AF3D7100E98DB6CD8D7EC4BF0B2
:108D0000E76E110EE7CFDBFFE668FB0EE66EE66A64
:108D100081EC4BF091EC67F0006E080EE15C02E232
:108D2000E16AE552E16E00506EDB47EC64F0006EE4
:108D3000080EE15C02E2E16AE552E16E005097EC58
:108D400040F0130EE15C02E2E16AE552E16E1FD3EE
:108D500018DB120EE12402E3E168E652E16E110E27
:108D6000DB6AF36EDBCFF4FFE850F45C03E237EC30
:108D70004BF0F7D764EC4BF002E2E16AE552E16EAA
:108D80000050DF50006E016AD890015004E6800E5A
:108D9000005C000E015803E2200EDF5C06E2040EC8
:108DA000006EBD0E14EC4BF00CD023EC4BF04D0ECE
:108DB000006EBB0E1BEC4BF002E2E16AE552E16E85
:108DC000035097EC40F0120EE15C02E2E16AE552DA
:108DD000E16EDDD228EC4BF0DF6A4CDBEF6A88EC09
:108DE0004BF002E1B4890CD0D8DA2C080BE0C5ECCA
:108DF0004BF002E2E16AE552E16E03500701B48BE9
:108E0000000E28D0E6DA04E1010E011801E1DE6B64
:108E10000D0EB2EC4BF009E02C0E016EBEDA015CD7
:108E200004E0FB0EDB50DF5C02E3DF5013D0B5DA69
:108E3000E66E20DBE552E750EF6ECBDA04E1010E7F
:108E4000011801E1DE6BDF2AFC0EDB2AFD0EE0E3F8
:108E5000DB2ADED7E5529BD294DA090EE12402E345
:108E6000E168E652E16E080EDB6A88EC4BF005E142
:108E7000FA0EDB5021E1B4891FD08FDA2C080EE006
:108E8000FA0EDB5009E1C5EC4BF002E2E16AE55273
:108E9000E16E03500701B48B020E24D19ADA04E18B
:108EA000010E011801E1DE6B0D0EB2EC4BF006E194
:108EB000FA0EDB5001E1B489030E14D12D0EB2EC91
:108EC0004BF020E1040E4DDB1DE0050E026EFD0EA1
:108ED000DB50025C17E0FD0EDB0401E1C9D0030E9C
:108EE00019DB01E1C5D0070E3CDB01E1C1D0010E69
:108EF000F36E080EF3CFDBFF6CDA04E1010E01180C
:108F000001E1DE6B040E06DB09E0050E2ADB06E05C
:108F10000A0E8BDAF0D8D7EC4BF036D0DE51ADDB51
:108F2000EFCF00F0000E00C0DFFF010EDB6A020E83
:108F3000DB6A030EDB6A050EEDDA1FE1000EDFCF00
:108F4000E6FF010EDBCFE6FFE4EC69F0E552E55207
:108F5000F3CF00F0F4CF01F0026A036A01AE02D051
:108F60000268036800C0DFFF010E01C0DBFF020ED4
:108F700002C0DBFF030E03C0DBFF07012ADA04E1B6
:108F8000010E011801E1DE6B080EDB5044E0FD0E1E
:108F9000DB5007E1FDEC4BF0800E4ADA000EEE5498
:108FA00014E3020EB7DA07E1FDEC4BF0000EEE54CD
:108FB000800E3EDA0AE3060ED4DA09E1FDEC4BF04E
:108FC000000E36DA800EEE5402E2070151D0F3D9DA
:108FD0008EDA080EDB5054E0040EDBCF38F0050EBD
:108FE000DBCF39F0060EDBCF3AF0070EDBCF3BF0DC
:108FF0003D683E683F68406880EC69F0040E34C00C
:10900000DBFF050E35C0DBFF060E36C0DBFF070EAB
:1090100037C0DBFF35D0FD0EDB5006E1EEDB7F0E07
:10902000EE54000E05DA23E3FD0EDB0404E12BDB36
:10903000000EFED91CE3020E6DDA04E124DB7F0E84
:10904000F7D915E3030E8DDA04E11DDBFF0EF0D92D
:109050000EE3060E026EFD0EDB50025C0CE113DB2C
:10906000FF0EEE54FF0EEE547F0EEE5404E20701A5
:10907000B48D010E37D0070E4DDA02E09CD937DAF5
:10908000FD0EDB50070A21E0010A17E0050A11E096
:10909000010A0FE0030A08E0050A06E0010A04E0FD
:1090A000050A02E0040E1ED002DA040EDBCFEFFF49
:1090B00018D034DBDBCFEDFF14D030DBDBCFEEFF9D
:1090C000060EDBCFEEFF070E0AD0F1D9DFCFEEFFA1
:1090D000010EDBCFEEFF020EDBCFEEFF030EDBCF88
:1090E000EEFF000E006E090EE15C02E2E16AE5525D
:1090F000E16E00504CD1ACDAE652BCD9EE6AEE6AB1
:10910000EE6AEE6A010EDB6AFB0EDB50F36E010EB7
:10911000C1D94FE20701DE51B0DAEFCFDFFF300EE9
:10912000DF5C42E3DF5039083FE3A4D9EECF00F023
:10913000EECF01F0EECF02F0EFCF03F00A0E3D6E5E
:109140003E6A3F6A406A00C038F001C039F002C090
:109150003AF003C03BF080EC69F034C000F035C059
:1091600001F036C002F037C003F0300EDF5C046E51
:10917000056A066A076AE850002605500122065073
:1091800002220750032276D900C0EEFF01C0EEFF95
:1091900002C0EEFF03C0EEFF07011BD907E1010E7D
:1091A000011804E1DE6B02D0000E04D0010EDB2AB0
:1091B000ABD7010EE552E552EAD00701AE51E66E9B
:1091C000E66A1A0E006EBB0E36DA02E2E16AE5527A
:1091D000E16E035012000401785108E0010E006EA8
:1091E0006550020B01E0010E005C17E1D7D90BE1DD
:1091F0006151621111E18C86A00E616F0F0E626FDA
:10920000010E636F12006151621152E18C96A00E43
:10921000616F0F0E626F636B1200780509E0020E3A
:10922000785D06E0040E785D03E0100E785D17E1CE
:10923000B5D90BE16151621111E18C86200E616F8D
:109240004E0E626F010E636F12006151621130E1C8
:109250008C96200E616F4E0E626F636B1200200EB3
:10926000785D26E19BD907E16151621121E18C868D
:10927000D2D9010E15D0630507E16151621118E1E1
:109280008C96C9D9020E0CD0020E635D0BE16151C0
:1092900062110EE18C86A00E616F860E626F030E66
:1092A000636F12006151621103E18C96B4D9636B54
:1092B000120067D8A4D9E8AE02D0003403D0E7503A
:1092C000D880005423E3FC0EDB5010E0E8D8E9BE60
:1092D000EA68A2D804E0E846FE0B0106FCE1006E55
:1092E000DED8E9BEEA6867DAEF1210D0D8D8E9BE56
:1092F000EA6892D804E0E846FE0B0106FCE1E81CAF
:10930000006ECDD8E9BEEA6856DAEF1640D039D8FB
:1093100076D9E8AE02D0003403D0E750D8800054AC
:1093200023E3FC0EDB5011E1BAD8E9BEEA6874D839
:1093300004E0E846FE0B0106FCE1E81C006EAFD835
:10934000E9BEEA683EDAEF160FD0A9D8E9BEEA68AE
:1093500063D804E0E846FE0B0106FCE1006E9FD8EE
:10936000E9BEEA682EDAEF1212D0016E026A00C07E
:10937000E6FFE66E02C0E6FFA9EF68F0E66E7CEF5E
:109380004BF061D9E1CFD9FFE2CFDAFF1200E5520D
:10939000E5CFDAFFE7CFD9FF1200DE516ED9EF50EB
:1093A0001200A951E96EEA6A47EF4BF0E66E000E33
:1093B000DA20E66E1200D9CFE9FFDACFEAFF120019
:1093C000E652E652FAEF4BF0DECFE9FFDDCFEAFFDF
:1093D0001200DE2BDE51006E016A000E0018120032
:1093E000D890F336E8061200010EF36EDB5012003F
:1093F000E96E000EDA20EA6E1200EA22EECF48F0A3
:10940000EFCF49F012001FD9100EE66E81EF4BF03E
:10941000006EDF50005C1200C80EE926060EEA223C
:10942000EF50016E010E01521200E66E23EF4BF079
:10943000EE54000EEE54000EEE541200DF6EDFCF3D
:10944000E6FFDC51016A000F006E020E012285D991
:109450007DEC61F0D7EF4BF0DECF00F0DDCF01F017
:10946000D89001501200E76E010EE7CFDBFF070135
:10947000B4511200FC0EDBCFE9FFFD0EDBCFEAFF9B
:109480001200EA22EECF4AF0EFCF4BF01200FFD8E5
:10949000E8061200DBCFF4FFF350F45C1200FD0E7F
:1094A000DBCFE9FFEA6A1200DD513DEF4BF0FB0E26
:1094B000DBCFE9FFFC0EDBCFEAFF1200EA22EE5021
:1094C000EFCFEAFFE96E00501200A951EA6A310FAE
:1094D000E96E0E0EEA22EF500E01EA6AAC25E96E43
:1094E000AD51EA221200036E050EE15C1200040E7B
:1094F000EECFDBFF050EEECFDBFF060EEECFDBFF80
:10950000070EEECFDBFF1200C2D8000EE926010ED7
:10951000EA221200006EFD0EDB50005C1200E652E3
:10952000E652E652020EDB6A1200EA6A290FE96E81
:10953000010EEA221200DBCFE6FFE66A1200036E9C
:10954000046A02C0E6FFE66E04C0E6FFA9EC68F01C
:10955000056E1200020EDBCF48F0030EDBCF49F0A0
:109560001200016EFD0EDB50015C1200DECF00F038
:10957000DDCF01F0000E005C100E01581200EECF9E
:10958000E6FFEECFE6FFEECFE6FFEFCFE6FF1200FD
:10959000070EB715486E010E48521200060161070A
:1095A000000E625B63511200000EE926030EEA22F0
:1095B0001200010EDBCFE9FFEA6A120068D8410E03
:1095C000E926010EEA221200040EDB28E96EEA6A9F
:1095D00047EF4BF0E66EE66AE4EC69F0E552E552DF
:1095E0001200FD0EDB50F80F006E010E005212004B
:1095F000020EDBCFEEFF030EDBCFEDFF1200FD0E00
:10960000DBCF00F0190EE76E00181200D9CF00F082
:10961000DACF01F01200100E616F270E626F120098
:10962000ADDEE66AD9501200A0DED7EF4BF0BEDE09
:10963000010EC1EF4BF099DE73EF4AF0B2DE010E7E
:10964000E9260E0E1200D9CFE6FFDACFE6FF1200B0
:1096500098DEE6521200010EE8DE90DE33EF4AF0AB
:10966000A6D895D69EDE790EE9260E0E1200CEDF24
:10967000110EB6D8110EDB2A1200EA6A000FE96E4D
:10968000030EEA221200B9D8FF0EEE541200D89051
:10969000E936EA361200110EE926060EAEDE94DE39
:1096A000010E1200A3D8C1EF4BF07BDE490EE92674
:1096B0000E0E12005ADE036E070EE15C1200110E50
:1096C000DB50D924F8EF49F09EDEF5EC68F0006E2F
:1096D000080EE15C1200D5DE48504A5C49504B58F8
:1096E0001200030E28DF020E9BEF4AF0D950010F43
:1096F0007FDEEE50ED1012002CEC47F058D8E5520A
:109700001200E66AE66AF80EE66EE66AE66A12009B
:109710000D0E006E070141DE005C1200C8DE040E73
:10972000DBCFEEFF050E1200ACDE4A5048181200E7
:10973000110EE926060EEA2212003DDEEE50ED1073
:10974000120039DE010EEE18120035DE020EEE18A0
:10975000120031DE030EEE18120000C0E6FF01C059
:10976000E6FF1200006E19DE005C120029DE050E15
:1097700057DF010F00EF4CF023DE010E51DF010F28
:109780001200FCDD0701B451120007DEE66EE66A46
:10979000260E006EBB0E1BEF4BF064DF2EDE4EDF9D
:1097A000EA224850120054DFE652E6521200E55217
:1097B000E552E55212006BDF960EE926060E5EEFCB
:1097C0004AF065DF640EE926060E5EEF4AF06DDFB3
:1097D00014DE1EEF4BF0030E23DF020F17EF4BF0EA
:1097E000DB500F01D92404DEEF6A1200020FDEDD28
:1097F000030E1200E66A23EF4BF0DDDDD880120085
:10980000D5DD010E10EF4BF023DFB0DF020F17EFB5
:029810004BF01B
:0E981200BBEC51F0A098636A626A0F01266BEE
:1098200083EC52F002E2E16AE552E16E00500F0172
:1098300047EC52F0DF6ADF50006E016A0C0E005CEC
:10984000000E015810E2DF50040DF3CFE9FFF4CF12
:10985000EAFF000EE926040EEA22EE6AEE6AEE6ADC
:10986000EE6ADF2AE8D7658C0F01386B6598659C36
:1098700062A607D0629604018F6B946B956B966B12
:10988000F7D70401010EA86FA96FAA6BAB6B9C6B95
:10989000DF6A030EDF5C11E2EA6ADF34B0EC52F0FB
:1098A000EA22EE6AED6AEA6ADF34B7EC52F0EA22A5
:1098B000EE6AED6AF9EC51F0ECD70401080E856F01
:1098C000040E866F0F01160E266F0401300E026F14
:1098D000040E036F400E016F840E006F0401796B5C
:1098E000786BBEEF51F0BBEC51F082BE06D0656ADA
:1098F0000F01366B0401786B7CD0040178510CE1C8
:10990000656A0F01366B47EC52F065B602D065868A
:10991000FCD70401010E786F78050AE165BA08D01A
:10992000626A0F01366B368136890401020E786F48
:109930006250040B06E00F013651040B02E0629402
:1099400059DB65B256D06250010B09E00F01365168
:10995000010B05E05EDF0401040E786F6290625037
:10996000100B06E00F013651100B02E033DB62985A
:1099700062AC15D00F0136AD0AD04EEC52F0730E2A
:10998000C5EC51F002E2E16AE552E16E0050629CE2
:109990000401A65101E0A607A65101E1F3D86250E7
:1099A000200B05E00F013651200B01E002DB625075
:1099B000020B14E00F013651020B10E04EEC52F096
:1099C000E6687F0EE66E87EC65F0006E060EE15CE1
:1099D00002E2E16AE552E16E0050636A040E04019E
:1099E000E76E7819E8AE02D0E73402D0E750785D30
:1099F00002E2A19834D00F0136A730D0DF6A040EFE
:109A0000DF5C2CE262A62AD064CF9DF404019D5154
:109A1000780BE842E842E8429E6F62969DB504D01A
:109A20009E51BEEC52F003D09E51C3EC52F0EA229C
:109A3000EF709E5102E1F0DA0FD0000EE66EE66A9A
:109A40009D0EE66E040EE66E720EC5EC51F002E25B
:109A5000E16AE552E16E0050DF2AD1D7A198BEEF4E
:109A600051F0ADEC52F0FC0EDBA403D0E66A37EC0B
:109A700052F0FC0EDBA204D0010EE66E37EC52F081
:109A8000FD0EDB50016A260F006E0F0E31EC52F016
:109A9000CDEC51F0FC0EDBCFEFFFE552BEEF51F005
:109AA000ADEC52F0FC0EDB5003E0C0EC51F002D004
:109AB000EAEC51F01DEC52F0D9CFE9FFDACFEAFF22
:109AC000EE50ED1003E1F36AF46A28D0CDEC51F0CA
:109AD000D2EC52F0FA0EDBCFEEFFFB0EDBCFEDFF48
:109AE000CDEC51F0EE52F90EDBCFEFFF400EC8EC9B
:109AF00052F0880ED7EC52F0FC0EDB5003E0C0ECC5
:109B000051F002D0EAEC51F0EA22EF74DECF00F01F
:109B1000DDCF01F000C0F3FF01C0F4FFE552BEEF5E
:109B200051F0ADEC52F0FD0EDB5003E18CEC52F045
:109B300009D0EFEC51F061EC52F0EFEC51F0010F75
:109B400061EC52F0E552BEEF51F093EC52F065A893
:109B500017D0A6EC52F0400EEE16EE6AEE6AEE6AF0
:109B6000A6EC52F0EE7CC0EC51F0EA22EF74400E0D
:109B7000006EA6EC52F00050EF16A6EC52F0EF7C0F
:109B80007DEF52F00401A85127E1010EA86FA95101
:109B900023E1010EA96F020E8C5D09E1D2EC51F0B8
:109BA000EE52EF6AD2EC51F0C80EEF6E12008C0547
:109BB00013E19F6BDFEC51F0EE52400EEF6EDFECE5
:109BC00051F06DEC52F0DFEC51F0840EEF6E010EAF
:109BD0009F6FCDDB800EEF6E12000401AA6BAB6BA2
:109BE000020E8C5D07E1CCEC52F0E4EC51F05CEC41
:109BF00052F010D090510401365D040191510401DE
:109C0000375904E236C490F437C491F45CD8CADB07
:109C1000DBDBC8DBC80EEF6E1200ADEC52F0000EBD
:109C2000DE6E040EDD6EDBDB040DF4CF01F0D9CF68
:109C3000E9FFDACFEAFFF350EE260150ED22ADDB6B
:109C4000EF9EFC0EDB5002E1C5DB01D099DBEA227E
:109C5000DECFEEFFDDCFEDFFA0DBEF9C9EDB040E41
:109C6000E926000EEA22EF8CE55288D365980401BC
:109C70008FBF0DD094AF09D0020E8C6FAB5101E1B4
:109C8000ACDF0401A96BA86B12008CEF52F0040149
:109C900030AF0DD00401010E8C6FAA5101E19DDFA0
:109CA0000401A96BA86BA7510DE1C2EF4DF00401AF
:109CB000020E8C6F5CDB840EEF6EA96BA86BA75154
:109CC00001E160DF120057DB400EDF6E0401905DA2
:109CD000000E91590AE290C4DFFF8B5102E1010EA0
:109CE00003D08B0502E1020E8B6FDF50016AE85052
:109CF000905D906F01509159916F54DBEE52DFCF20
:109D0000EFFF380E996F040E9A6F8FB10DD0DF50B0
:109D100017E08DC4F6FF8EC4F7FF8D2B000E8E2347
:109D20000800F5507DDBF3D7DF500AE08DC4E9FF72
:109D30008EC4EAFF8D2B000E8E23EF5071DBF4D71B
:109D40001DD3ADEC52F03BDBEE52EFCFDFFFDFCFA8
:109D500000F000500401955D000E965902E295C492
:109D6000DFFFDF50006E016AE850955D956F01508E
:109D70009659966F010EDB6ADF50F36E010EDBCF52
:109D8000F4FFF350F45C16E2010EDB50EA6A380F80
:109D9000E96E040EEA22EF50E66E92C4E9FF93C426
:109DA000EAFF922B000E9323E552E750EF6E010E6F
:109DB000DB2AE2D7000ED8809555000E96550DE2AD
:109DC000EBDB02DBFCDAEF50400B03E175DBC80E86
:109DD00002D072DB880EEF6E12D0C9DA840EEF6EFD
:109DE0009751981107E005D098C4FAFF04019751E4
:109DF000F96EFADF0401949FA75101E1C3DEE55239
:109E0000BDD2B9DA04018F8F7EDB02E2E16AE5524E
:109E1000E16E0050300EE66EE66AE66A000EE66E0F
:109E2000040EF1DA02E2E16AE552E16E0050658C5F
:109E3000DF6A030EDF5C02E2DCDAFBD7010EE66EBE
:109E4000E66AE66A7A0EE66E040EDDDA02E2E16A9E
:109E5000E552E16E0050659C0401080E856F040E0A
:109E6000866F000E7B6F040E7C6F7BC47DF47E6F6B
:109E700032C479F4795102E1100E10D0010EE66E71
:109E8000E66A790EE66E040EE66E010E7EDA02E2F6
:109E9000E16AE552E16E00500401200E786F6ED247
:109EA000800E0401305D4EE10401C00E8F6F04018D
:109EB0003351030A25E0010A09E0030A41E10401E4
:109EC000700E8D6FD30E8E6F120E34D03251F66E2F
:109ED000F76AD890F636F736C50EF626D30EF72277
:109EE0000900F5CF8DF40A00F5CF8EF4020E0401BF
:109EF000DCDAF5CF90F4030ED8DAF5CF91F4120046
:109F0000030E325D1AE204018F8104013251E96EC1
:109F1000EA6AD890E936EA36D40EE926020EEA2239
:109F2000EECF8DF4EDCF8EF48DC4E9FF8EC4EAFF41
:109F3000EF500401906F916B120004018F6B1200BF
:109F400004018F6B120009DB0401386B396B30514F
:109F50001F0B020A11E0030A0CE0010A1EE10401D2
:109F60008F8F0401388104019B0517E104013883B8
:109F700014D004018F8F11D004018F8F040134BFDE
:109F800002D0DADA01D0DDDA58DAE3DA06E005DA0F
:109F9000EF50040B02E0010E386F04018FAF07D0C1
:109FA000380E8D6F040E8E6F8F81020E906FE5520A
:109FB000E5D10F0126A10CD002DAEF50800807E1AD
:109FC000F1D9EF50840803E1FAD98C0EEF6E269197
:109FD000629A12000F013685629865820401010EB3
:109FE0009C6F31DA750ED1D902E2E16AE552E16E79
:109FF0000050120004019C6B26DA740EC6D902E2EE
:10A00000E16AE552E16E005065920F01369562A457
:10A0100002D06294FCD71200AED904012D0EA66FB7
:10A02000FD0E9D1539E17E0E9D15E8407F0B040D58
:10A03000F3CF7BF4F4CF7CF4000E7B27040E7C235B
:10A040007BC47DF47CC47EF47D75B9D9EF503C0BA4
:10A05000E842E8420D081EE1DF6A080EDF5C16E206
:10A06000AED9020EE926000ED5D9EF50E66EDF50CC
:10A07000EA6A300FE96E040EEA22E552E750EF6E0D
:10A080009ED990DAEE2AEF22DF2AE7D798D925DA8F
:10A0900009D807D027D805D0FD0E9D15040801E189
:10A0A00030D86CD104018B6BA76BAA6BAB6B9F6B29
:10A0B0008C6B78D9EF9E857575D9EF9E8575FCD927
:10A0C000EF9E8F6B906B916B946B956B966B55D8E5
:10A0D000BAD9030E5AD902E2E16AE552E16E0050A4
:10A0E00036EF4EF0020E04018C5D02E1A1EF4EF05E
:10A0F0008C6B9F5104E13BD98C0EEF6E12009F6B6D
:10A10000120039D94FD9EF50400B01E0010EDF6E3C
:10A1100004018575080E785D0BE132C438FF0F012C
:10A12000385103E00401100E02D00401040E786FD0
:10A130008C0513E137D948D9C6DD020E04018B5DC9
:10A1400003E130D9840E07D0DF5003E12BD9C80ECC
:10A1500002D028D9880EEF6E0FD094AF0CD0975153
:10A16000981107E005D098C4FAFF04019751F96EE1
:10A17000FADF0401949F8C6B01D104013051600B14
:10A18000E842E842E842E842E842000901E0120001
:10A1900031510C0A4AE00B0A3FE00C0A31E0010A97
:10A1A00022E00B0A1EE0020A1CE0030A18E0080A7B
:10A1B00010E0010A0CE00F0A08E0030A01E01200B7
:10A1C00004018F8F080E786F120050EF4FF001EFEF
:10A1D0004FF00401790E8D6F040E8E6F0CD0A3EF3B
:10A1E0004FF016EF51F0345104018D6F8E6B7A0EE3
:10A1F0008D27040E8E238F81010E906F8F8F12009A
:10A2000004018F8F04013451EA6A7A0FE96E040E5B
:10A21000EA2232C4EFFF120016D9020EB6D802E2CB
:10A22000E16AE552E16E00501200120096D9E65242
:10A23000E652E6520401320510E130511F0B0009CD
:10A240000CE104018F8F030E0401315D04E1040170
:10A25000010E9B6F02D004019B6B0401325101E09F
:10A260007FD030511F0B020801E07AD034510F0B20
:10A27000000901E175D034510F0B020871E3200E83
:10A280000401785D6DE18F8F040134BF04D054D98F
:10A29000D4D8DFD803D055D9D0D8DFD8EA22020EDF
:10A2A000EFCFDBFFECD8010B02E1DF9401D0DF84BC
:10A2B00034BF02D041D901D044D9EA22DECFEEFF2B
:10A2C000DDCFEDFF030E315D0CE143D907E034BF74
:10A2D00002D0BFD801D0C1D8EA22EF82840E67D95C
:10A2E0003FD0DF7436D90BE058D8EF9E56D8EF8CAC
:10A2F000FAD802E2E16AE552E16E005002D04DD890
:10A30000EF8CDF74BCD8020B02E123D912E0040108
:10A3100034BF02D09ED801D0A0D8EA22EF923B0EE3
:10A32000006E36D9E0D802E2E16AE552E16E0050F3
:10A3300002D03B0E2DD9040134510F0B016A260FB8
:10A34000006E0F0E0122030E00C0DBFF040E01C0E1
:10A35000DBFF030EDBCFE9FF040EDBCFEAFFEF905C
:10A36000050EE15C02E2E16AE552E16EC6D014D965
:10A37000B4D85CEF52F0D7D8E6521200E552BDD007
:10A38000FD0EEA6ADB34B0EF52F0E66EE66A87EC67
:10A3900065F0006E060EE15C1200DECFE9FFDDCF56
:10A3A000EAFF120085C4E9FF86C4EAFF12003451B7
:10A3B0000F0BE96EEA6AD890E936EA3612007BC4E0
:10A3C000E9FF7CC4EAFF1200EDD8380EEE6E040EF1
:10A3D000ED6E1200FD0EEA6ADB34B7EF52F0FC0EB0
:10A3E000DB50E824026EFD0EDB50040DF350022416
:10A3F0001200DF50C8D8EA22EF6ADF50BFD8EA2245
:10A40000EF6ADF2A1200E66E5CEC68F0006E050E63
:10A41000E15C1200EA22EE50EFCFEAFFE96E120093
:10A42000E66E99C4E9FF9AC4EAFF992B000E9A23BD
:10A43000E552E750EF6EDF061200EA22EECFDEFFB4
:10A44000EDCFDDFF1200000EE66EE66AE66EE66A0C
:10A45000120034510F0BBEEF52F034510F0BC3EF0B
:10A4600052F0012200C0DEFF01C0DDFF1200FD0E30
:10A47000DBCFE6FF0DEC4EF0E552E5521200D9506D
:10A48000020FE96E000EDA20EA6EEF501200160E8F
:10A49000396F9F0E376F7B0E366F1200010EE66E1E
:10A4A000E66A000EE66EE66A1200F76A8D25F66E21
:10A4B0008E51F722080012007DC4E9FF7EC4EAFF36
:10A4C0001200040DF3CF00F0F4CF01F0000E0026CF
:10A4D000040EC7DF840ED7EF52F064D8300EEE6E54
:10A4E000040EED6E1200020EE66EE66ADECFE6FFA7
:10A4F000DDCFE6FF050EC5EF51F0E552E5CFDAFFFF
:10A50000E7CFD9FF1200020EE66EE66AE66A270E72
:10A51000E66E0F0E03EF52F02ADF8C0EEF6E42DF75
:10A52000840EEF6E1200D9CFE6FFDACFE6FFE1CF5F
:10A53000D9FFE2CFDAFF12003ADF7F0EE926040EE0
:10A54000120035DF850EE926040E120019DF0AEF2E
:10A5500052F023DFEF50800B12000DDFE6521200A5
:10A56000FE0BEA36E96E850EE926040E1200FE0B9C
:10A57000EA36E96E7F0EE926040E1200EA6AA30F9E
:10A58000E96E040E1200EA6AA00FE96E040E1200D2
:10A5900004DFE850EF1612008FDFEE52400EEF6E30
:10A5A0005CEF52F0020EE926000EEA221200F5DE00
:06A5B000E850EF1212005A
:0AA5B60017EC58F0FB0EDBCFF3FFAB
:10A5C000DB06F35000090AE065EC58F0FA0ED0EC17
:10A5D00058F0F3E1011CF1E1010E01D0000E46EF4D
:10A5E00058F017EC58F03B0EE12402E3E168E65224
:10A5F000E16E010EDB6A020EDB6AF90EDBCFF6FFBD
:10A60000FA0EDBCFF7FFFB0EDBCFF8FF0800F550AB
:10A61000DF6EDF5002E16AEF57F0250EDF5C02E0EB
:10A620005DEF57F0030EDB6A040EDB6A050EDB6A92
:10A63000060EDB6A070EDB6A7FEC57F02D0EDF5C3F
:10A640000CE02B0EDF5C09E0200EDF5C06E0230E41
:10A65000DF5C03E0300EDF5C1AE1DF50300A14E00B
:10A66000130A0FE0030A0AE00B0A05E0060AE4E118
:10A67000030EDB80E1D7030EDB82DED7030EDB8423
:10A68000DBD7030EDB86D8D7030EDB88D5D72A0E9F
:10A69000DF5C1BE17BEC57F0C9EC57F010E0030ED8
:10A6A000DB803A683B68130EDBCF3FF0140EDBCF44
:10A6B00040F0B4EC5BF0040E38C0DBFF03D0130EA7
:10A6C000B2EC57F07FEC57F00BD0090EDB6A20ECB0
:10A6D00058F003E094EC58F0FAD7090EB2EC57F0BA
:10A6E000030EDBB0DB982E0EDF5C1BE17FEC57F036
:10A6F0002A0EDF5C0BE17BEC57F0C9EC57F003E16D
:10A70000130E04EC58F07FEC57F00BD0090EDB6A07
:10A7100020EC58F003E094EC58F0FAD7090E04EC62
:10A7200058F0680EDF5C07E17FEC57F0680EDF5CE5
:10A730001DE1030E18D0740EDF5C17E07A0EDF5CAB
:10A7400014E0480EDF5C06E0540EDF5C03E05A0EB6
:10A75000DF5C02E1020E07D06C0EDF5C03E06A0EE4
:10A76000DF5C04E1010E57EC58F0C9DBDF506E0AE4
:10A7700001E17FD31E0A01E192D1200A01E18FD1CC
:10A780003F0A01E149D11A0A01E146D10D0A01E16E
:10A7900043D1200A01E140D13A0A01E13DD1200A2A
:10A7A00001E13AD1260A01E135D10D0A01E132D1A8
:10A7B0001A0A01E1D9D0200A4AE0300A1FE0460A0D
:10A7C0000EE0250A01E083D3D950F90FE96EFF0EA0
:10A7D000DA20EA6E010EEE5E000EEE5AEE5A65ECDD
:10A7E00058F0250EE66E95DB03E1011C01E169D30B
:10A7F00061EC58F001E26BD3DB2A69D3080EDB6A07
:10A80000040EDB50010806E2040EDB0429EC58F0CC
:10A81000DB508BDB080EDB5009E0030EDB50010B35
:10A8200005E172DB01E04DD3080EDB6A64DBEFCF9C
:10A83000DFFFD9EC58F003E1011C01E142D361ECE8
:10A8400058F001E3DB2A60DB01E141D33AD3070E84
:10A85000DB5002080FE1A5EC58F0030E6CEC58F049
:10A860000E0EEECFDBFF0F0EEECFDBFF100EEECFA6
:10A87000DBFF20D0F70EDBCF03F0F80EDBCF04F0C8
:10A88000020E035E000E045AF70E03C0DBFFF80E43
:10A8900004C0DBFF03C0E9FF04C0EAFF5CEC58F032
:10A8A000026A0E0E00C0DBFF0F0E01C0DBFF100EB0
:10A8B00002C0DBFF0E0EDBCFE6FF0F0EDBCFE6FFA5
:10A8C000100EDBCFE6FF84EC68F0E552E552E5526E
:10A8D000130E39C0DBFF140E3AC0DBFF060EDB504F
:10A8E00005E0130EA0EC58F001E26ADBC4EC58F06E
:10A8F00002E2130E37DB87EC58F006E0040EA0EC02
:10A9000058F002E2050E2EDB030EDBB005D0FCDAB8
:10A9100001E0D7D2080EDB6A090EDB6A0E0EDBCF30
:10A92000F6FF0F0EDBCFF7FF100EDBCFF8FF0800AE
:10A93000F550DF6EDF5014E0CAEC58F011E2D9ECAC
:10A9400058F003E1011C01E1BCD2BBDB01E3DB2ACF
:10A95000090EDB2AD9500E0FE96E000ECBDBE7D7CC
:10A96000D3DA01E1B4D2ADD2C6DA110EEECFDBFFFD
:10A97000120EEDCFDBFF110EDBCFE6FF120EDBCFA9
:10A98000E6FF76EC68F0E552E552130EF3CFDBFFFD
:10A99000140EF4CFDBFF060EDB5004E0130ED0DB09
:10A9A00001E20EDBC4EC58F002E2130EDBDAAFDB9F
:10A9B00005E0040EC5DB02E2050ED4DA030EDBB0BF
:10A9C00005D0A2DA01E07DD2080EDB6A090EDB6A4F
:10A9D000110EDBCFE9FF120EDBCFEAFFEFCFDFFF77
:10A9E000DF5014E0D7DB12E2E4DB03E1011C01E1FC
:10A9F00068D267DB01E3DB2A090EDB2A110EDB2AB2
:10AA0000DBCFE9FF120EE8E3DB2AE6D77DDA01E1CE
:10AA10005ED257D2030EDB8E070EDB0410E195DB0E
:10AA2000040E5ADB0A0EEECFDBFF0B0EEECFDBFF80
:10AA30000C0EEECFDBFF0D0EEECFDBFF6CD0070E62
:10AA4000DB5003082CE1030EDBAE0DD0B2DA020EB0
:10AA500076DAEFCF00F0016A026A036A00AE39D0FD
:10AA60000168026835D0F70EDBCF01F0F80EDBCFBE
:10AA700002F0020E015E000E025AF70E01C0DBFF6B
:10AA8000F80E02C0DBFF01C0E9FF02C0EAFFEFCF12
:10AA900000F00A0E00C0DBFF0B0EDB6A38D0070E99
:10AAA000DB50020809E1030EDBAE04D059DB02AE35
:10AAB00010D00ED055DB0DD0030EDBAE12D079DAFC
:10AAC000020E3DDAF9DA026A036A01AE02D00268C8
:10AAD0000368E2DA0C0E02C0DBFF0D0E03C0DBFFE1
:10AAE0001AD0F70EDBCF02F0F80EDBCF03F0020E28
:10AAF000025E000E035AF70E02C0DBFFF80E03C021
:10AB0000DBFF02C0E9FF03C0EAFFD6DAC5DA0C0EAC
:10AB1000DB6A0D0EDB6A060EDB5005E1010EF36EFB
:10AB2000050EF3CFDBFF150EDB6A160EDB6AD9507C
:10AB3000370F006E000EDA20016E390E00C0DBFF09
:10AB40003A0E01C0DBFF380EDB6A080EDB6A0A0E24
:10AB5000AEDADF50780A12E0200A10E0280A0CE092
:10AB6000200A0AE03F0A06E00D0A02E0200A08E196
:10AB7000020E05D0080E03D0080EDF26100E97DA5D
:10AB8000030EDBBE02D0DB92DB94DB50800B24E0B3
:10AB90008ADAD890030EEB50000A08E6000EEE5C4D
:10ABA000000EEE58000EEE58000EEE5815E213DAC5
:10ABB0003D683E683F68406880EC69F00A0E34C02A
:10ABC000DBFF0B0E35C0DBFF0C0E36C0DBFF0D0EBE
:10ABD00037C0DBFF2D0E08D0030EDBA202D02B0EF8
:10ABE00003D0DBA408D0200EF36E170EF3CFDBFFEB
:10ABF000150EDB2A02D0170EDB6A050EDB5003E1CF
:10AC0000B7D901E189D02C0E006ED50E016E000E71
:10AC1000026E070EDBCF03F0046A056A066A03C002
:10AC20003DF004C03EF005C03FF006C040F0D3D96F
:10AC30000AEC6AF000503424F36E01503520F46EB3
:10AC400002503620F86EF4CFF7FFF3CFF6FF08007E
:10AC5000090EF5CFDBFF580EDF5C0FE1610EF36EDE
:10AC6000090E7BD90AE3200E006E090EDBCFE7FF49
:10AC70000050E75E090EE7CFDBFF070EDBCF00F0E9
:10AC8000016A026A036A0FDA00C03DF001C03EF0BB
:10AC900002C03FF003C040F0EECF38F0EECF39F005
:10ACA000EECF3AF0EFCF3BF00AEC6AF03BC0EDFF9D
:10ACB0003AC0EDFF39C0EDFF38C0EFFF390EDBCFF2
:10ACC000E9FFDB063A0EDBCFEAFF01E2DB06090E05
:10ACD000DBCFEFFF150EDB2A4BD995E1030EDBA688
:10ACE0001DD06F0EDF5C06E1C1D918E3150EDB281D
:10ACF0005BDA14D0780EDF5C09E0580EDF5C06E00A
:10AD0000620EDF5C03E0420EDF5C08E1020EF36ED0
:10AD1000160EF3CFDBFF02D0150EDB6A030EDB50FD
:10AD2000100B0EE0040EDBCF00F0050EDB50D880D8
:10AD3000005406E2060EDB5003E1040EDB5034DA69
:10AD400095D90AE2050EDBCFE7FF150EDB50E75E73
:10AD5000050EE7CFDBFF02D0050EDB6A040EDBCF6A
:10AD600000F0160E45D9D880005414E2160EDBCF41
:10AD7000E6FF150EDBCFE6FF040EDBCFE6FF050E88
:10AD8000DB50E552E75CE552D880E754E552D880C5
:10AD9000E7545FD9030EDB50010B0BE1080EDB50CB
:10ADA00008E0B2D801E08DD0080EDB50BED8080E06
:10ADB000DB6A170EDB5007E088D9170EF1D903E1E3
:10ADC000011C01E17ED0160EDB5016E07ED9300E5C
:10ADD000E66E9FD802E1011C74E077D9DFCFE6FF71
:10ADE0003EEC69F0E552E552E552F4CF01F0000186
:10ADF000F31C02E1011C65E0050EDBCF00F0160E2E
:10AE0000DB50D880005409E2050EDBCFE7FF160EB9
:10AE1000DB50E75E050EE7CFDBFF300EE66E050E7A
:10AE2000CBD94FE1390EDB2ADBCFE9FF3A0E01E344
:10AE3000DB2ADBCFEAFF090EEFCFDBFFDB500EE0B2
:10AE400044D9090EADD902E1011C3BE0390EDB2AE1
:10AE5000DBCFE9FF3A0EEDE3DB2AEBD755D831E142
:10AE6000160EDBCFE6FF080EC3D8E552E7245DD807
:10AE70002ED0070EDB50030A1CE0010A14E0030A7F
:10AE800007E07BD9DBCFEEFF020EDBCFEDFF1FD05B
:10AE9000F5D8056A03AE02D0046805682CD8BCD882
:10AEA00005C0EEFF14D0EAD803BE046824D8B4D895
:10AEB0000ED063D9DBCFEFFF0AD07BD905E1011CAF
:10AEC00003E1F368F46810D0FCD801E3DB2A79D9F8
:10AED00006EF53F0010EDBCF00F0020EDBCF01F0E6
:10AEE00000C0F3FF01C0F4FF3B0EE15C02E2E16A47
:10AEF000E552E16ECBD029D9020E6CEF58F061D942
:10AF00000800F550DF6E1200200EE66E080EDCEF32
:10AF100058F03EEC69F0E552E552E552F3CF00F00F
:10AF2000F4CF01F00001F31C1200006E016AD95049
:10AF3000010F4DD90050EE260150ED221200045EA3
:10AF4000000E055AF70E04C0DBFFF80E05C0DBFF4C
:10AF500004C0E9FF05C0EAFF1200DBCFF4FFF350A5
:10AF6000F45C1200DB50E76E040EE7CFDBFF12004B
:10AF70000A0EDBCF00F00B0EDBCF01F00C0EDBCFA7
:10AF800002F00D0EDBCF03F0005001100210031091
:10AF90001200130EEECFDBFF140EEDCFDBFF130E0E
:10AFA000DBCF00F0140EDBCF01F00001800E0114A6
:10AFB0001200F70EDBCF04F0F80EDBCF05F0120025
:10AFC000050EDB50E66ED950130F01D9E552E7505C
:10AFD000EE6EED6A12000A0EDBCF38F00B0EDBCFFF
:10AFE00039F00C0EDBCF3AF00D0EDBCF3BF0120048
:10AFF000DBCFE6FF150EDBCFE6FF050EDB50E5529B
:10B00000E724E552E7241200DB50CED8010EF36EA0
:10B01000060EF3CFDBFF1200EE50EFCFEAFFE96E32
:10B0200002C0EEFF03C0EEFF04C0EEFF1200D9CF56
:10B03000E6FFDACFE6FFE1CFD9FFE2CFDAFF120079
:10B04000DFCFE6FFE66AF8EC69F0E552E552F3502F
:10B050001200E76E080EE7CFDBFF1200EECF00F024
:10B06000EECF01F0EFCF02F0036A1200050EDBCF46
:10B0700000F0150EDB50D88000541200010EDBCF1B
:10B0800002F0020EDBCF03F0046A1200E552E5CFB6
:10B09000DAFFE7CFD9FF12000A0E00C0DBFF0B0E6C
:10B0A00001C0DBFF1200D9500A0FE7EF58F0F36E32
:10B0B000070EF3CFDBFF1200EECF00F0EFCF01F071
:10B0C0001200010EDB2A020E1200FC0EDBCFE6FF9F
:10B0D000FD0EDBCFE6FF1200005E000E015AF70EF8
:10B0E00000C0DBFFF80E01C0DBFF00C0E9FF01C0BC
:10B0F000EAFF1200DA20EA6EEF2AEECFF6FF000E2A
:10B10000EF22EECFF7FFEF22EECFF8FF1200040E92
:10B11000DBCFE6FF130EDB50E552E75C9ADFDB5036
:10B1200004DF060EDB501200090EDB500A0DF3504F
:10B13000DF24D00FE76E090EE7CFDBFF7FEF57F07C
:10B14000DB50F36E050EADEF57F0F70EDBCF00F0DE
:10B15000F80EDBCF01F01200DFCFE6FF89EF57F0EA
:10B1600028DF030EECDE2EEF58F0DBEC52F0E55258
:10B17000E552E552E55200091200BDDEEE50EFCF78
:10B18000EAFFE96E010E1200130EDB50F36E040E9F
:10B19000ADEF57F0040EDB50F36E090EADEF57F034
:10B1A000DBCFE6FF89EF57F0E76E050EE7CFDBFF59
:10B1B00012008BDFACEF58F0DBCFE6FF86DFB5EF98
:10B1C00058F0D950F90FE96EFF0E7AEF58F0E96E9A
:08B1D000000EDA20EA6E120005
:08B1D800439E08D0439E3BAEEC
:10B1E00005D03A6C3B1EE86A3B22438E3BC035F0EB
:10B1F0003AC034F0476A466A8E0E366E376AC6EF3A
:10B200005AF0439E0CD0439E3BAE09D0386C391E99
:10B210003A1E3B1EE86A39223A223B22438E3BC04B
:10B2200035F03AC034F039C047F038C046F09E0ED1
:10B23000366E376AC6EF5AF0436A02EC5BF01AECDE
:10B240005BF043B6AAEF5AF043A205D043BAAAEF87
:10B250005AF0B1EF5AF043BABDEF5AF043A005D00F
:10B2600043B8AAEF5AF0BDEF5AF043B8B1EF5AF025
:10B27000376A7F0E3C24366EE86A37224150365ECC
:10B28000E86A375A1A0E446E3C6A466A476A346A5C
:10B29000356A3E50395E3F503A5A40503B5A000E94
:10B2A0003C5A09E73E5039263F503A2240503B2253
:10B2B000000E3C2201D0468AD89039363A363B36C9
:10B2C0003C36D8904636473634363536442EE1D7AC
:10B2D0003B503A103910D8A4468AC6EF5AF0436A58
:10B2E00002EC5BF01AEC5BF043B6AAEF5AF043A213
:10B2F00005D043B8AAEF5AF0B1EF5AF043AA05D0EF
:10B3000043B0AAEF5AF0B1EF5AF043B002D043A8CD
:10B3100002D0BDEF5AF0376A41503C24366EE86ADD
:10B3200037227E0E365EE86A375A466A476A346AC2
:10B33000356A40503B02F4CF35F0F3CF34F03F5044
:10B340003B02F3504726F4503422000E3522405081
:10B350003A02F3504726F4503422000E35223E5074
:10B360003B02F3504626F4504722000E3422352289
:10B370003F503A02F3504626F4504722000E342242
:10B38000352240503902F3504626F4504722000E31
:10B39000342235223E503A02F4504626000E47220F
:10B3A000342235223F503902F4504626000E4722FF
:10B3B00034223522C6EF5AF0417E436A02EC5BF03C
:10B3C0001AEC5BF043B6AAEF5AF043A20AD043AAA4
:10B3D00003D043BEAAEF5AF043A4B6EF5AF0B3EF3E
:10B3E0005AF043AA05D043ACB6EF5AF0B3EF5AF087
:10B3F00043A00AD043A808D043BE04D043A402D03F
:10B40000BFEF5AF0C3EF5AF0466A376A41503C5CCE
:10B41000456E10E339C047F03AC034F03BC035F018
:10B420003CC044F03EC039F03FC03AF040C03BF071
:10B43000433A09D03EC047F03FC034F040C035F039
:10B4400041C044F0456C439E43BC438E44C036F03B
:10B4500043B0F2EF5AF01A0E4560F2EF5AF0366A36
:10B460003C6A43A408D0396C3A1E3B1E3C1EE86A75
:10B470003A223B223C2243AC08D0476C341E351E96
:10B48000361EE86A342235223622386A455207E0F1
:10B490003C343B323A3239323832452EF9D73950C2
:10B4A00047263A5034223B5035223C50362238C091
:10B4B00046F0439E36AE0BD0466C471E341E351EFA
:10B4C000361EE86A4722342235223622438E36A0C1
:10B4D00006D0D8803532343247324632442A44C00E
:10B4E00036F0C6EF5AF0436A02EC5BF043B67DEFEC
:10B4F0005AF043A20FD043B407D07F0E3B6EFF0E2D
:10B500003A6E396E386E25D0800E3B6E01D03B6AA4
:10B51000000EF6D743B0FBD7386A9F0E3C60EBD7DE
:10B520007E0E3C64F4D79E0E3C5C07E0D8903B3224
:10B530003A32393238323C2AF6D743A40AD0386C32
:10B54000391E3A1E3B1EE86A39223A223B223BAEA4
:10B55000DED712007F0E3C6EFF0E3B6E3A6E396EE8
:10B5600012007F0E43BEFF0E3C6E02D07F0E3C6E7B
:10B57000800E3B6E3A6A396AF3D743AE04D0800E30
:10B580003C6E3B6AF7D73C6A3B6AF4D735503410BF
:10B5900047104610F8E037BEF0D735BE0CD0365015
:10B5A0003710EBE0D8904636473634363536360617
:10B5B000D8A03706F2D73750D4E13628D2E046AECD
:10B5C00011D07F0E461402E147A00CD0472AE86A4A
:10B5D0003422352207E3D880353234324732362AD6
:10B5E0003628BFE03650C9E047C039F034C03AF0E1
:10B5F00035343B6E36303C6E3B323C9E43BE3C8E17
:10B60000B0EF5AF03B363C3602E34384437E06E11A
:10B6100043803C6A3B6A3A6A396A12003C2803E07C
:10B62000D8803B321200D8903B3202E143821200B4
:10B63000438612004036413602E3438C437E06E1E6
:10B640004388416A406A3F6A3E6A1200412803E02B
:10B65000D88040321200D8904032EAE1438A12008A
:10B66000426A40AE39EF5BF03F6C401EE86A402210
:10B67000421E3BAE41EF5BF03A6C3B1EE86A3B2258
:10B68000421E49EC6AF03BBE51EF5BF042AE000C4B
:10B690003A6C3B1EE86A3B22366C371EE86A37225A
:10B6A000000C42BE48EF5BF04388FF0C5FEC5BF0A0
:10B6B00043B6000C43B0000C43A4000C010C436AD9
:10B6C00002EC5BF01AEC5BF043B6120043AE08D01C
:10B6D00043A004D043A802D043801200439012003C
:10B6E00041503C5C0BE140503B5C08E13F503A5C10
:10B6F00005E13E50395C02E143801200D8A002D03F
:10B70000438E10D03C5041C03CF0416E3B5040C095
:10B710003BF0406E3A503FC03AF03F6E39503EC069
:10B7200039F03E6E41503C5C10E0FF0F09E0439061
:10B7300043B403D043AE4384120043AE439412009B
:10B74000412AD89040323F323E323E50395E3F501F
:10B750003A5A40503B5A3BBEEAD7D89039363A362F
:10B760003B363C2EF8D7C8D73BC047F03AC046F02E
:10B770003A503F02F4CF39F0F3CF38F03B5040025B
:10B78000F4CF3BF0F3CF3AF03F02F3503926F450B8
:10B790003A22E86A3B2246504002F3503926F450E0
:10B7A0003A22E86A3B2240AEDAEF5BF046503A5E5E
:10B7B00047503B5A47AE000C3F503A5E40503B5A10
:02B7C000000C7B
:0EB7C200256C692C256C690A0D00514D2C2553
:10B7D000692C25692C25692C25690A0D0025303432
:10B7E000692C253034690D0A002531690D0A0025C0
:10B7F0003033690D0A00253031306C750D0A002593
:10B80000640A0D0025642C256C752C256C752C257F
:10B810006C752C256C750A0D004D616A6F72206D78
:10B82000616C66756E6374696F6E204178697332FE
:10B830002053746570436F756E746572207A6572FB
:10B840006F0A0D004D616A6F72206D616C66756ED6
:10B850006374696F6E204178697332205374657028
:10B86000436F756E74657220746F6F2068696768C6
:10B87000203A20256C750A0D004D616A6F72206DAB
:10B88000616C66756E6374696F6E2041786973319F
:10B890002053746570436F756E746572207A65729B
:10B8A0006F0A0D004D616A6F72206D616C66756E76
:10B8B0006374696F6E2041786973312053746570C9
:10B8C000436F756E74657220746F6F206869676866
:10B8D000203A20256C750A0D002130204572723AFD
:10B8E000203C61786973323E207374657020726108
:10B8F0007465203C20312E3331487A2E0A0D002108
:10B9000030204572723A203C61786973323E207370
:10B910007465702072617465203E2032354B20734F
:10B92000746570732F7365636F6E642E0A0D00214A
:10B9300030204572723A203C61786973313E207341
:10B940007465702072617465203C20312E3331485B
:10B950007A2E0A0D002130204572723A203C61781F
:10B960006973313E20737465702072617465203E86
:10B970002032354B2073746570732F7365636F6E5F
:10B98000642E0A0D002130204572723A203C6D6F02
:10B9900076655F6475726174696F6E3E206C61726A
:10B9A000676572207468616E2031363737373231FF
:10B9B00035206D732E0A0D002130204572723A2019
:10B9C0003C61786973323E20616363656C657261C6
:10B9D00074696F6E2076616C756520697320302EF6
:10B9E0000A0D002130204572723A203C617869735B
:10B9F000313E20616363656C65726174696F6E20AE
:10BA000076616C756520697320302E0A0D00213037
:10BA1000204572723A203C61786973323E206C6135
:10BA200072676572207468616E203136373737323D
:10BA300031352073746570732E0A0D002130204556
:10BA400072723A203C61786973313E206C61726792
:10BA50006572207468616E20313637373732313580
:10BA60002073746570732E0A0D00213020457272A8
:10BA70003A203C76656C6F636974795F66696E61C4
:10BA80006C3E206C657373207468616E20342E0ADE
:10BA90000D002130204572723A203C76656C6F6350
:10BAA0006974795F696E697469616C3E206C657355
:10BAB00073207468616E20342E0A0D0021302045F9
:10BAC00072723A203C76656C6F636974795F66695F
:10BAD0006E616C3E206C6172676572207468616E85
:10BAE0002032353030302E0A0D0021302045727260
:10BAF0003A203C76656C6F636974795F696E69742E
:10BB000069616C3E206C6172676572207468616E59
:10BB10002032353030302E0A0D0053746174757345
:10BB20003D25690D0A002135204572723A204E6587
:10BB3000656420636F6D6D61206E6578742C20667E
:10BB40006F756E643A20272563270D0A0025730D53
:10BB50000A00506172616D383D25630D0A00506125
:10BB600072616D373D25630D0A00506172616D365B
:10BB70003D256C750D0A00506172616D353D256C77
:10BB8000640D0A00506172616D343D25750D0A0027
:10BB9000506172616D333D25640D0A005061726120
:10BBA0006D323D25640D0A00506172616D313D2595
:10BBB000640D0A0050492C2531750D0A004D522C98
:10BBC000253033750D0A002C253032753A25303476
:10BBD00075004100492C253033692C253033692C00
:10BBE000253033692C253033692C253033690D0A13
:10BBF000002138204572723A20556E6B6E6F776E59
:10BC000020636F6D6D616E642027256325633A257F
:10BC10003258253258270D0A002138204572723AD1
:10BC200020556E6B6E6F776E20636F6D6D616E6405
:10BC3000202725633A253258270D0A002137204551
:10BC400072723A204578747261207061726D61740D
:10BC500065720D0A002136204572723A20496E76CF
:10BC6000616C696420706172616D746572207661C7
:10BC70006C75650D0A002134204572723A204D69B9
:10BC80007373696E6720706172616D657465722887
:10BC900073290D0A002133204572723A2052582030
:10BCA000427566666572206F76657272756E0D0AF2
:10BCB000002132204572723A20545820427566663F
:10BCC0006572206F76657272756E0D0A00213120E3
:10BCD0004572723A2043616E277420737465702038
:10BCE0007468617420666173740D0A002130200D40
:10BCF0000A002008002573001B5B421B5B314B1BB5
:07BD00005B3047000D0A0053
:08BD0800D9CFE6FFDACFE6FF18
:10BD1000E1CFD9FFE2CFDAFF240EE12402E3E168AC
:10BD2000E652E16ED950FA0FE96EFF0EDA20EA6EA4
:10BD3000020EEECFDBFF030EEECFDBFF040EEECFE5
:10BD4000DBFF050EEECFDBFFE8D9F2D976EC66F02B
:10BD5000006E060EE15C02E2E16AE552E16E00501F
:10BD6000E76E0D0EE7CFDBFFDB50800815E0A0D9B2
:10BD70003E6A3F6A406A416A00C039F001C03AF049
:10BD800002C03BF003C03CF056EC5BF0010A10E14E
:10BD9000210E0501F16FF26B020EDB68030EDB680A
:10BDA000040EDB687F0EF36E050EF3CFDBFF66D16A
:10BDB0000D0EDB50050B01E061D10A0EDBCF00F068
:10BDC0000B0EDBCF01F0830E0026FF0E012200C018
:10BDD000DEFF01C0DDFFD950060F65D976D9DF50EF
:10BDE000010B0FE0DF06010E01E2DB06D950180F50
:10BDF0005AD9D890EF36010EEB36020EEB36030E11
:10BE0000EB36D9CFE9FFDACFEAFF020E3F6E406A88
:10BE1000EECF3AF0EDCF3BF030EC5BF03AC0EEFF06
:10BE20003BC0EDFF140EDB6A150EDB6A160EDB6AF3
:10BE3000170EDB6A1C0EDB6A1D0EDB6A1E0EDB6A48
:10BE4000010EF36E1F0EF3CFDBFF010EF36E0E0E2D
:10BE5000F3CFDBFF0F0EDB6A0E0EDBCF00F00F0E11
:10BE6000DBCF01F0D890015004E61A0E005C000E02
:10BE7000015801E398D0180EDBCF00F0190EDBCF8C
:10BE800001F01A0EDBCF02F01B0EDBCF03F0010E28
:10BE90001F0B07E0D8900036013602360336E8065D
:10BEA000F9E1180E00C0DBFF190E01C0DBFF1A0E0E
:10BEB00002C0DBFF1B0E03C0DBFF140EDBCF08F05C
:10BEC000150EDBCF09F0160EDBCF0AF0170EDBCF15
:10BED0000BF0010E1F0B07E0D890083609360A3622
:10BEE0000B36E806F9E1D9501C0FDDD80850EE24D6
:10BEF000046E0950EE20056E0A50EE20066E0B50BF
:10BF0000EE20076ED950180FCED80450EE5C006EAC
:10BF10000550EE58016E0650EE58026E0750EE586E
:10BF2000036E200E00C0DBFF210E01C0DBFF220EDE
:10BF300002C0DBFF230E03C0DBFF200EDBCF39F096
:10BF4000210EDBCF3AF0220EDBCF3BF0230EDBCF0E
:10BF50003CF03C34000E3C1809E6D880000E395401
:10BF6000000E3A54000E3B54000E3C5411E2D950DE
:10BF7000200F99D8AAD8D8D81C0EDB50EE121D0E6F
:10BF8000DB50EE121E0EDB50EE121F0EDB50EE12D7
:10BF9000D9501C0F88D8AFD80E0EDB2A0F0E01E245
:10BFA0005BD7DB2A59D7C9D8100E00C0DBFF110EB2
:10BFB00001C0DBFF180EDBCF3AF0190EDBCF3BF0F0
:10BFC000120E3AC0DBFF130E3BC0DBFFADD893D897
:10BFD000D950100F68D8EE50ED1012E0D950120F62
:10BFE00062D8EE50ED1006E1A8D800500110021002
:10BFF000031006E099D8EE2A000EEE22EE22EE2281
:10C000000C0EDB6A91D8060EEECFDBFF070EEECFEB
:10C01000DBFF080EEECFDBFF090EEECFDBFF7E0E5F
:10C02000F36E0A0EF3CFDBFF0B0EDB6AD950020F63
:10C03000E66E000EDA20E66E70D804EC67F0E5528A
:10C04000E552E552E552DECFE6FFDDCFE6FF70D8E0
:10C05000DAEC65F0006E060EE15C02E2E16AE552A0
:10C06000E16E0050020E38C0DBFF030E39C0DBFF6B
:10C07000040E3AC0DBFF050E3BC0DBFF19D800C041
:10C0800038F001C039F002C03AF003C03BF0240E92
:10C09000E15C02E2E16AE552E16EE552E5CFDAFFEA
:10C0A000E7CFD9FF1200E96E000EDA20EA6E120027
:10C0B000020EDBCF00F0030EDBCF01F0040EDBCF6E
:10C0C00002F0050EDBCF03F01200180EEECFDBFFFF
:10C0D000190EEECFDBFF1A0EEECFDBFF1B0EEECFFD
:10C0E000DBFF1200EECFE6FFEECFE6FFEECFE6FF7E
:10C0F000EFCFE6FF1200D890030EEB32020EEB32C8
:10C10000010EEB32EF321200EE500016EE50011627
:10C11000EE500216EE5003161200D950060FE66ECE
:10C12000000EDA20E66E1200D950140F53EF60F0C3
:10C13000D950020FB8DF72EF60F0010E006E016A95
:0AC14000026A036AF1DF84EF60F089
:06C14A00040130511F0B3F
:10C15000010801E012003051600BE842E842E84279
:10C16000E842E842010801E01200345103E03405DE
:10C1700001E012003151220A31E0030A24E0010AF1
:10C1800015E0210A0DE0010A01E012000401A00EF1
:10C190008D6F070E8E6F080E906F916B8F8121D07F
:10C1A0000401A00E8D6F070E8E6F1BD036C495F460
:10C1B00037C496F40401800E926F070E936F976B4D
:10C1C000986B948F12000401800E8D6F070E8E6F96
:10C1D000070E906F916BC10E8F6F120032C49BF7E8
:10C1E00004018F8F12000701806B4B0E816F826BF1
:10C1F000836B846B856B080E866F8F6B1A0EE66EF1
:10C20000010EE66E31EC4DF0E552E5521E0EE66E83
:10C21000020EE66E31EC4DF0E552E5522FD902E206
:10C22000E16AE5524FD90701996B9A6B906B120046
:10C230001CD982D9050E3A1801E13B5002E0000EEC
:10C2400018D051D907019751001808E198510118E9
:10C2500005E114D902E2E16AE55234D944D9070173
:10C260009951001805E19A51011802E1906B956B04
:10C27000010E0CD1FAD807018F6B9751981102E18A
:10C28000000E05D045D9EF50800B01E0010E0009EA
:10C2900031E1FB0EDBCF00F03BD9EE52EF50D880FE
:10C2A000005405E235D9EE52FB0EEFCFDBFF8F6B6A
:10C2B000FB0EDB508F5D19E28F51EA6A400FE96E89
:10C2C000070EEA22EF50E66E8F51E76EFC0EDBCFD1
:10C2D000E9FFFD0EDBCFEAFFE750E926000EEA2278
:10C2E000E552E750EF6E8F2BE3D7C8D802E2E16A40
:10C2F000E552E8D807018F51C9D0B7D8070190514E
:10C3000007E1E7D8FB0EDBCF95F7010E966F906F34
:10C31000BDD00BD917E1C0D8EDD802E101500BE038
:10C32000010EDBCFE9FFDB2A020EDBCFEAFF01E3E0
:10C33000DB2AEF50F1E1CDD8DFCF95F70701010EF1
:10C34000966F906FE552E552E552A0D0EED818E115
:10C35000A3D8D0D802E101500CE0010EDBCFF6FFEC
:10C36000DB2A020EDBCFF7FF01E3DB2A0800F550E2
:10C37000F0E1AFD8DFCF95F70701966B010E906F14
:10C38000E552E552E55282D070D8E652E6520701F6
:10C3900099519A1102E1000E08D099C7E9FF9AC796
:10C3A000EAFFEF50800B01E0010E00095BE1030E94
:10C3B000905D01E1906B905155E0020E905D0DE1B2
:10C3C000E66A000EE66EE66A8BD802E2E16AE552A2
:10C3D00098D80701030E906F45D0900543E1400EB9
:10C3E000006E016A9551005C000E015803E2400E98
:10C3F000DF6E02D095C7DFFFDF50955D956F000EB1
:10C40000936F070E946F010EDFCFDBFF96510BE1A8
:10C41000010EDB5012E091C7F6FF92C7F7FF08004C
:10C42000F55043D8F5D7010EDB5007E091C7E9FF7F
:10C4300092C7EAFFEF5039D8F6D70701955107E1C7
:10C44000400EDF5C02E1020E01D0030E906FDFCFE1
:10C45000E6FF000EE66E070EE66E42D802E2E16AE3
:10C46000E5524FD8E552E55211D0D9CFE6FFDACFE9
:10C47000E6FFE1CFD9FFE2CFDAFF1200400EE66E11
:10C48000400EE66E070EE66EE66A47D0E552E5CF4F
:10C49000DAFFE7CFD9FF1200DF6A4ED8DE523AC08A
:10C4A000DEFF3BC0DDFFDD52120093C7E9FF94C7FA
:10C4B000EAFFEF6E932B000E9423912B9223010E33
:10C4C000DB061200E16E0050F3CF97F7F4CF98F738
:10C4D0001200FC0EDBCF91F7FD0EDBCF92F71200BE
:10C4E000010EE66E1AD0FA0EDBCF00F0FB0EDBCFAA
:10C4F00001F01200DF2ADF50006E016AFF0E001803
:10C500001200E16E0050F3CF99F7F4CF9AF71200C2
:10C5100097C7E9FF98C7EAFF1200020EE66E50ECDB
:10C520004DF0006E050EE15C12009FDFE652E65210
:10C53000E652070190511200FC0EDBCF3AF0FD0EDF
:06C54000DBCF3BF012000E
:0AC546006AD9E6520E01006BA96BE2
:10C55000DF6A180EDF5C14E283D9010EE9260E0EA5
:10C5600085D9DF5077D9EF6A7BD9490EE9260E0EBF
:10C570007DD976D9790EE9260E0E78D9DF2AE9D74A
:10C580000E01C60EAC6F0E0EAD6F3F0E7914000992
:10C59000796ECF0E79140009796E79827B6A7A6A96
:10C5A00079900F0152815293F00EB4140909B46EC0
:10C5B0000E01080EAA6F030EAB6F800EAE6F3E0E1B
:10C5C000AF6FE00EB06F2E0EB16F040EB66F900E0F
:10C5D000B26F010EB36F900EB46F010EB56F000E07
:10C5E000E66EE66A010EE66EDFEC31F0E552E552EA
:10C5F000E552E55229D112D9E652DF6A180EDF5C06
:10C600000AE2DF5027D9EFCF00F0FD0EDB50005CCF
:10C610000AE0DF2AF3D7DF6A180EDF5C08E2DF509A
:10C6200019D9EF5002E1DF2803D0DF2AF5D7000E39
:10C63000E5520AD1F3D8070EE12402E3E168E6529D
:10C64000E16EDE6ADD6A020EDB6A030EDB6A040E4F
:10C65000DB6A050EDB6A060EDB6A010EE66ED9CFD9
:10C66000E6FFDACFE6FF030EE2D8020F03D9010E90
:10C67000DED8030FFFD8030EDAD8050FFBD8030E60
:10C68000FED80701B45124E1020EDB50180802E283
:10C69000B48D1ED0050EDBCFE6FF060EDBCFE6FF26
:10C6A000030EDBCFE6FF040EDBCFE6FF020EDBCF8F
:10C6B000E6FFDECFE6FFDDCFE6FF11D8006E070E06
:10C6C000E15C02E2E16AE552E16E005097EC40F075
:10C6D000070EE15C02E2E16AE552E16EB5D09ED858
:10C6E000E652E652FB0EDBCFE6FF85DFE552E76E52
:10C6F000010EE7CFDBFFDB5002E1000E8CD0D950FA
:10C70000FC0FE96EFF0EDA20EA6EEE50ED101FE12D
:10C71000010EDB049FD8EF500E01EA6AAC25E96EEA
:10C72000AD51EA22EF6A88D8790EE9260E0E9ED81E
:10C7300083D8490EE9260E0E99D8010EDB048AD85B
:10C74000EF6A7AD8010EE9260E0E90D862D0010E5B
:10C75000DB04006E0E01AA51005C5BE2FB0EDB50B5
:10C76000180857E3FB0EDB50070802E10501E36BF5
:10C7700063D8010EE9260E0EEA22EE50ED1010E10C
:10C78000E66AFB0EDBCFE6FF87EC49F0E552E552A7
:10C79000E66AFB0EDBCFE6FF59EC49F0E552E552C5
:10C7A00005012751FDE00501030E346FF70EDBCFC5
:10C7B0004EF5F80EDBCF4FF5506B516B190E3D6EF9
:10C7C0003E6A3F6A406A4EC538F04FC539F050C5E1
:10C7D0003AF051C53BF080EC69F034C04EF535C0FD
:10C7E0004FF536C050F537C051F5010EDBCF55F58A
:10C7F000FB0EDBCF54F5FC0EDBCF52F5FD0EDBCF8D
:10C8000053F5F90EDBCF56F5FA0EDBCF57F50501E0
:10C81000276B010EDB50E552E55216D0D9CFE6FF6B
:10C82000DACFE6FFE1CFD9FFE2CFDAFF120027D857
:10C83000010EE66ED9501200010EDB04E96EEA6AC1
:10C84000D890E936EA361200E552E5CFDAFFE7CFB5
:10C85000D9FF1200EA6A310FE96E0E0EEA221200C9
:10C86000EA6ADF34FE0BEA36E96E1200EA22EE6A6B
:10C87000ED6A1200E66E000EDA20E66E1200E66E39
:0EC880002CEC47F0E552E552E552E55212006D
:02C88E00D9CF00
:10C89000E6FFDACFE6FFE1CFD9FFE2CFDAFF060EFF
:10C8A000E12402E3E168E652E16EDF6A010EDB6A31
:10C8B000D950FA0FE96EFF0EDA20EA6E020EEECFC3
:10C8C000DBFF030EEECFDBFF040EEECFDBFF050E2A
:10C8D000EECFDBFFD950FA0FE96EFF0EDA20EA6ED9
:10C8E000060EE76ED890030EEB32020EEB32010E0D
:10C8F000EB32EF32E706F6E1D950FA0FE96EFF0EA0
:10C90000DA20EA6E060EE76ED890EF36010EEB36AF
:10C91000020EEB36030EEB36E706F6E1D950FA0FBE
:10C92000E96EFF0EDA20EA6E400EEE26000EEE22D1
:10C93000000EEE22000EEE22FA0EDBCF04F0FB0E0C
:10C94000DBCF05F0FC0EDBCF06F0FD0EDBCF07F0F2
:10C95000D950020FE96E000EDA20EA6EEE50045C48
:10C96000006EEE500558016EEE500658026EEE5005
:10C970000758036E0050DF6ED950F80FE96EFF0EB6
:10C98000DA20EA6EEE50ED1065E0040EDB50F86E32
:10C99000030EDB50F76E020EDB50F66EDF50DF0643
:10C9A00000091AE0F60EDBCFE9FFDB2AF70EDBCF3A
:10C9B000EAFF01E3DB2AEF50F56E0D00F80EDB060F
:10C9C000DBCF00F0F90E01E2DB06DBCF01F0005017
:10C9D000011001E101D0E2D7040EDB50F86E030E26
:10C9E000DB50F76E020EDB50F66EA684F2AE04D07A
:10C9F000F29EDE52010EDD6E550EA76EAA0EA76ED8
:10CA0000A682A694010EDB5003E0F28E010EDB6AD3
:10CA1000400EDF6E400E006E016A026A036AD95052
:10CA2000020FE96E000EDA20EA6EEE500026EE509C
:10CA30000122EE500222EE500322020E00C0DBFF64
:10CA4000030E01C0DBFF040E02C0DBFF050E03C0B6
:10CA5000DBFF92D7060EE15C02E2E16AE552E16E8D
:0CCA6000E552E5CFDAFFE7CFD9FF120066
:04CA6C0005D873EC8A
:10CA70004CF02DEC3CF0FBD78ED8E652E6520F017D
:10CA800048694969600ED36E9B8C580EDE6E020EAB
:10CA9000DD6EDFCF00F0DF06010EDBCF01F001E23B
:10CAA000DB0600500110F5E1948E62EC3BF009ECDE
:10CAB0004CF0E552E55278D012001200120012003C
:10CAC000A5EF60F01200F3EF60F004019B051EE19A
:10CAD00004019C051BE1F1DF659204019C6B0501DB
:10CAE000100EEF6F0E0EF06FEF07000EF05BEF51C0
:10CAF000F011FAE16584080EEF6F070EF06FEF0793
:10CB0000000EF05BEF51F011FAE16594120043D88A
:10CB1000FC0EDBCF3AF0FD0EDBCF3BF0050E3A18F2
:10CB200001E13B5036E0E8683A1802E17F0E3B181D
:10CB30002FE0030E3A1801E13B5028E0020E3A18AC
:10CB400001E13B5021E0010E3A1801E13B501AE0AF
:10CB5000740E3A1801E13B5013E0750E3A1801E1EA
:10CB60003B500CE0730E3A1801E13B5005E0720EA9
:10CB70003A180FE13B500DD0A1DF0BD09DDF09D05B
:10CB80009CDF07D0A0DF05D09DDF03D099DF01D067
:10CB900096DF010E09D0D9CFE6FFDACFE6FFE1CF6D
:10CBA000D9FFE2CFDAFF1200E552E5CFDAFFE7CF97
:04CBB000D9FF120097
:0CCBB40096D8E1CFD9FFE2CFDAFF0C0EDB
:10CBC000E12402E3E168E652E16ED950FA0FE96E22
:10CBD000FF0EDA20EA6E080EEECFDBFF090EEECF75
:10CBE000DBFF0A0EEECFDBFF0B0EEECFDBFF79D8BB
:10CBF000D950080FE96E000EDA20EA6EEECFE6FF9C
:10CC0000EECFE6FFEECFE6FFEFCFE6FF76EC66F085
:10CC1000006E060EE15C02E2E16AE552E16E005050
:10CC2000E76E070EE7CFDBFFDB50840B3AE1070E20
:10CC3000DB041AE1060EDB5006E0006A016A026AB4
:10CC4000800E036E04D0006A016A026A036A080E4D
:10CC500000C0DBFF090E01C0DBFF0A0E02C0DBFFD4
:10CC60000B0E03C0DBFF1DD0F80EDBCF00F0F90E7A
:10CC7000DBCF01F0D950040FE96E000EDA20EA6E26
:10CC80000050EE260150ED22D950080FE66E000E3E
:10CC9000DA20E66E26D804EC67F0E552E552E5525C
:10CCA000E552080EDBCF00F0090EDBCF01F00A0ED3
:10CCB000DBCF02F00B0EDBCF03F000C038F001C079
:10CCC00039F002C03AF003C03BF00C0EE15C02E226
:10CCD000E16AE552E16EE552E5CFDAFFE7CFD9FF31
:0CCCE0001200D9CFE6FFDACFE6FF120009
:04CCEC00D9CFE6FFB7
:10CCF000DACFE6FFE1CFD9FFE2CFDAFFE6520068F4
:10CD000001687F0E026E036AD950FA0FE96EFF0EBA
:10CD1000DA20EA6EEE500016EE500116EE500216C2
:10CD2000EE5003166AD800C0EEFF01C0EEFF02C04D
:10CD3000EEFF03C0EEFFFD0EDB50800B02E0010EA4
:10CD400001D0000EE66E59D8060EE926000EEA2242
:10CD5000E552E750EF6EFC0EDBCF00F0FD0EDBCFAF
:10CD600001F0D89000360136FC0E00C0DBFFFD0E4E
:10CD700001C0DBFFDB50E66E40D8040EE926000E52
:10CD8000EA22E552E750EE6EED6AFD0EDB50006ED2
:10CD9000016AFF0E001818E1015016E12ED8EECFFF
:10CDA00000F0EECF01F0EECF02F0EFCF03F0005035
:10CDB00001100210031006E0210E0501F16FF26B65
:10CDC000800E0BD0040E09D0FD0EDB5008E115D803
:10CDD000EE6AEE6AEE6AEE6A010EDF6E06D0020EB1
:10CDE000DF6E0BD8EE52EE52EE8EDF50E552E5527A
:10CDF000E5CFDAFFE7CFD9FF1200F80EDBCFE9FF6E
:08CE0000F90EDBCFEAFF12007E
:08CE0800D9CFE6FFDACFE6FF07
:10CE1000E1CFD9FFE2CFDAFF5BD8013411E2005055
:10CE2000FE08000E01540CE276D805E06CD8800EA6
:10CE3000EE6EEE6847D067D8800EEE6E7F0E0ED095
:10CE400047D8D890015004E6010E005C000E01584E
:10CE50000BE261D805E057D8EE6A800EEE6E32D054
:10CE600052D8EE6AEE6A2ED047D8EECF00F0EECF61
:10CE700001F0EECF02F0EFCF03F032D800C0EEFFAA
:10CE800001C0EEFF02C0EEFF03C0EEFF21D800504C
:10CE9000010B05E025D8020E3AD8EF8E04D020D839
:10CEA000020E35D8EF9E14D8D8900132003218D82F
:10CEB000030E2DD800C0EFFF1AD804E011D8030EDE
:10CEC00026D8EF8EE552E5CFDAFFE7CFD9FF120083
:10CED00013D8040E1CD8EECF00F0EFCF01F01200F3
:10CEE000FA0EDBCFE9FFFB0EDBCFEAFF120004D81E
:10CEF000060E0DD8EF501200FC0EDBCFE9FFFD0E41
:10CF0000DBCFEAFF1200ECDFEE6AEE6A1200E926E0
:10CF1000000EEA221200220E0501F16FF26B77EF8C
:02CF200067F0B8
:0ECF2200D9CFE6FFDACFE6FFE1CFD9FFE2CFAD
:10CF3000DAFFE652E652E652E652E652DF6AD9508E
:10CF4000FA0FE96EFF0EDA20EA6E010EEECFDBFF7C
:10CF5000020EEECFDBFF030EEECFDBFF040EEECFB3
:10CF6000DBFFF60EDBCF00F0F70EDBCF01F0F80EA3
:10CF7000DBCF02F0F90EDBCF03F048D80050EE5CB7
:10CF80000150EE580250EE580350EE5833E2030EB3
:10CF9000DB50F86E020EDB50F76E010EDB50F66EC2
:10CFA000A684A688F2AE03D0F29E010EDF6E550E67
:10CFB000A76EAA0EA76EA682DF5001E0F28E006A6D
:10CFC000040E016E026A036A21D8EE500026EE506C
:10CFD0000122EE500222EE500322010E00C0DBFFC0
:10CFE000020E01C0DBFF030E02C0DBFF040E03C014
:10CFF000DBFFB7D7050EE15C02E2E16AE552E16EC4
:10D00000E552E5CFDAFFE7CFD9FF1200D950010F83
:0AD01000E96E000EDA20EA6E12004D
:06D01A002A0EF66E100E56
:10D02000F76E000EF86E05010900F550EA6F090071
:10D03000F550EB6F03E1EA6701D03DD00900F550F0
:10D04000E56F0900F550E66F0900F550E76F09003C
:10D050000900F550E96E0900F550EA6E0900090073
:10D060000900F550E86F0900F550E96F0900090063
:10D07000F6CFECF5F7CFEDF5F8CFEEF5E5C5F6FF19
:10D08000E6C5F7FFE7C5F8FF0501E85302E1E953FC
:10D0900007E00900F550EE6EE807F8E2E907F9D776
:10D0A000ECC5F6FFEDC5F7FFEEC5F8FF0501EA0791
:08D0B000000EEB5BBFD712007C
:08D0B800FE0EE3CFE9FFFF0EBD
:10D0C000E3CFEAFFE9CFF3FFEACFF4FFFB0EE35033
:10D0D00003E1FC0EE35009E0FB0EE30602E2FC0E66
:10D0E000E306FD0EE350EE6EF1D71200FE0EE3CF25
:10D0F000E9FFFF0EE3CFEAFFF36AF46AEE5203E0C2
:10D10000F34AF42AFBD71200FF0EE3CFF8FFE552F3
:10D11000FF0EE3CFF7FFE552FF0EE3CFF6FFE55238
:10D12000E66AE66AE66A0900F55209E0FD0EE32ABE
:10D1300005E1FE0EE32A02E1FF0EE32AF4D7FD0E1D
:10D14000E3CF39F0FE0EE3CF3AF0FF0EE3CF3BF032
:02D150001200CB
:0ED15200D9CFE6FFDACFE6FFE1CFD9FFE2CF7B
:10D16000DAFFE652E652E652E652D950FB0F006E65
:10D17000FF0EDA20016E00C0DEFFDD6EDECFE6FFBF
:10D18000DDCFE6FFFB0EDBCFE6FFFC0EDBCFE6FFDD
:10D19000FD0EDBCFE6FFF3C5E6FFF4C5E6FFF1ECDD
:10D1A00052F0006E070EE15C02E2E16AE552E16EC8
:10D1B0000050020EF3CFDBFF030EF4CFDBFF020EB5
:10D1C000DBCF00F0030EDBCF01F000C0F3FF01C0A6
:10D1D000F4FF040EE15C02E2E16AE552E16EE55221
:0AD1E000E5CFDAFFE7CFD9FF120018
:06D1EA00D9CFE6FFDACF09
:10D1F000E6FFE1CFD9FFE2CFDAFFE652E652E65290
:10D20000E652D9CFE9FFDACFEAFFFA0EDBCFEEFF25
:10D21000FB0EDBCFEEFFFC0EDBCFEEFFFD0EDBCF18
:10D22000EEFF020EDB50F86E010EDB50F76EDF50A2
:10D23000F66EF80EDBCF00F0DB06F90EDBCF01F067
:10D2400001E2DB06005001100DE00900F60EDBCF15
:10D25000E9FFDB2AF70EDBCFEAFF01E3DB2AF5CF9C
:10D26000EFFFE7D7040EE15C02E2E16AE552E16E0E
:0CD27000E552E5CFDAFFE7CFD9FF12004E
:04D27C00D9CFE6FF21
:10D28000DACFE6FFE1CFD9FFE2CFDAFFFB0EDBCF4B
:10D2900000F0FC0EDBCF01F00001800E01141AE15A
:10D2A000FB0EDBCFE9FFFC0EDBCFEAFFEECFF3FF97
:10D2B000EDCFF4FFEE2A000EEF22F3CFE9FFF4CF1B
:10D2C000EAFFFD0EDBCFEFFFEF50016AF36E01C006
:10D2D000F4FF10D0FB0EDB50FE0806E1FD0EDBCFA5
:10D2E000E6FF7DEC6AF005D0FD0EDBCFE6FFA1EC9A
:10D2F0003DF0E552E552E5CFDAFFE7CFD9FF120066
:10D3000038503D02F3CF34F0F4CF35F03E02F35005
:10D310003526000EF420366E38503F02F350362684
:10D32000000EF420376E38504002F3503726395043
:10D330003D02F3503526F4503622000E3722395084
:10D340003E02F3503626F450372239503F02F35054
:10D3500037263A503D02F3503626F45037223A50E1
:10D360003E02F35037263B503D02F3503726120061
:10D370001201000202000040D80492FD8201010265
:10D38000000109024300020100C03209040000014B
:10D3900002020100052400100104240202052406F3
:10D3A00000010524010001070581030800020904AA
:10D3B0000100020A00000007050202400000070504
:07D3C000820240000082D34D
:08D3C800FF0EE124E96EFF0EE7
:10D3D000E220EA6EEDCFF4FFEFCFF3FFF46607D063
:10D3E000600EF36404D07B0EF36001D0F39A120058
:10D3F000F36AF46AFF0EE124E96EFF0EE220EA6EA2
:10D40000ED6607D02F0EEF6404D03A0EEF6001D026
:04D41000F32A1200E9
:0CD41400376A366A356A346A200EE76E0B
:10D42000D890383639363A363B3634363536363695
:10D4300037363D50345C3E5035583F50365840509A
:10D44000375809E33D50345E3E50355A3F50365A06
:0CD450004050375A382AE72EE4D712006B
:04D45C004F4B0D0A1B
:10D46000000D0A004542427631335F616E645F61B0
:10D47000626F7665204542204669726D77617265FC
:10D480002056657273696F6E20322E352E340D0A68
:01D49000009B
:0ED49200376A366A100EE76ED8903A363B368F
:10D4A000363637363F50365C4050375805E33F50EC
:0ED4B000365E4050375A3A2AE72EF0D7120067
:02D4BE00C00E9E
:10D4C000F36E00EE00F00E0E01D81200EA6002D0FA
:0ED4D000EE6AFCD7F350E9601200EE6AFCD75A
:02D4DE001DEE41
:10D4E00000F02DEE00F0F86A439C0DEC68F09FEC24
:0AD4F0006AF036EC65F0FBD712007D
:06D4FA00FF0EE350ADBA85
:10D5000004D0B06AAC8EAD8A949CADA2FED7AE6E4C
:06D51000F36EF46A120044
:0AD51600F36AF46AF32A0F0B05E034
:0CD52000D890F336F436E804FBE112006A
:04D52C003031323335
:0DD530003435363738396162636465660052
:02D53E001200D9
:10D540000403090418035300630068006D006100C0
:10D550006C007A00480061007500730038034500D4
:10D56000690042006F00740042006F0061007200A9
:10D5700064002C000000000000000000000000001B
:10D58000000000000000000000000000000000009B
:0AD5900000000000800284029C02EB
:02D59A00FEFF92
:04D59C00000000008B
:05D5A000000000000185
:0BD5A50000000000000000000000007B
:10D5B000000000000000000000000000000000006B
:10D5C000000000000000000000000000000000005B
:10D5D000000000000000000000000000000000004B
:10D5E000000000000000000000000000000000003B
:10D5F000000000000000000000000000000000002B
:10D60000000000000000000000920F920F920F93A4
:10D610000F930F930F930F930F930F930F930F94F9
:10D620000F940F940F940F940F940F940F940F95E1
:10D630000F950F950F950F950F950F890F890F89EE
:10D640000F8A0F8A0F8A0F8A0F8A0F8A0F8A0F8A12
:10D650000F8B0F8B0F8B0F8B0F8B0F8B0F8B0F8BFA
:10D660000F8C0F8C0F8C0F8C0F8C0F8C0F00010503
:10D670000001020304050607000102030405060772
:06D6800002030405060789
:00000001FF
